:020000040000FA
:1000000000040020E90800007D050000C908000088
:1000100087050000910500009B050000000000001E
:100020000000000000000000000000000D090000BA
:10003000A505000000000000AF050000B9050000A4
:10004000C3050000CD050000D7050000E105000054
:10005000EB050000F5050000FF05000009060000A3
:10006000130600001D0600002706000031060000F0
:100070003B060000450600004F0600005906000040
:10008000630600006D060000770600008106000090
:100090008B060000950600009F060000A9060000E0
:1000A000B3060000BD060000C7060000D106000030
:1000B000DB060000E5060000EF060000F906000080
:1000C000030700000D0700001707000021070000CC
:1000D0002B070000350700003F070000490700001C
:1000E000530700005D07000067070000710700006C
:1000F0007B070000850700008F07000099070000BC
:10010000A30700001FB500F003F88DE80F001FBD26
:1001100000F0E0BB1FB56FF00100009040100390AD
:10012000029001904FF010208069000B420900F00E
:100130001F045DF822300120A04083434DF8223097
:10014000684600F045F91FBDF0B54FF6FF734FF458
:10015000B4751A466E1E11E0A94201D3344600E080
:100160000C46091B30F8027B641E3B441A44F9D14B
:100170009CB204EB134394B204EB12420029EBD17E
:1001800098B200EB134002EB124140EA0140F0BD8F
:10019000DE4992B00446D1E90001CDE91001FF2209
:1001A0004021684600F03CFB94E80F008DE80F000A
:1001B000684610A902E004C841F8042D8842FAD12B
:1001C00010216846FFF7C0FF1090AA208DF8440068
:1001D000FFF7A0FF00F0F3F84FF01024A069102201
:1001E0006946803000F002F9A069082210A900F0E9
:1001F000FDF800F0D8F84FF080510A6949690068AD
:100200004A43824201D8102070470020704710B541
:10021000D0E900214FF0805002EB8103026944696C
:100220006243934209D84FF01022536903EB8103D4
:100230000169406941438B4201D9092010BD5069D1
:10024000401C01D0002010BD0F2010BD70B501680A
:100250000446AF4D4FF01020072952D2DFE801F0DD
:10026000330419293C1E2500D4E902656468294637
:10027000304600F0CDF82A462146304600F0B6F868
:10028000AA002146304600F09FFA002800D0032043
:1002900070BD00F051FB4FF4805007E0201DFFF7C8
:1002A000AAFF0028F4D100F047FB60682860002016
:1002B00070BD241D94E80700920000F085FA002824
:1002C000F6D00E2070BD8069401C12D0201DFFF7B3
:1002D0009EFF0028F6D109E08069401C09D0201D4E
:1002E000FFF789FF0028EDD1606820B12046FFF7B5
:1002F0004FFF042070BDFFF70DFF00F060F800F025
:1003000052F8072070BD10B50C46182802D0012005
:10031000086010BD2068FFF799FF206010BD4FF006
:100320001024A069401C05D0A569A66980353079E4
:10033000AA2808D06069401C2DD060690068401C64
:1003400029D060692CE010212846FFF7FDFE3168B6
:1003500081421CD1A16901F18002C03105E030B1B8
:1003600008CA51F8040D984201D1012000E0002094
:100370008A42F4D158B1286810B1042803D0FEE7AE
:10038000284600F057F862496868086008E000F005
:1003900016F800F008F84FF480500168491C01D0AD
:1003A00000F0A4FAFEE7BFF34F8F5A4801685A4A9B
:1003B00001F4E06111430160BFF34F8FFEE74FF09E
:1003C00010208169491C02D0806900F0AEB87047E6
:1003D000524A01681160121D416811604F4A8168DC
:1003E00010321160111DC068086070472DE9F0419E
:1003F00017460D460646002406E03046296800F000
:10040000A7F8641C2D1D361DBC42F6D3BDE8F08153
:1004100070B50C4605464FF4806608E0284600F0AB
:1004200084F8B44205D3A4F5806405F58055002C0A
:10043000F4D170BD4168044609B1012500E00025F2
:100440004FF010267069A268920000F0BDF9C8B1A3
:10045000204600F01AF89DB17669A56864684FF4EB
:10046000002084420AD2854208D229463046FFF74E
:10047000CFFF2A4621463046FFF7B8FFFFF79FFF20
:10048000FFF791FFFFF746FEF8E72DE9FF414FF038
:100490001024616980680D0B01EB800000F6FF708D
:1004A000010B0020009001900290024603906846E4
:1004B00001230BE0560902F01F0C50F8267003FAD6
:1004C0000CFC47EA0C0740F82670521CAA42F1D3F4
:1004D0000AE04A0901F01F0650F8225003FA06F616
:1004E000354340F82250491C8029F2D3A169090BF9
:1004F0004A0901F01F0150F822408B409C4340F80C
:100500002240FFF765FFBDE8FF8100005C090000A5
:10051000000000200CED00E00400FA050006004099
:10052000144801680029FCD07047134A0221116069
:1005300010490B68002BFCD00F4B1B1D186008687E
:100540000028FCD00020106008680028FCD070470C
:10055000094B10B501221A60064A1468002CFCD021
:10056000016010680028FCD0002018601068002886
:10057000FCD010BD00E4014004E5014008208F4993
:1005800009680958084710208C4909680958084724
:1005900014208A49096809580847182087490968BA
:1005A0000958084730208549096809580847382004
:1005B00082490968095808473C2080490968095858
:1005C000084740207D4909680958084744207B496D
:1005D00009680958084748207849096809580847B0
:1005E0004C20764909680958084750207349096822
:1005F0000958084754207149096809580847582084
:100600006E490968095808475C206C49096809580F
:100610000847602069490968095808476420674904
:100620000968095808476820644909680958084753
:100630006C20624909680958084770205F490968B9
:100640000958084774205D49096809580847782007
:100650005A490968095808477C20584909680958C7
:10066000084780205549096809580847842053499C
:1006700009680958084788205049096809580847F7
:100680008C204E4909680958084790204B49096851
:10069000095808479420494909680958084798208B
:1006A00046490968095808479C204449096809587F
:1006B0000847A0204149096809580847A4203F4934
:1006C000096809580847A8203C490968095808479B
:1006D000AC203A49096809580847B02037490968E9
:1006E00009580847B4203549096809580847B8200F
:1006F0003249096809580847BC2030490968095837
:100700000847C0202D49096809580847C4202B49CB
:10071000096809580847C82028490968095808473E
:10072000CC202649096809580847D0202349096880
:1007300009580847D4202149096809580847D82092
:100740001E49096809580847DC201C4909680958EE
:100750000847E0201949096809580847E420174963
:10076000096809580847E8201449096809580847E2
:10077000EC201249096809580847F0200F49096818
:1007800009580847F4200D49096809580847F82016
:100790000A49096809580847FC20084909680958A6
:1007A00008475FF480700549096809580847000048
:1007B00003480449024A034B704700000000002030
:1007C000680900006809000040EA010310B59B07B2
:1007D0000FD1042A0DD310C808C9121F9C42F8D0AB
:1007E00020BA19BA884201D9012010BD4FF0FF305C
:1007F00010BD1AB1D30703D0521C07E0002010BD72
:1008000010F8013B11F8014B1B1B07D110F8013BFD
:1008100011F8014B1B1B01D1921EF1D1184610BDDE
:1008200002F0FF0343EA032242EA024200F005B865
:100830007047704770474FF000020429C0F01280E3
:1008400010F0030C00F01B80CCF1040CBCF1020F83
:1008500018BF00F8012BA8BF20F8022BA1EB0C0158
:1008600000F00DB85FEAC17C24BF00F8012B00F84E
:10087000012B48BF00F8012B70474FF0000200B574
:10088000134694469646203922BFA0E80C50A0E8B3
:100890000C50B1F12001BFF4F7AF090728BFA0E861
:1008A0000C5048BF0CC05DF804EB890028BF40F82D
:1008B000042B08BF704748BF20F8022B11F0804F6F
:1008C00018BF00F8012B7047014B1B68DB68184705
:1008D0000000002009480A497047FFF7FBFFFFF7B7
:1008E00011FC00BD20BFFDE7064B1847064A10600B
:1008F000016881F30888406800470000680900002B
:10090000680900001F030000000000201EF0040F13
:100910000CBFEFF30881EFF3098188690238007892
:10092000182803D100E00000074A1047074A126860
:100930002C3212681047000000B5054B1B68054AB1
:100940009B58984700BD00000703000000000020EE
:100950005809000004000000001000000000000022
:0809600000FFFFFF0090D0032F
:10100000A8110020F5EA0100BD2F000067EA0100E9
:10101000BD2F0000BD2F0000BD2F0000000000000C
:101020000000000000000000000000004DEB010087
:10103000BD2F000000000000BD2F0000BD2F0000EC
:10104000B5EB0100BBEB0100BD2F0000BD2F000080
:10105000BD2F0000BD2F0000BD2F0000BD2F0000E0
:10106000C1EB0100BD2F0000BD2F0000C7EB010048
:10107000BD2F0000CDEB0100D3EB0100D9EB010047
:10108000BD2F0000BD2F0000BD2F0000BD2F0000B0
:10109000BD2F0000BD2F0000BD2F0000BD2F0000A0
:1010A000BD2F0000DFEB0100BD2F0000BD2F0000B1
:1010B000BD2F0000BD2F0000BD2F0000BD2F000080
:1010C000E5EB0100BD2F0000BD2F0000BD2F00008B
:1010D000BD2F0000BD2F0000BD2F0000BD2F000060
:1010E000BD2F0000BD2F0000BD2F0000BD2F000050
:1010F000BD2F0000BD2F0000BD2F0000BD2F000040
:10110000BD2F0000BD2F000000F002F81DF0DFFC35
:101110000AA090E8000C82448344AAF10107DA4552
:1011200001D11DF0D4FCAFF2090EBAE80F0013F0A4
:10113000010F18BFFB1A43F001031847F8DE010046
:1011400018DF01000A444FF0000C10F8013B13F0C7
:10115000070408BF10F8014B1D1108BF10F8015B10
:10116000641E05D010F8016B641E01F8016BF9D103
:1011700013F0080F1EBF10F8014BAD1C0C1B09D15A
:101180006D1E58BF01F801CBFAD505E014F8016BCC
:1011900001F8016B6D1EF9D59142D6D3704700005E
:1011A0000023002400250026103A28BF78C1FBD870
:1011B000520728BF30C148BF0B6070471FB500F011
:1011C0003DF88DE80F001FBD1EF0040F0CBFEFF3BC
:1011D0000880EFF30980014A1047000011B80000B1
:1011E0008269034981614FF001001044704700009B
:1011F000F511000001B41EB400B511F01DFF01B4DB
:101200000198864601BC01B01EBD0000F0B4404606
:10121000494652465B460FB402A0013001B506486C
:10122000004700BF01BC86460FBC804689469246F7
:101230009B46F0BC70470000091100001DF044BC43
:1012400070B51A4C054609202070A01C00F05FF80C
:101250005920A08029462046BDE8704007F02CBBED
:1012600007F035BB70B50C461149097829B1A0F1DA
:101270006001562908D3012013E0602804D06928B2
:1012800002D043F201000CE020CC0A4E94E80E009C
:1012900006EB8000A0F58050241FD0F8806E284611
:1012A000B047206070BD012070470000080000209A
:1012B0001C00002014EC010010B5044600210120A0
:1012C00000F03DF800210B2000F039F8042119202E
:1012D00000F035F804210D2000F031F804210E2033
:1012E00000F02DF804210F2000F029F80421C84354
:1012F00000F025F80621162000F021F8062115201F
:1013000000F01DF82046FFF79BFF002010BDA5212F
:1013100001807047FFF7A4BF11487047104870471D
:10132000104A10B514680F4B0F4A08331A60FFF7C4
:1013300099FF0C48001D046010BD704770474907B5
:10134000090E002806DA00F00F0000F1E02080F816
:10135000141D704700F1E02080F800147047000071
:1013600003F90042100502400100000130B5FA4DBA
:10137000044610280AD0112C06D02846122CC17819
:1013800006D0132C08D0FFDFEC7030BDFFDFFBE789
:101390001129F9D0FFDFF7E71129F5D0FFDFF3E7D7
:1013A0002DE9F04110F000FB044611F094FC201AE6
:1013B000C5B206200EF094FB044606200EF098FB02
:1013C000211AE54CE078132818D000200F180720C8
:1013D0000EF086FB064607200EF08AFB301A3918FD
:1013E000E07812280CD0002001442078022809D08F
:1013F00000200844281AC0B2BDE8F0810120E5E7CA
:101400000120F1E70120F4E7D34810B5817900F11C
:101410000700490805D00CF079FEBDE8104007F040
:10142000FFB80CF054FEF8E702210EF0B1BB2DE935
:10143000FC411D4690460E460746FFF7F5FF0400A7
:101440000AD02078222804D3A07FC0F34010A842FD
:1014500005D10820BDE8FC8143F20200FAE7ADF8AF
:1014600000703DB101208DF802008DF803608DF809
:10147000048002E000208DF8020068460DF015FCA3
:10148000A07F65F34510A0770020E3E730B5044660
:10149000A1F120000D460A284AD2DFE800F0050736
:1014A0000C1C2328353A3F44FFDF42E020782028F7
:1014B0003FD1FFDF3DE0A8480178032939D0C0784B
:1014C000132836D02078242833D0252831D023285B
:1014D0002FD0FFDF2DE0207822282AD0232828D8FB
:1014E000FFDF26E02078222823D0FFDF21E02078CC
:1014F00022281ED024281CD026281AD0272818D00D
:10150000292816D0FFDF14E02078252811D0FFDF2E
:101510000FE0207825280CD0FFDF0AE0207825286E
:1015200007D0FFDF05E02078282802D0FFDF00E0A9
:10153000FFDF257030BD1FB504466A46002001F06C
:101540005EFCB4B1BDF802204FF6FF700621824266
:1015500001D1ADF80210BDF80420824201D1ADF8EE
:101560000410BDF80810814203D14FF44860ADF873
:10157000080068460DF067F807F052F804B010BD97
:1015800070B514460D46064611F0D6FF58B90DB198
:10159000A54201D90C2070BD002408E056F82400B3
:1015A00011F0CAFF08B1102070BD641CE4B2AC4257
:1015B000F4D3002070BDF0B50024059D10B1A94200
:1015C00003D850E009B90020F0BD0920F0BD055D49
:1015D000D5B1071997F801C0BCF1150F2DD03BDC30
:1015E000BCF1150F38D2DFE80CF037122020262688
:1015F00028282F2F373737373737373737372000F7
:10160000025D22BB641CE4B28C42F9D3DBE7022DFD
:10161000DBD1BD781D70072D01D26D0701D40A20E2
:10162000F0BD157845F0010515E0EF43FF0707E031
:10163000012D07D010E00620F0BD2F07A7F180573D
:10164000002FF5D03046F0BD1578AF0701D50B203F
:10165000F0BD45F002051570055D641C2C44E4B234
:101660008C4202D9B1E74FF448568C42AFD3AAE777
:1016700010B50278540809D0012243F20223012C4C
:1016800007D0022C0DD0032C13D10FE000200870DE
:1016900005E080790324B4EB901F0AD10A70002082
:1016A00010BD8079B2EB901F03D1F7E780798009F4
:1016B000F4D0184610BD284A117C39B1517C02295A
:1016C00008D0032908D043F2022070470146901D3C
:1016D00001F002BC032100E00121017000207047ED
:1016E00038B50C460546694601F0F6FB00280DD1D9
:1016F0009DF80010207861F34700207055F8010F25
:10170000C4F80100A888A4F80500002038BD38B549
:101710001378C0B1022816D010A46D462468009436
:101720004C7905EB9414247864F347031370032871
:101730000ED003F0FE0010700868C2F8010088881F
:10174000A2F8050038BD23F0FE0313700228EED185
:10175000D8B240F00100EEE7C80100200302FF010B
:1017600038B50C460978222901D2082038BDADF8D9
:1017700000008DF8022068460CF010FD06F050FFC6
:10178000050003D121212046FFF780FE284638BD01
:101790001CB500208DF80000CDF80100ADF8050063
:1017A000FE48007C022801D0012000E000208DF8D6
:1017B000070068460CF030FE002800D0FFDF1CBD9B
:1017C0002DE9FF470220F54E8DF804000027B08A6E
:1017D000ADF80600B84643F202094CE001A80EF04D
:1017E0003EF9050006D0B08AA8B3A6F81480ADF87B
:1017F00006803EE0039CA07F01072DD504F1240064
:101800000090A28EBDF80800214604F1360301F0D5
:101810007DFF050005D04D452AD0112D3CD0FFDFBE
:101820003AE0A07F20F00800A077E07F810861F314
:101830000000C10861F34100E07794F8210000F056
:101840001F0084F820002078282826D1292120464E
:10185000FFF71CFE21E014E040070AD5BDF80800A0
:1018600004F10E0101F050FB05000DD04D4510D1E3
:1018700000257F1CFFB202200EF032F9401CB84256
:10188000ACD8052D12D008E0A07F20F00400A0778E
:1018900003E0112D00D0FFDF0025BDF80600B08267
:1018A000052D05D0284604B0BDE8F087A6F81480C1
:1018B0000020F8E770B50646FFF7B6FD054607F0CD
:1018C00079F8040000D1FFDF6680207820F00F0057
:1018D000801C20F0F000203020700620207295F847
:1018E0003E006072BDE8704007F067B82DE9F04730
:1018F00086B0040000D1FFDF2078A84E20F00F0052
:10190000801C20F0F0007030207060680178091FA2
:10191000182931D2DFE801F0FD30303053FC300CB3
:10192000FCFC40FD3030FD76FDFD3030FDFDFBFA66
:1019300086883046FFF778FD0546304608F0E0FB24
:10194000E0B16068807985F83E0021212846FFF7E4
:101950009DFD304603F0CBFF304605F037F93146A8
:10196000022011F09DFDA87F20F01000A877FFF75E
:1019700027FF002800D0FFDF06B095E7207820F091
:10198000F000203020700620207266806068807928
:10199000607207F012F8D8E785882846FFF744FD03
:1019A00000B9FFDF60688078012800D0FFDF606841
:1019B000817906B02846BDE8F04708F07DBF8688EB
:1019C0003046FFF731FD050000D1FFDF06F0F5FFDF
:1019D00060683146C08828816068008968816068D5
:1019E0004089A881022011F05BFD0020A875A87F26
:1019F00000F003000228BFD1FFF7E2FE0028BBD0B1
:101A0000FFDFB9E780783C2803D0002502280AD000
:101A100000E00125002720B13C2802D0022800D098
:101A2000FFDF17B1B3E00127F5E706F0C6FF1DB1F0
:101A3000B07801F022FA9CE06568B5F804A0A879B6
:101A4000AD1C012806D03079814606F055FD07000F
:101A500003D101E0B078F7E7FFDF00220221504612
:101A60000EF08DF8040000D1FFDF22212046FFF7A1
:101A70000DFD2879012800D00220A17F804668F35F
:101A80000101A177288B2081688B6081A88BA081C0
:101A900084F822908DF80880B8680090F86801906A
:101AA0006A46032150460EF06AF800B9FFDFB88895
:101AB000ADF81000B8788DF8120004AA0521504640
:101AC0000EF05DF800B9FFDFB888ADF80C00F878CB
:101AD0008DF80E0003AA042150460EF050F800B90C
:101AE000FFDF062105F1120001F02CFA28B3687916
:101AF000800700D5FFDF6979E07D61F34700E0757D
:101B0000D5F80600A0616889A08303E05CE055E099
:101B10004EE060E0062105F10C0001F013FAB0B1CF
:101B2000B0794108607861F347006070D6F807002B
:101B3000C4F80200B6F80B0012E0E07D20F0FE00D1
:101B4000801CE075D5F81200A061E88ADCE76078B7
:101B500020F0FE00801C6070E868C4F80200288A4B
:101B6000E080B8F1010F04D0B8F1020F0FD0FFDF11
:101B700002E73078032800D0FFDF0021084611F08B
:101B80008FFC06B00120BDE8F04701F045B9F078C0
:101B9000132800D0FFDF0021062001E0C80100204B
:101BA00011F07EFC06B01120BDE8F047FFF7DEBB68
:101BB00006B02046BDE8F04702F030B806F0FDFE62
:101BC000B07C40F0020004E006F0F7FEB07C40F08C
:101BD0000400B074D0E606B0BDE8F04706F0EDBEF4
:101BE0002DE9F04705460078914600270209FB4899
:101BF0000C463E46012A6DD000234FF6FF71022AA3
:101C000069D0072A09D00A2A71D0FFDFA9F800603D
:101C10000CB127806680002046E6D5F804C09CF809
:101C20000060142E7DD010DC04F1080204F11808C5
:101C30000F2E21D004DC042E5AD0082E57D10DE0EF
:101C4000122E6FD0132EF9D11FE0153E072E4ED263
:101C5000DFE806F0C14D4D099FEAB00012271026BB
:101C6000BCF8040014E11C27092694B3BCF8020058
:101C7000A080686800795AE11B2709264CB303202D
:101C8000207268684088A080C0E79CF802003C2869
:101C900027D0102718260CF1020CD4B1BCF8020092
:101CA000A080BCF818006082BCF818002082BCF844
:101CB0001A00A082BCF81C00E0829CF805000CF120
:101CC0000601FFF724FD9CF8040028B10120E07311
:101CD0009CE703E0BFE0DFE00220F8E7A9F800603E
:101CE00099E71B270926002CF8D023728EE720E104
:101CF0001D273726002CF1D0A18069680879491D7D
:101D0000FFF705FD686890F82B00A0756868C0783B
:101D10000428E07D16D020F00100E0756968C978DC
:101D200001E06DE011E061F34200E07569681F2297
:101D3000C97A61F3C700E075696840460C311CF050
:101D4000C4FD63E740F00100E7E71D273726002CBC
:101D5000C4D0A1806868411D0079FFF7D8FC69688C
:101D600004F10F0201F10C00CB7A01461846FFF78F
:101D7000CEFC6868807CA0756868C178E07D61F3FE
:101D8000420020F0F900E0751F2140461CF03EFEA5
:101D90003CE720271026002CA0D0A180686804F121
:101DA0000902407A20726968CB1C88781946FFF7CF
:101DB000AEFC2BE721270A26002C8FD0BCF802109E
:101DC000A180696809792172696849796172817CA9
:101DD00021F0040157E022270B26002C84D0BCF808
:101DE0000400A0806868807820726868807901F0BB
:101DF000B8F860726868C07901F0B3F8A07205E7BE
:101E000024271026002CA3D0BCF80200A08068680C
:101E1000007920816868007A60816868C088A08144
:101E200068684089E081F1E623271026002C8FD0D6
:101E3000BCF80210A1806968898821816968C98815
:101E4000618169680989A18169684989E181817C29
:101E500021F0020117E0297A012903D0022914D0C8
:101E6000FFDFD3E61F271026002C95D06988A180BC
:101E7000A9892181E9896181298AA181698AE18110
:101E8000817C21F001018174C0E612276888102648
:101E9000214601F044F8B9E6287A072850D2DFE855
:101EA00000F0373D3D484848040011270926002C22
:101EB00094D0B5F802804046FFF7B6FA90F822A019
:101EC000A4F80480687A2072042140460DF072FE66
:101ED000052140460DF06EFE002140460DF06AFEE1
:101EE000012140460DF066FE032140460DF062FEE2
:101EF000022140460DF05EFE062140460DF05AFEDE
:101F0000072140460DF056FE504600F0B6FF7DE634
:101F10001B270926002C8AD0A180E6E61B2709266C
:101F2000002C84D0A180287A012800D002202072C1
:101F30006CE64A4621462846BDE8F04701F0F8BF66
:101F4000FFDF63E670B5254DE878132801D008203F
:101F500070BD0CF0B3FC06F063FB040002D12879DD
:101F600000F08BFF0021062011F09AFA204670BD88
:101F70001A4810B5C078122801D0082010BD0021E1
:101F800008460CF0FAFA06F04BFB0028F6D10021C7
:101F9000062011F085FA1120FFF7E8F9002010BDA6
:101FA00010B50E4C207801280ED000200CF0A1FDB9
:101FB00006F036FB002808D10021084611F070FA1F
:101FC0002078032802D004E0082010BDA07800F09B
:101FD00054FF012000F020FF002010BDC8010020A8
:101FE00070B5002538B1022817D0062836D007284A
:101FF00000D0FFDF70BDFFF7D3FF0028FAD106F055
:10200000D9FC0028F6D0017821F00F01891C21F0BD
:10201000F0012031017005723FE08EB23046FFF7CB
:1020200003FA040000D1FFDF20782128E2D006F077
:10203000C1FC60B1017821F00F01891C21F0F00191
:1020400010310170022101724680A57525E02146FC
:102050003046BDE870401322FFF782BBFE48C478CB
:10206000122C03D0132C04D0FFDF70BDFFF780FFCC
:1020700001E0FFF767FF0028F7D106F09BFC00287E
:10208000F3D0017821F00F01891C21F0F0012031FB
:102090000170122C05D002210172BDE8704006F0DB
:1020A0008CBC0121F8E72DE9F04116460C00804672
:1020B00000D1FFDF307820F00F00801C20F0F0000E
:1020C000103030702078012804D0022817D0FFDFAC
:1020D000BDE8F0814046FFF7A7F9050000D1FFDF1A
:1020E0000320A87506F069FC94E80F00083686E81E
:1020F0000F00D948817C41F001018174E8E7404636
:10210000FFF792F9050000D1FFDFA1884FF6FF70BD
:102110000027814202D1E288824203D0814201D16C
:10212000E08840B106F049FC94E80F00083686E8E4
:102130000F00AF75CCE7A87D0128C9D17823002214
:102140004146022011F002F90220A875C0E738B517
:1021500005460C46084611F0EFF920BB203D072D3F
:1021600051D2DFE805F0041C383D4349310000211D
:10217000072011F06BF908B1112038BDA01C0CF03C
:1021800010FC06F04DFA05003ED10022082311464E
:10219000072011F0DBF8072836D0FFDF34E0606855
:1021A00011F00EFA08B1102038BD618820886A4607
:1021B0000CF0CBFD06F034FA050025D1606818B3A9
:1021C000BDF8001001801FE0A07800F00101208818
:1021D0000CF0F1FD14E0206802F057F9054613E019
:1021E000207800F001000CF058FE09E0207800F0A3
:1021F00001000BF05FFF03E0618820880CF02DFDEB
:1022000006F00EFAEAE70725284638BD70B5054600
:102210000C46084611F0B6F908B1102070BD203DFB
:10222000072D1BD2DFE805F0041818181A1A180039
:102230002088FFF7F9F820B10078222804D208207E
:1022400070BD43F2020070BD2088A11C0CF003F8A1
:10225000BDE8704006F0E4B9062070BD072070BDEF
:102260007D48801D704738B516217B481CF0ACFBBB
:10227000012000F0D1FD1120FFF778F8764C684678
:10228000E11D06F02DFB9DF80010A07961F34700D9
:1022900020F00100A071002020744FF46170E081F3
:1022A00002206074FFF7B0F800B1FFDF00F0BEFE5F
:1022B00001F07FFC38BD10B50C46402120461CF0D3
:1022C00083FBA07F20F00300A07720202070002057
:1022D000A07584F8230080E670477CB5054611F0B0
:1022E0002BF908B110207CBD5B4CA11DD4F8060071
:1022F0000090D4F80A0001902846FFF7F1F9002871
:10230000F1D1FFF781F80028EDD00099C4F806104C
:10231000BDF8041061819DF8061021737CBD10B5D5
:10232000044611F02FF908B1102056E64A4922461A
:102330008879C91D4008FFF7EAF900204DE6FEB58F
:102340000D4604004FF0000711D00822FFF718F9DE
:10235000002811D1002608E054F826006946FFF74E
:1023600087F9002808D1761CF6B2AE42F4D30BF000
:102370000BFE10B143F20320FEBD374E7771FCB166
:1023800000271AE054F8270002A9FFF771F900B1FD
:10239000FFDF9DF808008DF8000054F8270050F882
:1023A000011FCDF801108088ADF8050068460BF0DC
:1023B00010FE00B1FFDF7F1CFFB2AF42E2D37571A8
:1023C0000020FEBD2DE9F0478AB01546894604007D
:1023D0001DD00F4608222946FFF7D2F8002810D159
:1023E000002612E054F826006946103000F074FD13
:1023F000002806D13FB157F8260011F09DF810B122
:1024000010200AB008E4761CF6B2AE42EAD30026E9
:10241000A5F101081CE000BF06F1010A0AF0FF0760
:1024200012E000BF54F82600017C4A0854F8271037
:102430000B7CB2EB530F05D10622113011311CF089
:1024400018FA70B17F1CFFB2AF42EBD30AF0FF065F
:102450004645E1DB4E4601E0C801002024B10120E1
:1024600003E043F20520CCE700200BF0D2FD10B9C9
:102470000BF0DBFD10B143F20420C2E764B3002788
:102480000DF1170826E000BF54F827006946103008
:1024900000F022FD00B1FFDF54F82700102250F8B1
:1024A000111FCDF801108088ADF8050054F82710F1
:1024B0000DF107001CF009FA96B156F8271010220A
:1024C00040461CF002FA68460BF068FD00B1FFDFE1
:1024D0007F1CFFB2AF42D7D3FFF75AF9002090E735
:1024E000404601F0C6FFEEE730B585B0044611F076
:1024F00023F818B9606811F06CF810B1102005B01D
:1025000030BD60884AF2B811884206D82078F74D6D
:1025100028B1012806D0022804D00720EFE7FEF7F3
:1025200073FF17E06078022804D0032802D043F23A
:102530000220E4E76874C1B200200090ADF8040006
:1025400002292BD0032926D0FFDF68460BF0DEFDE1
:1025500006F066F80028D2D1606801F07DFF20788F
:1025600058B101208DF800000DF1010001F081FF4C
:1025700068460CF07CFC00B1FFDF20782874FFF780
:1025800007F9608860B1E88180B20BF03AFD00B1D4
:10259000FFDF0020B3E78DF80500D6E74020FAE71B
:1025A0004FF46170EFE710B5044610F0EBFF20B96F
:1025B000606838B111F004F808B110200DE56068CA
:1025C00001F057FFC948C1896180417C6170007C7E
:1025D0002070002001E52DE9F04186B0054600207D
:1025E0008DF80C008DF804008DF808008DF81000AF
:1025F0001E4614468846284610F0EBFF18B92046C0
:1026000010F0E7FF10B1102006B061E555EA0400B4
:1026100018D01F2702AB03AA414628460097FEF7B1
:10262000CAFF0028F0D104AB01AA3146204600972A
:10263000FEF7C1FF0028E7D19DF80400C00703D0D2
:102640000A20E1E70720DFE73DB1294640460CF0CC
:102650003EFA05F0E5FF0028D6D13CB121463046D0
:102660000CF03EFA05F0DCFF0028CDD19F499DF823
:10267000080048700020C7E72DE9F04387B089467D
:102680004FF000089AA104468DF81080D1E90001AE
:10269000CDE90501204610F04FFF80B920780128D0
:1026A00003D1606810F048FF48B9904D287C50B1C4
:1026B000687C022807D1606810F08BFF18B11020E9
:1026C00007B0BDE8F0832878012801D00820F7E79B
:1026D00007200DF00DFA18B9207878B101280DD037
:1026E000FEF75EFE60B1608943F6E172A0F1200161
:1026F000914221780CD3012904D0B2E01220DFE707
:102700001320DDE700287CD1A189002979D109E0D7
:10271000012907D06978C90704D0A189002970D0A0
:10272000B4296ED8217831B1012908D0022904D00A
:10273000032966D10AE0002609E0022607E008B96D
:10274000A08908B1042609E0012607E00326287CB9
:1027500050B1687C022807D1606828B104A960687C
:10276000FEF786FF0028ABD1207A30B1012806D0D1
:10277000022806D0032874D105E0002704E00127D1
:1027800002E0022700E003270EB1022E0ED16FB146
:102790006879B0B36878800702D043F201208FE7F0
:1027A000022E03D1022F5CD0032F5AD0207808B11B
:1027B000012806D1484600F043FB002880D185F867
:1027C00002906089ADF800006089ADF802008DF8D4
:1027D00004600DF10500FEF76EFF00B1FFDF9DF80C
:1027E00010008DF806002078012806D0287C68B1FA
:1027F000687C02280AD1606840B1606850F8011F07
:1028000000E02EE0CDF80710808802E04046CDF8C9
:102810000780ADF80B008DF80E70A07BC0F340026E
:10282000014662F35F01C0F3800041EA800005A920
:10283000085C8DF80D00A0B168460CF017F905F0A2
:10284000EFFE0028ABD101200CF053F905F0E8FEB3
:102850000028A4D1052E0ED2DFE806F005050A0AED
:10286000050007202CE7A87800F0FAFA032000E022
:10287000022000F0D1FA012E0AD0A08940B1002236
:1028800083001146104610F061FD08B1032017E7E0
:10289000002015E72DE9FC4180460E460325084639
:1028A00010F097FE00286DD14046FEF7BDFD0400F4
:1028B00005D02078222805D20820BDE8FC8143F20B
:1028C0000200FAE7A07F00F003073EB1012F13D00A
:1028D00000203146FEF72FFE0500EED1012F0DD06E
:1028E000022F21D0FFDF2846E7E70000C8010020C3
:1028F00007060504030201000120EAE7A07D314636
:10290000022801D011B107E01120D6E7684600F097
:102910009AFC0028D1D16946404607F090FF050097
:10292000E1D10120A075DEE7A07D032803D1FE4898
:10293000807CC00701D02EB30EE026B1A07F4007F7
:102940001ED4002100E00121404607F098FF050059
:10295000C9D1A075002EC6D03146404600F0D4FA49
:1029600005461128BFD1A07F4107BCD4316844F887
:102970000E1F7168616040F0040020740025B2E70A
:102980001125B0E7102098E770B50C460546FEF714
:102990004BFD010005D022462846BDE87040FEF7F9
:1029A000DFBE43F2020070BD10B50BF05CFBBDE86A
:1029B000104005F035BE0123FEF739BD00231A464D
:1029C0001946FEF734BD7CB5044610F0B5FD08B1DC
:1029D00010207CBD628843F6FD73111F07209942C9
:1029E000F7D2A1880429F4D3B1F5804FF1D89142F0
:1029F000EFD8CD4DE878112801D008207CBDFEF736
:102A0000CFFCB0B32078810701D5697991B300F08C
:102A100001008DF800006088ADF80200A088ADF8D4
:102A2000040020780222C0F3400102EA5000014372
:102A30008DF807100DF10600FEF73DFE00B1FFDF37
:102A400068460BF05EFD05F0EBFD0028D6D10021B5
:102A500001200BF092FD05F0E3FD0028CED1E088C7
:102A600000F044FA0400C9D11220FEF77FFC204692
:102A70007CBD00E001E01320FAE70720F8E72DE92C
:102A8000F043DFF8A482074687B098F80300994620
:102A900015460C46122803D1FFF76AFA00281CD10C
:102AA000204610F049FDB8B9284610F045FD98B908
:102AB0006088ADF80000A088ADF8020020784FF0E3
:102AC0000006C0F340008DF80400207880071ED473
:102AD000384610F031FD08B11020F1E53878400893
:102AE00008D0012809D0022807D0032805D043F2D6
:102AF0000220E5E58DF8056002E001208DF8050073
:102B000057F8010FCDF80600B888ADF80A0003A801
:102B1000FEF7D1FD08B10320D2E52888ADF80E00FC
:102B20006888ADF81000A888ADF81200E888ADF804
:102B30001400ADF81660ADF8186068460BF0A8FDFB
:102B4000B8B998F803004546112801D00820B7E528
:102B500006200CF0CDFF50B12078800701D56879B0
:102B600038B1FEF71DFC022805D21320A8E512207B
:102B7000A6E50720A4E5484600F062F90028ACD19C
:102B800085F8049068460BF0C0FD05F049FD00286B
:102B9000A3D1287900F064F9E08800F0A7F90400D7
:102BA0009BD11320FEF7E2FB204689E570B5054670
:102BB0000C46084610F0E6FC08B1102070BD28460F
:102BC000FEF732FC38B10178222902D3807F8006DB
:102BD00004D4082070BD43F2020070BD214628468F
:102BE0000CF097F8BDE8704005F01ABD38B5054601
:102BF0000C46084610F0A0FC08B1102038BD28464D
:102C0000FEF712FC20B10078222804D2082038BD3B
:102C100043F2020038BD4448807C400701D51120B2
:102C200038BD2078800802D16078800801D0072064
:102C300038BDADF8005020788DF8020060788DF82E
:102C4000030068460BF04EFC05F0EAFC38BD2DE9A8
:102C5000F0418EB014460D460646FEF7E5FB070030
:102C600006D03878222806D208200EB0BDE8F081C0
:102C700043F20200F9E7284610F0ABFC30B94FF000
:102C800000084CB1204610F09BFC08B11020ECE786
:102C9000C4F80080A4F804802348807C800701D514
:102CA0001120E2E797F8220005F026FC8088011D3C
:102CB000FB2901D2001D00E0FB20C0B26A46294674
:102CC00000F0E5F8ADF81060BDF80200ADF81200B4
:102CD000BDF80600ADF81400BDF80000ADF8160010
:102CE000BDF80400ADF8180007A904A80BF03FFBDD
:102CF00000B1FFDFBDF81E00ADF80800BDF82000F0
:102D0000ADF80A00BDF82200BDF82410BDF800207F
:102D10000844ADF80C0007201B2AA6D3BDF802100A
:102D20001B29A2D3FB2A01E0C80100209DD8FB2962
:102D30009BD806278A4210D10121104600F056F890
:102D4000BDF80410884208D1BDF80200012100F04E
:102D50004DF8BDF80610884201D0384685E7BDF829
:102D6000080028B9BDF80A1011B9BDF80C1029B334
:102D70005DB1298849B1698839B124B102982060D0
:102D8000BDF80C00A08013206FE7BDF80010BDF85F
:102D90000A20081A80B2ADF80000BDF80210891AA6
:102DA000ADF80210012100F021F8ADF80400BDF8E3
:102DB0000200012100F01AF8ADF80600ADF8286015
:102DC000BDF80200ADF82A00BDF80600ADF82C00F1
:102DD000BDF80000ADF82E00BDF80400ADF83000DD
:102DE0000AA80BF076FA05F01BFC3EE7022903D097
:102DF000C000703080B2704780003C30FAE710802D
:102E00000888508048889080C88810818888D08041
:102E1000002050819081704730B5564D040008D095
:102E2000012C04D0022C06D0032C04D0FFDF2C7020
:102E300030BDFFDFFBE728780128F8D0FFDFF6E799
:102E400010B5044605F058FB30B1407830B120464B
:102E500005F057FE002010BD072010BD122010BD48
:102E600010B505F049FB040000D1FFDF607800B920
:102E7000FFDF6078401E607010BD10B505F03CFBB0
:102E8000040000D1FFDF6078401C607010BD10B5F9
:102E9000144631B10A68226049686160218839B1FD
:102EA00007E0208060800121FFF7A0FFA0800DE0F7
:102EB0002080618801B96080A08820B92088012124
:102EC000FFF794FFA080E088002804D160880121EA
:102ED000FFF78CFFE08010BD0278520804D0012A71
:102EE00002D043F202207047FEF7C2BB10B548B1D2
:102EF000830000221146062010F028FA062801D08F
:102F0000032010BD002010BD1FB56A46FFF777FFF4
:102F100068460BF0FCFC05F083FB04B010BD70B5F7
:102F20000C0006460DD0FEF77FFA050000D1FFDF4A
:102F3000A68028892081288960816889A081A88944
:102F4000E08170BD10B500231A4603E0845C234382
:102F5000521CD2B28A42F9D30BB1002010BD01201D
:102F600010BD00B5012803D0022801D0FFDF0020EA
:102F700000BD0000C80100200A4810B504680949D6
:102F80000948083108600FF0FCFB0648001D04608A
:102F900010BD0649002008604FF0E0210220C1F872
:102FA000800270471005024001000001FC1F004034
:102FB0000F4A12680D498A420CD118470C4A126810
:102FC0000A4B9A4206D101B510F02AF808F009FC24
:102FD000BDE80140074909680958084706480749FC
:102FE000054A064B7047000000000000BEBAFECA4A
:102FF000B000002004000020A8110020A81100202B
:103000002CFFFFFFDBE5B15100300200A500FFFF00
:1030100084000000284F4C00DA0D499A2F95338424
:1030200077AC2F1307CD6F7D177A70DEFE48002135
:1030300001604160018170472DE9F743044692B079
:103040009146406810F0BCFA40B1606810F0C1FAD7
:1030500020B9607800F00300022801D0012000E0D0
:103060000020F14E3072484610F066FA18B1102078
:1030700015B0BDE8F08349460120FEF75CFA002850
:10308000F6D101258DF842504FF4C050ADF8400004
:10309000002210A9284604F061F80028E8D18DF834
:1030A00042504FF428504FF00008ADF8400047461A
:1030B0001C216846CDF81C801BF0A8FC9DF81C0064
:1030C00008AA20F00F00401C20F0F00010308DF80E
:1030D0001C0020788DF81D0061789DF81E0061F3BA
:1030E000420040F001008DF81E009DF800000AA982
:1030F00040F002008DF800002089ADF83000ADF8F6
:103100003270608907AFADF834000B97606810AC7F
:103110000E900A94684603F016FE0028A8D1BDF868
:10312000200030808DF8425042F60120ADF840007A
:103130009DF81E0008AA20F00600801C20F0010067
:103140008DF81E000220ADF83000ADF8340013A851
:103150000E900AA9684603F0F6FD002888D1BDF854
:1031600020007080311D484600F033F9002887D1D7
:103170008DF8425042F6A620ADF840001C2168466A
:10318000CDF81C801BF042FC9DF81C00ADF83450BB
:1031900020F00F00401C20F0F00010308DF81C00D3
:1031A0009DF81D0008AA20F0FF008DF81D009DF875
:1031B0001E000AA920F0060040F00100801C8DF8D6
:1031C0001E009DF800008DF8445040F002008DF87C
:1031D0000000CDE90A4711A80E90ADF830506846BE
:1031E00003F0B1FD002899D1BDF82000F080002047
:1031F0003EE73EB504460820ADF80000204610F03A
:103200009BF908B110203EBD21460120FEF793F93D
:103210000028F8D12088ADF804006088ADF80600D9
:10322000A088ADF80800E088ADF80A007E4801AB40
:103230006A468088002104F08BF9BDF80010082947
:10324000E1D003203EBD1FB50446002002900820B7
:10325000ADF80800CDF80CD0204610F06DF910B193
:10326000102004B010BD704802AA81884FF6FF708C
:1032700004F0B0FB0028F4D1BDF80810082901D0F3
:103280000320EEE7BDF800102180BDF80210618038
:10329000BDF80410A180BDF80610E180E1E701B59A
:1032A00082B00220ADF800005F4802AB6A46408859
:1032B000002104F04DF9BDF80010022900D00320D0
:1032C0000EBD1CB5002100910221ADF80010019047
:1032D00010F058F908B110201CBD53486A464188C7
:1032E0004FF6FF7004F076FBBDF800100229F3D012
:1032F00003201CBDFEB54C4C06461546207A0F46F1
:10330000C00705D0084610F017F918B11020FEBD0F
:103310000F20FEBDF82D01D90C20FEBD304610F067
:103320000BF918BB208801A903F053FA0028F4D147
:1033300030788DF80500208801A904F0E8F800280D
:10334000EBD100909DF800009DF8051040F00200C0
:103350008DF80000090703D040F008008DF8000048
:103360002088694604F070F80028D6D1ADF80850DE
:1033700020883B4602AA002104F0EAF8BDF80810B4
:10338000A942CAD00320FEBD7CB5054600200090AE
:1033900001900888ADF800000C462846019510F011
:1033A0000FF918B9204610F0EDF808B110207CBDD7
:1033B00015B1BDF8000050B11B486A4601884FF6B0
:1033C000FF7004F007FBBDF8001021807CBD0C20CD
:1033D0007CBD30B593B0044600200D46009014210A
:1033E00001A81BF013FB1C2108A81BF00FFB9DF884
:1033F0000000CDF808D020F00F00401C20F0F000B5
:1034000010308DF800009DF8010020F0FF008DF8CD
:1034100001009DF8200040F002008DF820000120FE
:103420008DF8460002E00000DE01002042F6042094
:10343000ADF8440011A801902088ADF83C006088E8
:10344000ADF83E00A088ADF84000E088ADF842003D
:103450009DF8020006AA20F00600801C20F0010062
:103460008DF802000820ADF80C00ADF810000FA890
:10347000059001A908A803F066FC002803D1BDF857
:1034800018002880002013B030BD000010B504469D
:1034900010F052F808B1102010BD2078C0F30210CF
:1034A000042807D86078072804D3A178102901D808
:1034B000814201D2072010BDE078410706D421796E
:1034C0004A0703D4000701D4080701D5062010BD20
:1034D000002010BD10B513785C08C37F64F30003AF
:1034E000C3771478A40864F34103C3771078C30941
:1034F000487863F34100487013781C090B7864F333
:1035000047130B701378DB0863F3000048705078A2
:10351000487110BD10B5C4780B7864F300030B70CC
:10352000C478640864F341030B70C478A40864F39E
:1035300082030B70C478E40864F3C3030B7003794F
:10354000117863F30001117003795B0863F34101A3
:10355000117003799B0863F3820111700079C00830
:1035600060F3C301117010BD70B514460D460646D8
:1035700005F020FA80B10178182221F00F01891C92
:1035800021F0F001A03100F8081B21461BF0E2F900
:10359000BDE8704005F011BA29463046BDE87040DC
:1035A0001322FEF7DDB82DE9F047064608A8894644
:1035B00090E830041F469046142128461BF026FA56
:1035C0000021CAF80010B8F1000F03D0B9F1000FC4
:1035D00003D114E03878C00711D020680FF0D2FF73
:1035E000C0BBB8F1000F07D12068123028602068F6
:1035F000143068602068A8602168CAF80010387824
:10360000800724D560680FF0DBFF18BBB9F1000F0D
:1036100021D0FEF725FE0168C6F868118188A6F85A
:103620006C11807986F86E0101F0FBFCF94FEF60B8
:10363000626862B196F8680106F2691140081032BA
:10364000FEF765F81022394660681BF03EF900204D
:10365000BDE8F08706E0606820B1E8606068C6F801
:103660006401F4E71020F3E730B5054608780C460E
:1036700020F00F00401C20F0F001103121700020DC
:10368000607095F8230030B104280FD0052811D0C0
:10369000062814D0FFDF20780121B1EB101F04D2DF
:1036A00095F8200000F01F00607030BD21F0F000A0
:1036B000203002E021F0F00030302070EBE721F004
:1036C000F0004030F9E7F0B591B0022715460C46FE
:1036D00006463A46ADF80870092103AB05F089FFAC
:1036E0000490002810D004208DF804008DF801709B
:1036F000E034099605948DF818500AA968460DF033
:1037000039FF00B1FFDF012011B0F0BD10B588B066
:103710000C460A99ADF80000CBB11868CDF802004C
:10372000D3F80400CDF80600ADF80A20102203A853
:103730001BF0CBF868460BF061F904F071FF00282C
:1037400003D1A17F41F01001A17708B010BD002086
:10375000CDF80200E6E72DE9F84F0646808A0D46CF
:1037600080B28246FDF760FE04463078DFF8A4821E
:1037700000274FF00509A8F120080F2870D2DFE8D4
:1037800000F06FF23708387D8CC8F1F0EFF35FF38B
:10379000F300A07F00F00300022809D05FF00000D2
:1037A00080F0010150460CF0F3F9050003D101E06F
:1037B0000120F5E7FFDF98F85C10C90702D0D8F8C0
:1037C00060000BE0032105F11D000FF090FBD5F820
:1037D0001D009149B0FBF1F201FB1200C5F81D007C
:1037E00070686867B068A8672078252800D0FFDF78
:1037F000CAE0A07F00F00300022809D05FF00000BB
:1038000080F0010150460CF0C3F9060003D101E03D
:103810000120F5E7FFDF3078810702D521782529DF
:1038200004D040F001003070BDE8F88F022028700D
:10383000307F287106F11D002D36C5E90206F3E739
:10384000A07F00F00300022808D0002080F00101D2
:1038500050460CF09DF9040004D102E00120F5E788
:10386000A5E1FFDF2078C10604D5072028703D348C
:103870006C60D9E740F008002070D5E7E07FC00613
:1038800000D5FFDF307CB28800F0010301B0504664
:10389000BDE8F04F092106F035BD04B9FFDF7168BE
:1038A00021B1102204F124001BF00FF8282120463A
:1038B000FDF7ECFDA07F00F0030002280ED104F11B
:1038C0002400002300901A4621465046FFF71EFFB1
:1038D000112807D029212046FDF7D8FD307A84F839
:1038E0002000A1E7A07F000700D5FFDF14F81E0F1E
:1038F00040F008002070E782A761E7616178084620
:1039000061F38200410861F3C3006070307AE070B7
:103910008AE7A07F00F00300022809D05FF00000D2
:1039200080F0010150460CF033F9040003D101E0AE
:103930000120F5E7FFDF022104F185000FF0D7FA3F
:103940000420287004F5B4706860B4F885002882FB
:10395000304810387C346C61C5E9028064E703E0CC
:1039600022E15BE02DE015E0A07F00F003000228DB
:1039700007D0002080F0010150460CF009F918B979
:1039800001E00120F6E7FFDF324621465046BDE860
:10399000F84FE9E504B9FFDF20782128A1D9307973
:1039A000012803D1E07F40F01000E0773246214645
:1039B0005046FFF7D9FD2046BDE8F84F2321FDF71B
:1039C00065BD3279AA8005F108030921504605F04A
:1039D00010FEE86010B185F8009025E7A07F00F0A8
:1039E0000300022808D0002080F0010150460CF0AE
:1039F000CFF8040003D101E00120F5E7FFDF04F177
:103A0000620102231022081F0BF049FF0770317971
:103A1000417009E70802002040420F00A07F00F03B
:103A20000300022808D0002080F0010150460CF06D
:103A3000AFF8050003D101E00120F5E7FFDF95F8BD
:103A4000840000F00300012878D1A07F00F0030774
:103A5000E07FC0F3400616B1022F04D132E095F8A2
:103A6000A000C0072AD0D5F8601119B395F88320BB
:103A7000087C62F387000874E27FD5F8601162F376
:103A800041000874D5F8601166F300000874AEB107
:103A9000D5F86001102204F1240188351AF015FFD1
:103AA000287E40F001002876287820F0010005F8F3
:103AB000880900E016B1022F04D02CE095F88800A8
:103AC000C00726D0D5F85C1119B395F88320087C7F
:103AD00062F387000874E27FD5F85C1162F341005D
:103AE0000874D5F85C1166F3000008748EB1D5F83F
:103AF0005C01102204F1240188351AF0E6FE2878D2
:103B000040F0010005F8180B287820F0010005F8B6
:103B1000A009022F44D0002000EB400005EBC000BC
:103B200090F88800800709D595F87C00D5F86421C5
:103B3000400805F17D011032FDF7E9FD8DF8009098
:103B400095F884006A4600F003008DF8010095F8AE
:103B500088108DF8021095F8A0008DF8030021461A
:103B6000504601F047FA2078252805D0212807D0B3
:103B7000FFDF2078222803D922212046FDF786FC8A
:103B8000A07F00F0030002280CD0002080F001018B
:103B900050460CF00FF800283FF451AEFFDF43E62B
:103BA0000120B9E70120F1E7706847703CE6FFDFCC
:103BB0003AE670B5FE4C002584F85C5025660DF0A1
:103BC000A6FC04F11001204604F0B0FE84F8305049
:103BD00070BD70B50D46FDF727FC040000D1FFDF76
:103BE0004FF4B87128461AF011FF04F1240028613F
:103BF000A07F00F00300022808D0012105F1E000B9
:103C00000DF086FC002800D0FFDF70BD0221F5E733
:103C10000A46014602F1E0000DF09ABC70B5054677
:103C2000406886B00178092906D00C2933D00D29C7
:103C30002FD0FFDF06B070BD46883046FDF7F4FB9D
:103C4000040000D1FFDF20782128F3D028281BD1E1
:103C5000686802210C3001F0C2F9A8B16868082137
:103C6000001D01F0BCF978B104F1240130460AF0DE
:103C7000B9FF04F0D5FC00B1FFDF06B02046BDE877
:103C800070402921FDF702BC06B0BDE8704004F089
:103C900094BE01218171686886883046FDF7C4FBB7
:103CA000040000D1FFDFA07F00F00301022902D150
:103CB00020F01000A077207821280AD06868817948
:103CC00009B1807880B1A07F00F00300022862D0A3
:103CD000FFDFA07F00F003000228ABD1FDF770FDED
:103CE0000028A7D0FFDFA5E704F067FEE07FC1074B
:103CF00029D0800705D594F8200000F01F00102877
:103D00001FD0052084F82300207829281DD02428DE
:103D1000DFD1314605200FF0C3FB22212046FDF7FD
:103D2000B5FBA07F00F00300022832D05FF0000056
:103D300080F0010130460BF03DFF0028C9D0FFDFC5
:103D4000C7E70620DEE70420DCE7A07F00F00300E1
:103D5000022809D05FF0000080F0010130460BF02E
:103D600017FF050003D101E00120F5E7FFDF252162
:103D70002046FDF78BFB03208DF80000694605F116
:103D8000E0000DF0DCFB0228A3D00028A1D0FFDF6B
:103D90009FE70120CCE704F010FE9AE72DE9F043FD
:103DA00087B09946164688460746FDF73DFB040056
:103DB0004BD02078222848D3232846D0E07FC00665
:103DC00043D4A07F00F00300022809D05FF0000078
:103DD00080F0010138460BF0DBFE050002D00CE05C
:103DE0000120F5E7A07F00F00300022805D00121A3
:103DF000002238460BF0C3FE05466946284601F00E
:103E000020F9009800B9FFDF45B10098E035056161
:103E10002078222806D0242804D007E0009900202A
:103E2000086103E025212046FDF730FB00980121C1
:103E300041704762868001A9C0E902890DF09AFBB2
:103E4000022802D0002800D0FFDF07B0BDE8F083D1
:103E500070B586B00546FDF7E7FA017822291ED92C
:103E6000807F00F00300022808D0002080F00101CC
:103E700028460BF08DFE04002FD101E00120F5E76C
:103E8000FFDF2AE0B4F85E0004F1620630440178F6
:103E9000427829B121462846FFF715FCB0B9C9E69A
:103EA000ADF804200921284602AB05F0A2FB0390DF
:103EB0000028F4D005208DF80000694604F1E000E8
:103EC0000DF03DFB022801D000B1FFDF02231022DC
:103ED000314604F15E000BF018FDB4F860000028D4
:103EE000D0D1A7E610B586B00446FDF79DFA01785B
:103EF00022291BD9807F00F00300022808D000206F
:103F000080F0010120460BF043FE040003D101E0E4
:103F10000120F5E7FFDF06208DF80000694604F177
:103F2000E0000DF00CFB002800D0FFDF06B010BD54
:103F30002DE9F05F05460C46002700789046010900
:103F40003E4604F1080BBA4602297DD0072902D06B
:103F50000A2909D146E068680178092905D00C29A9
:103F600030D00D292ED0FFDFBCE114271C26002CF9
:103F70006BD04088A080FDF757FA5FEA000900D1B6
:103F8000FFDF99F817005A46400809F11801FDF7BC
:103F9000BEFB68688089208269684868C4F812009E
:103FA0008868C4F81600A07E20F0060002E0000039
:103FB000E801002040F00100A07699F81E0040F0D2
:103FC00040014DE01A270A26002CD1D08088A0801D
:103FD000FDF72AFA050000D1FFDF59462846FFF712
:103FE00043FB7FE10CB1A88BA080287A0B287DD001
:103FF00006DC01287BD0022808D0032804D135E054
:104000000D2875D00E2874D0FFDF6BE11E2709261E
:10401000002CADD0A088FDF707FA5FEA000900D1B7
:10402000FFDF287B00F003000128207A1BD020F05E
:1040300001002072297B890861F341002072297BED
:10404000C90861F3820001E041E1F2E02072297BBE
:10405000090961F3C300207299F81E0040F0800145
:1040600089F81E103EE140F00100E2E713270D261B
:10407000002CAAD0A088FDF7D7F98146807F00F0F8
:104080000300022808D0002080F00101A0880BF076
:104090007FFD050003D101E00120F5E7FFDF99F87E
:1040A0001E0000F00302022A50D0686F817801F0F0
:1040B00003010129217A4BD021F00101217283787B
:1040C0009B0863F3410121728378DB0863F382016B
:1040D000217283781B0963F3C3012172037863F3B0
:1040E00006112172437863F3C71103E061E0A9E090
:1040F00090E0A1E0217284F809A0C178A172022A9F
:1041000029D00279E17A62F30001E1720279520862
:1041100062F34101E1720279920862F38201E17275
:104120000279D20862F3C301E1724279217B62F322
:10413000000121734279520862F3410121734279EF
:10414000920862F382012173407928E0A86FADE7FD
:1041500041F00101B2E74279E17A62F30001E172D4
:104160004279520862F34101E1724279920862F3A6
:104170008201E1724279D20862F3C301E1720279ED
:10418000217B62F3000121730279520862F341013D
:1041900021730279920862F3820121730079C008C9
:1041A00060F3C301217399F80000232831D9262137
:1041B00040E018271026E4B3A088FDF735F98346C0
:1041C000807F00F00300022809D0002080F0010168
:1041D000A0880BF0DDFC5FEA000903D101E00120BB
:1041E000F4E7FFDFE868A06099F8000040F0040100
:1041F00089F8001099F80100800708D50120207384
:104200009BF8000023286DD92721584651E084F8F7
:104210000CA067E015270F265CB1A088FDF704F914
:10422000814606225946E86809F0A8FC0120A073DF
:10423000A2E041E048463CE016270926E4B3287B8B
:1042400020724FE0287B19270E26ACB3C4F808A0D3
:10425000A4F80CA0012807D0022805D0032805D017
:10426000042803D0FFDF0DE0207207E0697B0428FB
:1042700001F00F0141F0800121721ED0607A20F020
:1042800003006072A088FDF7CFF80546007821286A
:1042900028D0232800D0FFDFA87F00F003000228E9
:1042A00013D0002080F00101A0880BF083FC2221B4
:1042B0002846FDF7EBF815E004E0607A20F00300F3
:1042C000401CDEE7A8F8006011E00120EAE70CB12D
:1042D0006888A080287A03282ED004280AD00528D0
:1042E00050D0FFDFA8F800600CB127806680002066
:1042F000BDE8F09F15270F26002CE3D0A088FDF71E
:1043000093F8807F00F00300022809D05FF00000DE
:1043100080F00101A0880BF03BFC050003D101E017
:104320000120F5E7FFDFD5F81D000622594609F008
:1043300025FC84F80EA0D5E717270926002CC1D04C
:10434000A088FDF771F88146807F00F00300022805
:1043500008D0002080F00101A0880BF019FC0500B6
:1043600003D101E00120F5E7FFDF6878800701D580
:10437000022000E00120207299F800002328B1D922
:10438000272157E719270E26002C9BD0A088FDF780
:104390004BF85FEA000900D1FFDFC4F808A0A4F8D9
:1043A0000CA084F808A0A07A40F00300A07299F84D
:1043B0001F1061F38200A07299F81F10C1F3400230
:1043C000114205D099F8201001F01F0110292CD0BE
:1043D00020F00800A07299F81F004108607A61F38C
:1043E000C3006072697A01F003010129A3D140F092
:1043F0000400607299F81E0000F003000228E87AB9
:1044000016D0217B60F300012173AA7A607B62F3EE
:1044100000006073EA7A520862F341012173A97ABD
:10442000490861F3410060735CE740F00800D1E7A0
:10443000617B60F300016173AA7A207B62F3000064
:104440002073EA7A520862F341016173A97A49083C
:1044500061F34100207345E710B5FE4C30B10146D1
:10446000102204F120001AF030FA012084F8300004
:1044700010BD10B5044600F0D4FDF64920461022C8
:10448000BDE8104020311AF020BA70B5F14D060099
:104490004FF0000412D00FF04FF808B110240BE0D9
:1044A0000621304609F051FB411C04D0286601204A
:1044B00085F85C0000E00724204670BD0020F7E787
:1044C000007810F00F0204D0012A05D0022A0CD186
:1044D00010E0000909D10AE00009012807D00228EC
:1044E00005D0032803D0042801D0072070470870A6
:1044F000002070470620704705282AD2DFE800F028
:1045000003070F171F00087820F0FF001EE008784F
:1045100020F00F00401C20F0F000103016E008786A
:1045200020F00F00401C20F0F00020300EE0087852
:1045300020F00F00401C20F0F000303006E008783A
:1045400020F00F00401C20F0F000403008700020E8
:104550007047072070472DE9F041804688B00D462E
:10456000002708460FF035F8A8B94046FCF75CFF75
:10457000040003D02078222815D104E043F2020081
:1045800008B0BDE8F08145B9A07F010603D500F071
:104590000300022801D01020F2E7A07FC10601D459
:1045A000010702D50DB10820EAE7E17FC90601D570
:1045B0000D20E5E700F00300022805D125B12846CB
:1045C000FEF764FF0700DBD1A07F00F003000228A4
:1045D00008D0002080F0010140460BF0D9FA060017
:1045E00002D00FE00120F5E7A07F00F003000228D1
:1045F0000ED0002080F00101002240460BF0BFFAEF
:10460000060007D0A07F00F00300022804D009E0D4
:104610000120EFE70420B3E725B12A4631462046C2
:10462000FEF758FF6946304600F00BFD009800B9D0
:10463000FFDF0099022006F1E0024870C1F82480F3
:104640004A6100220A81A27F02F00302022A1CD0E2
:1046500001200871287800F00102087E62F3010051
:1046600008762A78520862F3820008762A7892083F
:1046700062F3C30008762A78D20862F30410087641
:1046800024212046FCF702FF33E035B30871301DCA
:1046900088613078400908777078C0F34000487727
:1046A000287800F00102887F62F301008877E27FBA
:1046B00062F382008877E27F520862F3C300887752
:1046C000727862F304108877A878C87701F1210224
:1046D00028462031FEF71EFF03E003200871052065
:1046E000087625212046FCF7D1FEA07F20F080002F
:1046F000A07701A900980CF03DFF022801D000B17D
:10470000FFDF38463CE72DE9FF4F534A0D4699B08D
:104710009A4607CA0BAB002783E807001998FCF7F5
:1047200083FE060006D03078262806D008201DB06B
:10473000BDE8F08F43F20200F9E7B07F00F0030913
:10474000B9F1020F03D00020284302D006E0012077
:10475000FAE71B98FEF79AFE0028E8D1B07F00F038
:104760000300022801D11B9979BB022808D0002040
:1047700080F0010119980BF00BFA040003D101E05D
:104780000120F5E7FFDF852D28D007DCF5B1812D6D
:104790001ED0822D1ED0832D08D11DE0862D1FD066
:1047A000882D1FD0892D1FD08A2D1FD00F2020715A
:1047B0000F281DD004F0FEF8E0B101208DF8400074
:1047C000201D11902079B8B165E111E00020EEE7DD
:1047D0000120ECE70220EAE70320E8E70520E6E70E
:1047E0000620E4E70820E2E70920E0E70A20DEE708
:1047F00007209CE711209AE7B9F1020F03D0A56FBB
:1048000003D1A06F02E0656FFAE7606F804632D097
:104810004FF0010000904FF0020001902146304619
:104820001B9AFEF757FE1B98007800F00101A8784C
:1048300061F30100A870F17F61F38200A870F17F3D
:10484000490861F3C300A870617861F30410A8708F
:10485000207803E0E801002068ED0100400928709D
:104860006078C0F3400068701B988078E870002082
:104870006871287103E00220009001200190A8785F
:1048800098F80210C0F3C000C1F3C00108405FEA0D
:10489000000B2CD050460EF04FFE90BBDAF80C0007
:1048A0000EF04AFE68BBDAF81C000EF045FE40BB75
:1048B000DAF80C00A060DAF81C00E06098F801005B
:1048C000617800F0010041EA4000607098F8021041
:1048D000C0B2C1F30011891E08406070002020772B
:1048E000019906F1170002290CD001210BE098F87C
:1048F0000110607801F00101FD2242EA4101084007
:10490000E3E732E0002104EB810148610099701C6B
:10491000022901D0012100E0002104EB810148615E
:10492000A87800F00300012858D198F8020000F0A0
:104930000300012852D1B9F1020F04D02A1D691DCC
:104940001B98FEF7E7FD297998F8040001408DF8DF
:104950003810687998F8052010408DF83C00014324
:104960003CD050460EF0E8FD08B11020DFE60AF119
:1049700010010491B9F1020F18D008465FF0000150
:1049800004F18C03CDE9000304F5AE7202920EAB84
:104990005A462046FEF707FE0028E7D1B9F1020F7C
:1049A00008D0504608D14FF0010107E050464FF0C3
:1049B0000101E5E70498F5E74FF0000104F1A403D5
:1049C000CDE9000304F5B072029281F001010FAB52
:1049D0005A462046FEF7E7FD0028C7D160788007D9
:1049E00034D4A87898F80210C0F38000C1F3800195
:1049F00008432BD0297898F800000BAAB9F1020FD0
:104A000006D032F811204300DA4002F003070AE032
:104A100032F810204B00DA4012F0030705D0012FC6
:104A20000BD0022F0BD0032F07D0BBF1000F0DD0FE
:104A3000012906D0042904D008E00227F5E7012760
:104A4000F3E7012801D0042800D10427F07F40F0CB
:104A500001006BF34100F077607881074FF00300AD
:104A60000CD5A071BBF1000F15D100BF8DF85C0013
:104A700017AA3146199800F0BDFA0CE00221022F66
:104A800018D0012F18D0042F22D00020A071F07F61
:104A900020F00100F07725213046FCF7F7FC10A943
:104AA00004F1E0000CF04BFD10B1022800D0FFDF54
:104AB00000203CE6A171D9E7A1710D2104F120008D
:104AC00019F0A4FF207840F0020020700420CDE708
:104AD0000120A071DFE72DE9F04387B090468946B9
:104AE00004460025FCF7A0FC060006D030782728F5
:104AF00006D0082007B0BDE8F08343F20200F9E7D2
:104B0000B07F00F00300022808D0002080F00101EF
:104B100020460BF03DF8040003D101E00120F5E749
:104B2000FFDFA7795FEA090005D0012821D0B9F19C
:104B3000020F26D110E0B8F1000F22D1012F05D0CD
:104B4000022F05D0032F05D0FFDF2DE00C252BE031
:104B5000012529E0022527E040460EF0EDFCB0B922
:104B6000032F0ED11022414604F11D0019F0ADFEB5
:104B70001AE0012F02D0022F03D104E0B8F1000F98
:104B800012D00720B6E740460EF0D6FC08B1102040
:104B9000B0E7102104F11D0019F016FF0621404670
:104BA00008F0D3FFC4F81D002078252140F0020052
:104BB00020703046FCF76AFC2078C10713D020F043
:104BC0000100207002208DF8000004F11D00029009
:104BD0008DF804506946C3300CF0B1FC022803D0B4
:104BE00010B1FFDF00E02577002083E730B587B004
:104BF0000D460446FCF718FCA0B1807F00F00300CE
:104C0000022812D05FF0000080F0010120460AF077
:104C1000BFFF04000ED028460EF08EFC38B11020E5
:104C200007B030BD43F20200FAE70120ECE720783C
:104C3000400701D40820F3E7294604F13D00202273
:104C4000054619F042FE207840F010002070010760
:104C50000FD520F00800207007208DF8000069466D
:104C600004F1E00001950CF06AFC022801D000B1CB
:104C7000FFDF0020D4E770B50D460646FCF7D4FBF5
:104C800018B10178272921D102E043F2020070BD5A
:104C9000807F00F00300022808D0002080F001018E
:104CA00030460AF075FF040003D101E00120F5E76A
:104CB000FFDFA079022809D16078C00706D02A4614
:104CC00021463046FEF7FFFC10B10FE0082070BD12
:104CD000B4F860000E280BD204F162010223102206
:104CE000081F0AF0DCFD012101704570002070BD35
:104CF000112070BD70B5064614460D4608460EF0EC
:104D00001BFC18B920460EF03DFC08B1102070BD08
:104D1000A6F57F40FF380ED03046FCF785FB38B152
:104D2000417822464B08811C1846FCF7F0FC07E04E
:104D300043F2020070BD2046FDF7F1FA0028F9D1D8
:104D40001021E01D0EF0D3F8E21D294604F11700F2
:104D500000F087F9002070BD2DE9F04104468AB0CB
:104D600015468846002708460EF033FC18B9284639
:104D70000EF02FFC18B110200AB0BDE8F0812046DB
:104D8000FCF752FB060003D0307827281BD102E045
:104D900043F20200F0E7B07F00F00300022809D0E0
:104DA0005FF0000080F0010120460AF0F1FE0400EF
:104DB00003D101E00120F5E7FFDF2078400702D5AD
:104DC0006078800701D40820D6E7B07F00F00300A8
:104DD000022803D0A06F03D1A16F02E0606FFAE751
:104DE000616F407800B19DB1487810B1B8F1000F03
:104DF0000ED0ADB1EA1D06A8E16800F032F910222C
:104E000006A905F1170019F034FD18B1042707E0D1
:104E10000720B1E71022E91D04F12D0019F055FD1E
:104E2000B8F1000F06D0102208F1070104F11D00AF
:104E300019F04BFD2078252140F00200207030460B
:104E4000FCF724FB2078C10715D020F0010020706A
:104E500002208DF8000004F11D0002901030039034
:104E60008DF804706946B3300CF069FB022803D05A
:104E700010B1FFDF00E0277700207DE7F8B5154689
:104E80000E460746FCF7D0FA040004D0207822280A
:104E900004D00820F8BD43F20200F8BDA07F00F066
:104EA0000300022802D043F20400F8BD30460EF0A1
:104EB00043FB18B928460EF03FFB08B11020F8BD9F
:104EC00000953288B31C21463846FEF71FFC112896
:104ED00014D00028F3D1297C4A08E17F62F3000155
:104EE000E1772A7C62F34101E177297C890884F823
:104EF0002010A17F21F08001A177F8BDA17F0907D3
:104F0000FBD4D6F80200C4F83600D6F80600C4F880
:104F10003A003088A0861022294604F1240019F0B6
:104F2000D4FC287C4108E07F61F38200E077297C93
:104F300061F3C300E077287C800884F82100A07F1B
:104F400040F00800A0770020D3E770B50D46064674
:104F50000BB1072070BDFCF767FA040007D020787A
:104F6000222802D3A07F400604D4082070BD43F25B
:104F7000020070BDA5B12946304609F033FE03F0AA
:104F80004FFB297C4A08E17F62F30001E1772A7C2C
:104F900062F34101E177297C890884F8201004E05C
:104FA000304609F042FE03F03BFBA17F21F04001B7
:104FB000A17770BD70B50D46FCF736FA040005D038
:104FC00028460EF0DFFA20B1102070BD43F2020037
:104FD00070BD29462046FEF747FB002070BD04E067
:104FE00010F8012B0AB100207047491E89B2F7D290
:104FF0000120704770B51546064603F0DBFC04003F
:1050000000D1FFDF207820F00F00801C20F0F0009E
:105010002030207066802868A060BDE8704003F0F2
:10502000CCBC10B5134C94F83000002808D104F122
:105030002001A1F110000CF0C4FA012084F8300026
:1050400010BD10B190F8B9202AB10A4890F8350087
:1050500018B1002003E0B83001E0064834300860A1
:10506000704708B50023009313460A460AF08BFFE9
:1050700008BD0000E8010020F0B5007B059F1E463A
:1050800014460D46012800D0FFDF0C2030803A2066
:105090003880002C08D0287A032806D0287B0128E5
:1050A00000D0FFDF17206081F0BDA889FBE72DE964
:1050B000F04786B0144691F80C900E9A0D46B9F15F
:1050C000010F0BD01021007B2E8A8846052807D0BF
:1050D000062833D0FFDF06B0BDE8F0870221F2E7F3
:1050E000E8890C2100EB400001EB400018803320E0
:1050F0001080002CEFD0E889608100271AE000962C
:10510000688808F1020301AA696900F085FF06EBCF
:105110000800801C07EB470186B204EB4102BDF892
:10512000040090810DF1060140460E320CF0B2FAF7
:105130007F1CBFB26089B842E1D8CCE73420108030
:10514000E889B9F1010F11D0122148430E301880BF
:10515000002CC0D0E88960814846B9F1010F00D029
:105160000220207300270DF1040A1FE00621ECE75E
:105170000096688808F1020301AA696900F04CFFF3
:1051800006EB0800801C86B2B9F1010F12D007EBC4
:10519000C70004EB4000BDF80410C18110220AF1E1
:1051A0000201103019F091FB7F1CBFB26089B84238
:1051B000DED890E707EB470104EB4102BDF804009D
:1051C000D0810AF10201404610320CF063FAEBE79D
:1051D0002DE9F0470E4688B090F80CC096F80C8088
:1051E000378AF5890C20109902F10C044FF0000A5F
:1051F000BCF1030F08D0BCF1040F3ED0BCF1070F87
:105200007DD0FFDF08B067E705EB850C00EB4C00B5
:10521000188031200880002AF4D0A8F1060000F0A0
:10522000FF09558125E0182101A819F0EFFB00972F
:105230007088434601AA716900F0EEFEBDF80400D3
:105240002080BDF80600E080BDF808002081A21C87
:105250000DF10A0148460CF01DFAB9F1000F00D01B
:1052600018B184F804A0A4F802A007EB080087B2E4
:105270000A346D1EADB2D6D2C4E705EB850C00EB47
:105280004C00188032200880002ABBD0A8F105000D
:1052900000F0FF09558137E000977088434601AA66
:1052A000716900F0B9FE9DF80600BDF80410E180B8
:1052B0002179420860F3000162F34101820862F340
:1052C0008201C20862F3C301020962F304114209B8
:1052D00062F34511820962F386112171C009607180
:1052E000BDF80700208122460DF1090148460CF067
:1052F000D1F918B184F802A0A4F800A000E007E0FA
:1053000007EB080087B20A346D1EADB2C4D279E74C
:10531000A8F1020084B205FB08F000F10E0CA3F81E
:1053200000C035230B80002AA6D0558194810097B8
:1053300083B270880E32716900F06EFE62E72DE96B
:10534000F84F1E460A9D0C4681462AB1607A00F548
:105350008070D080E089108199F80C000C274FF004
:1053600000084FF00E0A0D2873D2DFE800F09E0708
:105370000E1C28303846556A737373002146484620
:105380000095FFF779FEBDE8F88F207B914608284D
:1053900002D0032800D0FFDF378030200AE000BFB2
:1053A000A9F80A80EFE7207B9146042800D0FFDFB0
:1053B000378031202880B9F1000FF1D1E3E7207B5D
:1053C0009146042800D0FFDF37803220F2E7207BAF
:1053D0009146022800D0FFDF37803320EAE7207BA8
:1053E0001746022800D0FFDF3420A6F800A028804E
:1053F000002FC8D0A7F80A80C5E7207B17460428ED
:1054000000D0FFDF3520A6F800A02880002FBAD0FA
:105410004046A7F80A8012E0207B1746052802D0F4
:10542000062800D0FFDF1020308036202880002F93
:10543000A9D0E0897881A7F80E80B9F80E00B8816C
:10544000A1E7207B9146072800D0FFDF3780372077
:10545000B0E72AE04FF0120018804FF03800170034
:10546000288090D0E0897881A7F80E80A7F8108076
:1054700099F80C000A2805D00B2809D00C280DD06B
:10548000FFDF80E7207B0A2800D0FFDF01200AE051
:10549000207B0B2800D0FFDF042004E0207B0C28B9
:1054A00000D0FFDF052038736DE7FFDF6BE770B5D5
:1054B0000C460546FBF7B8FF20B10078222804D23D
:1054C000082070BD43F2020070BD052128460AF095
:1054D0005FFB206008B1002070BD032070BD30B4B8
:1054E0004880087820F00F00C01C20F0F0009030B9
:1054F00001F8080B1DCA81E81D0030BC03F05DBA3D
:105500002DE9FF4784B0002782460297079890460E
:105510008946123006F086FA401D20F003060798EF
:1055200028B907A95046FFF7C2FF002853D1B9F1A7
:10553000000F05D00798017B19BB052504681BE007
:1055400098F80000092803D00D2812D0FFDF45E0AD
:10555000079903254868B0B3497B4288714391425B
:1055600038D98AB2B3B2011D0AF085F90446078022
:1055700002E0079C042508340CB1208810B1032DEB
:1055800028D02BE007980121123006F07DFAADF803
:105590000C00024602AB2946504604F02AF80700E8
:1055A00001D1A01C029007983A461230C8F80400B6
:1055B000A8F802A003A94046029B06F072FAC0B107
:1055C000072814D200E005E0DFE800F0060811111A
:1055D0000F0A0C00132015E6002013E6112011E637
:1055E00008200FE643F203000CE607200AE603203A
:1055F00008E6BDF80C002346CDE900702A46504667
:10560000079900F019FD57B9032D08D10798B3B2D7
:10561000417B406871438AB2011D0AF040F9B9F13B
:10562000000FD9D0079981F80C90D5E72DE9FE4FEE
:1056300091461A881C468A468046FAB102AB494612
:1056400003F0D7FF050019D04046A61C27880AF0B2
:10565000E3FB3246072629463B46009609F0F1FF58
:1056600020882346CDE900504A465146404600F086
:10567000E3FC002020800120BDE8FE8F0020FBE736
:1056800010B586B01C46AAB104238DF800301388EB
:10569000ADF808305288ADF80A208A788DF80E20CF
:1056A0000988ADF80C1000236A462146FFF728FF51
:1056B00006B010BD1020FBE770B50D4605210AF0BD
:1056C00067FA040000D1FFDF294604F11200BDE8AB
:1056D000704006F0C2B92DE9F8430D468046002619
:1056E00003F068F904462878102878D2DFE800F043
:1056F000773B34533131123131310831313131316D
:105700002879001FC0B2022801D0102810D114BB84
:10571000FFDF35E004B9FFDF052140460AF038FA23
:10572000007B032806D004280BD0072828D0FFDFF1
:10573000072655E02879801FC0B2022820D050B13A
:10574000F6E72879401FC0B2022819D0102817D0D8
:10575000EEE704B9FFDF13E004B9FFDF2879012881
:105760000ED1172137E0052140460AF011FA070053
:1057700000D1FFDF07F11201404606F04BF92CB1D2
:105780002A4621464046FFF7AAFE29E0132140465B
:10579000FDF7FAF824E004B9FFDF052140460AF0DE
:1057A000F7F9060000D1FFDF694606F1120006F0A6
:1057B0003BF9060000D0FFDFA988172901D2172284
:1057C00000E00A46BDF80000824202D9014602E02C
:1057D00005E01729C5D3404600F03EFCD0E7FFDFC7
:1057E0003046BDE8F883401D20F0030219B102FBEA
:1057F00001F0001D00E000201044704713B5009830
:1058000050B100244FEA0D0009F0DFFF002C02D157
:10581000F74A009911601CBD01240020F4E72DE92E
:10582000F0470C4615462421204619F0EFF805B93B
:10583000FFDFA87860732888DFF8B4A3401D20F04C
:105840000301AF788946DAF8000009F0DCFF0600B2
:1058500000D1FFDF4FF000082660A6F8008077B186
:1058600009FB07F1091D0AD0DAF8000009F0CBFFA7
:10587000060000D1FFDF6660C6F8008001E0C4F8D2
:105880000480298804F11200BDE8F04706F0B4B89E
:105890002DE9F047804601F112000D46814606F0E1
:1058A000C1F8401DD24F20F003026E7B14462968D8
:1058B000386809F0D3FF3EB104FB06F2121D03D095
:1058C0006968386809F0CAFF05200AF009F904463A
:1058D00005200AF00DF9201A012802D1386809F0D4
:1058E00087FF49464046BDE8F04706F09AB870B5D4
:1058F000054605210AF04CF9040000D1FFDF04F150
:1059000012012846BDE8704006F084B82DE9F04F3A
:1059100091B04FF0000BADF834B0ADF804B047884B
:105920000C4605469246052138460AF031F9060034
:1059300000D1FFDF24B1A780A4F806B0A4F808B016
:10594000297809220B20B2EB111F7DD12A7A04F1AC
:10595000100138274FF00C084FF001090391102A6D
:1059600073D2DFE802F072F2F1F07F08D2888D9FE7
:105970003DDBF3EEB6B6307B022800D0FFDFA8890E
:1059800008EBC001ADF804103021ADF83410002C44
:1059900025D06081B5F80E9000271DE004EBC70804
:1059A000317C88F80E10F189A8F80C10CDF8009021
:1059B0006888042304AA296900F02EFBBDF81010A2
:1059C000A8F8101009F10400BDF812107F1C1FFA8E
:1059D00080F9A8F81210BFB26089B842DED80DE194
:1059E000307B022800D0FFDFE98908EBC100ADF869
:1059F00004003020ADF83400287B0A90001FC0B2AC
:105A00000F90002CEBD06181B5F81090002725E0B5
:105A1000CDF800906888696903AA0A9B00F0FCFA37
:105A20000A9804EBC70848441FFA80F908F10C02F1
:105A300004A90F980BF02EFE18B188F80EB0A8F844
:105A40000CB0BDF80C1001E0D4E0CFE0A8F81010C5
:105A5000BDF80E107F1CA8F81210BFB26089B842C2
:105A6000D6D8CBE00DA8009001AB2246294630469F
:105A7000FFF71DFBC2E0307B082805D0FFDF03E005
:105A8000307B082800D0FFDFE8891030ADF8040033
:105A90003620ADF83400002C3FD0A9896181F1890E
:105AA000A18127E0307B092800D0FFDFA88900F121
:105AB0000C01ADF804103721ADF83410002C2CD0B7
:105AC0006081E8890090AB89688804F10C0229693B
:105AD00056E0E8893921103080B2ADF80400ADF805
:105AE0003410002C74D0A9896181287A0E280AD03C
:105AF00002212173E989E181288A0090EB89688875
:105B00006969039A3CE00121F3E70DA8009001AB1D
:105B1000224629463046FFF75BFB6FE0307B0A28C0
:105B200000D0FFDF1220ADF80400ADF834704CB3A4
:105B3000A9896181A4F810B0A4F80EB084F80C9083
:105B40005CE020E002E031E039E042E0307B0B280D
:105B500000D0FFDF288AADF834701230ADF80400B1
:105B600084B104212173A9896181E989E181298AAC
:105B70002182688A00902B8A688804F11202696980
:105B800000F04AFA3AE0307B0C2800D0FFDF122008
:105B9000ADF80400ADF834703CB305212173A4F8CE
:105BA0000AB0A4F80EB0A4F810B027E00DA8009039
:105BB00001AB224629463046FFF75EFA1EE00DA8EB
:105BC000009001AB224629463046FFF7B8FB15E0AE
:105BD00036E03B21ADF80400ADF8341084B3A4F8EE
:105BE0000690A4F808B084F80AB007E0FFDF05E0EB
:105BF00010000020297A012919D0FFDFBDF8040028
:105C0000AAF800007CB1BDF834002080BDF8040083
:105C10006080BDF83400392805D03B2803D03C28EB
:105C200001D086F80CB011B00020BDE8F08F3C2107
:105C3000ADF80400ADF8341014B1697AA172DDE753
:105C4000FFE7AAF80000EEE72DE9F84356880F4673
:105C5000804615460521304609F09AFF040000D120
:105C6000FFDF123400943B46414630466A6806F036
:105C70004AF8B6E570B50D46052109F089FF040024
:105C800000D1FFDF294604F11200BDE8704005F0A5
:105C9000D6BE70B50D46052109F07AFF040000D18B
:105CA000FFDF294604F11200BDE8704005F0F4BEA4
:105CB00070B50546052109F06BFF040000D1FFDF38
:105CC00004F1080321462846BDE870400422ADE4F3
:105CD00070B50546052109F05BFF040000D1FFDF28
:105CE000214628462368BDE8704005229EE470B531
:105CF0000646052109F04CFF040000D1FFDF04F146
:105D0000120005F08FFE401D20F0030511E0011D7B
:105D100000880322431821463046FFF787FC0028FD
:105D20000BD0607BABB2684382B26068011D09F0A2
:105D3000ECFD606841880029E9D170BD70B50E4660
:105D4000054602F037FE040000D1FFDF012020727B
:105D500066726580207820F00F00C01C20F0F000F3
:105D600030302070BDE8704002F027BE2DE9F043CE
:105D70008BB00D461446814606A9FFF798FB002814
:105D800014D14FF6FF7601274FF420588CB1032031
:105D90008DF800001020ADF8100007A8059007AAA4
:105DA000204604A90BF095FC78B107200BB0BDE8A4
:105DB000F0830820ADF808508DF80E708DF80000C3
:105DC000ADF80A60ADF80C800CE00698A17801747B
:105DD0002188C1818DF80E70ADF80850ADF80C80A7
:105DE000ADF80A606A4602214846069BFFF788FB29
:105DF000DCE708B501228DF8022042F60202ADF878
:105E000000200A4603236946FFF73AFC08BD08B59F
:105E100001228DF8022042F60302ADF800200A4666
:105E200004236946FFF72CFC08BD00B587B079B1A3
:105E300002228DF800200A88ADF808204988ADF8C4
:105E40000A1000236A460521FFF75AFB07B000BD80
:105E50001020FBE709B1072312E40720704770B553
:105E600088B00D461446064606A9FFF720FB002819
:105E70000ED17CB10620ADF808508DF80000ADF8C9
:105E80000A40069B6A460821DC813046FFF738FB52
:105E900008B070BD05208DF80000ADF80850F0E79F
:105EA00000B587B059B107238DF80030ADF8082050
:105EB000039100236A460921FFF722FBC6E7102061
:105EC000C4E770B588B00C460646002506A9FFF762
:105ED000EEFA0028DCD106980121123005F0D4FD3D
:105EE0009CB12178062921D2DFE801F020050516B2
:105EF0000318801E80B2C01EE28880B20AB1A36877
:105F00001BB1824203D90C20C2E71020C0E704294C
:105F100004D0A08850B901E00620B9E7012913D0C8
:105F2000022905D004291CD005292AD00720AFE773
:105F300009208DF800006088ADF80800E088ADF811
:105F40000A00A068039023E00A208DF80000608812
:105F5000ADF80800E088ADF80A00A0680A250390B3
:105F600016E00B208DF800006088ADF80800A088CE
:105F7000ADF80A00E088ADF80C00A0680B2504908D
:105F800006E00C208DF8000060788DF808000C25E4
:105F90006A4629463046069BFFF7B2FA78E700B515
:105FA00087B00D228DF80020ADF8081000236A4656
:105FB0001946FFF7A5FA49E700B587B071B102228B
:105FC0008DF800200A88ADF808204988ADF80A103D
:105FD00000236A460621FFF793FA37E7102035E7DA
:105FE00070B586B0064601200D46ADF808108DF854
:105FF0000000014600236A463046FFF781FA04009C
:1060000008D12946304601F0BDFA0021304601F0A2
:10601000D7FA204606B070BDF8B51C4615460E46A8
:10602000069F09F0E7FE2346FF1DBCB231462A4613
:10603000009409F0D2FAF8BD30B41146DDE902420D
:106040003CB1032903D0002330BC04F05BB9012329
:10605000FAE71A8030BC704770B50C460546FFF76A
:106060002BFB2146284601F09CFA2846BDE87040EB
:10607000012101F0A5BA000018B18178012938D1B9
:1060800001E010207047018842F60112881A9142FF
:1060900031D018DC42F60102A1EB020091422AD075
:1060A0000CDC41B3B1F5C05F25D06FF4C0500818C7
:1060B00021D0A0F57060FF381BD11CE001281AD058
:1060C00002280AD117E0B0F5807F14D008DC01283F
:1060D00011D002280FD003280DD0FF2809D10AE0E3
:1060E000B0F5817F07D0A0F58070033803D0012878
:1060F00001D0002070470F2070470A281ED007DC0F
:1061000018D2DFE800F0191B1F1F171F231D1F21C6
:10611000102815D008DC0B2812D00C2810D00D2820
:1061200016D00F2806D10DE011280BD084280BD0F3
:1061300087280FD003207047002070470520704744
:10614000072070470F2070470420704706207047D3
:106150000C20704743F20200704738B50C4605002A
:1061600041D06946FEF7ACF9002819D19DF800101E
:10617000607861F3020060706946681CFEF7A0F960
:1061800000280DD19DF80010607861F3C5006070A3
:10619000A978C1F34101012903D0022905D00720C4
:1061A00038BD217821F0200102E0217841F0200162
:1061B0002170410704D0A978C90861F38610607086
:1061C000607810F0380F07D0A978090961F3C7107B
:1061D000607010F0380F02D16078400603D5207847
:1061E00040F040002070002038BD70B5044600200B
:1061F000088015466068FFF7B0FF002816D1208997
:10620000A189884211D860688078C0070AD0B1F5AA
:10621000007F0AD840F20120B1FBF0F200FB12101F
:10622000288007E0B1F5FF7F01D90C2070BD01F295
:1062300001212980002070BD10B50478137864F323
:10624000000313700478640864F341031370047846
:10625000A40864F3820313700478E40864F3C303AE
:1062600013700478240964F3041313700478640928
:1062700064F3451313700078800960F3861313707C
:1062800031B10878C10701D1800701D5012000E0B4
:10629000002060F3C713137010BD4278530702D07B
:1062A00002F0070306E012F0380F02D0C2F3C20377
:1062B00000E001234A7863F302024A70407810F04C
:1062C000380F02D0C0F3C20005E0430702D000F04F
:1062D000070000E0012060F3C5024A7070472DE915
:1062E000F04F95B00D00824612D01221284618F0CA
:1062F0006BFB4FF6FF7B05AA0121584607F065FAB4
:106300000024264637464FF420586FF4205972E097
:10631000102015B0BDE8F08F9DF81E0001280AD1AD
:10632000BDF81C1041450BD011EB09000AD0012823
:106330000CD002280CD0042C0ED0052C0FD10DE06F
:10634000012400E00224BDF81A6008E0032406E0FE
:106350000424BDF81A7002E0052400E00624BDF80C
:106360001A10514547D12C74BEB34FF0000810AA43
:106370004FF0070ACDE90282CDE900A80DF13C09F2
:106380001023CDF8109042463146584607F0D0FA17
:1063900008BBBDF83C002A46C0B210A90BF07AF940
:1063A000C8B9AE81CFB1CDE900A80DF1080C0AAE95
:1063B00040468CE84102132300223946584607F034
:1063C000B7FA40B9BDF83C00F11CC01EC0B22A1D8E
:1063D0000BF060F910B103209BE70AE0BDF829003B
:1063E000E881062C05D19DF81E00A872BDF81C009E
:1063F000288100208DE705A807F0F3F900288BD04D
:10640000FFF77BFE85E72DE9F0471C46DDE90978BB
:10641000DDF8209015460E00824600D1FFDF0CB15A
:10642000208818B1D5B11120BDE8F087022D01D028
:10643000012100E0002106F1140006F0B7F8A8F8E9
:10644000000002463B462946504603F0D2F8C9F800
:10645000000008B9A41C3C600020E5E71320E3E736
:10646000F0B41446DDE904528DB1002314B1022CBE
:1064700009D101E0012306E00D7CEE0703D025F0F1
:10648000010501230D742146F0BC03F03BBF1A80C7
:10649000F0BC70472DE9FE4F91461A881C468A468B
:1064A0008046FAB102AB494603F0A3F8050019D0C3
:1064B0004046A61C278809F0AFFC3246072629462D
:1064C0003B46009609F0BDF820882346CDE90050F0
:1064D0004A4651464046FFF7C3FF00202080012076
:1064E000BDE8FE8F0020FBE72DE9F04786B091461E
:1064F000DDE90E460F46824603AA05A904A8109DB1
:106500008DE807009846324621465046FFF77BFF4C
:10651000049909B1012200E000222A70002817D155
:10652000F84A03AB1060059A009104F11400CDE91C
:1065300001204A463946504606F0EFFB90B1082844
:106540000ED2DFE800F00407040D0D090B0B00204C
:1065500006B069E71120FBE70720F9E70820F7E715
:106560000320F5E7BDF80C100498CDE9000143467F
:10657000324621465046FFF773FFE8E72DE9F04326
:1065800089B00D46DDE9108781461C461646142168
:1065900003A818F03BFA012002218DF810108DF8A5
:1065A0000C008DF81170ADF8146064B1A278D207B8
:1065B00009D08DF81600E088ADF81A00A088ADF873
:1065C0001800A068079008A80095CDE90110424680
:1065D00003A948466B68FFF787FF09B0BDE8F08361
:1065E000F0B58BB00024064606940794072708945C
:1065F00005A80994019400970294CDE903400D4643
:1066000010232246304607F093F978B90AA806A964
:10661000019400970294CDE90310BDF814300022D4
:106620002946304606F05AFF002801D0FFF765FDE5
:106630000BB0F0BD06F0FABD2DE9FC410C468046DA
:10664000002602F0B7F9054620780D287ED2DFE853
:1066500000F0BC0713B325BD49496383AF959B0088
:10666000A848006820B1417841F010014170ADE0C8
:10667000404602F0CFF9A9E00421404609F088FA2B
:10668000070000D1FFDF07F11401404605F022FFAB
:10669000A5BB13214046FCF777F997E0042140465B
:1066A00009F076FA070000D1FFDFE088ADF80000BE
:1066B0000020B8819DF80000010704D5C00602D56E
:1066C000A088B88105E09DF8010040067ED5A0882D
:1066D000F88105B9FFDF22462946404601F066FCF5
:1066E000022673E0E188ADF800109DF8011009065C
:1066F0000FD5072803D006280AD00AE024E0042199
:10670000404609F045FA060000D1FFDFA088F0817D
:106710000226CDB9FFDF17E00421404609F038FA20
:10672000070000D1FFDF07F1140006F0B6FD90F07E
:10673000010F02D1E079000648D5387C022640F0EE
:106740000200387405B9FFDF224600E03DE029462B
:10675000404601F02BFC39E00421404609F018FACC
:10676000017C002D01F00206C1F340016171017C42
:1067700021F002010174E7D1FFDFE5E702260121E4
:10678000404602F079F921E00421404609F000FA80
:106790000546606800902089ADF804000122694632
:1067A000404602F08AF9287C20F0020028740DE0AF
:1067B000002DC9D1FFDFC7E7022600214046FFF7C1
:1067C00068FA002DC0D1FFDFBEE7FFDF3046BDE82D
:1067D000FC813EB50C0009D001466B4601AA0020A1
:1067E00007F028F920B1FFF788FC3EBD10203EBD20
:1067F00000202080A0709DF8050002A900F007008D
:10680000FDF77AFE50B99DF8080020709DF805004C
:1068100002A9C0F3C200FDF76FFE08B103203EBD20
:106820009DF8080060709DF80500C109A07861F32B
:106830000410A0709DF80510890961F3C300A070D1
:106840009DF80410890601D5022100E0012161F3C1
:1068500042009DF8001061F30000A07000203EBDD2
:1068600070B5144606460D4651EA040005D075B1D0
:1068700008460CF0A5FE78B901E0072070BD294656
:10688000304607F038F910B1BDE8704035E454B136
:1068900020460CF095FE08B1102070BD2146304610
:1068A000BDE8704095E7002070BD2DE9FC5F0C4607
:1068B00090460546002701780822007A3E46B2EB52
:1068C000111F7DD104F10A0100910A31821E4FF09F
:1068D000020A04F1080B0191092A72D2DFE802F0E2
:1068E000EDE005F528287BAACE006888042109F090
:1068F0004FF9060000D1FFDFB08928B152270726E3
:10690000C3E000004C02002051271026002C7DD04F
:106910006888A0800120A071A88900220099FFF753
:106920009FFF002873D1A8892081288AE081D1E0C7
:10693000B5F81290072824D1E87B000621D551270D
:1069400009F1140086B2002CE1D0A8890022009938
:10695000FFF786FF00285AD16888A08084F806A037
:10696000A88920810120A073288A2082A4F812908F
:10697000A88A009068884B46A969019A01F0F3FA49
:10698000A8E0502709F1120086B2002C3ED0A88959
:1069900000225946FFF764FF002838D16888A0809C
:1069A000A889E080287A072813D002202073288A3B
:1069B000E081E87BC0096073A4F81090A88A01E028
:1069C00085E082E0009068884B4604F11202A969D4
:1069D000D4E70120EAE7B5F81290512709F1140035
:1069E00086B2002C66D06888042109F0D1F883466D
:1069F0006888A080A88900220099FFF731FF00284D
:106A00006ED184F806A0A889208101E052E067E0F9
:106A10000420A073288A2082A4F81290A88A0090EB
:106A200068884B46A969019A01F09DFAA989ABF8DB
:106A30000E104FE06888FAF7F7FC074668880421D3
:106A400009F0A6F8064607B9FFDF06B9FFDF687B45
:106A5000C00702D05127142601E0502712264CB35C
:106A60006888A080502F06D084F806A0287B59465D
:106A700001F089FA2EE0287BA11DF9E7FE49A889DB
:106A80004989814205D1542706269CB16888A08097
:106A900020E053270BE06888A080A889E08019E0F7
:106AA0006888042109F074F800B9FFDF552708262B
:106AB000002CF0D1A8F8006011E056270726002C22
:106AC000F8D06888A080002013E0FFDF02E00128F2
:106AD00008D0FFDFA8F800600CB127806680002096
:106AE000BDE8FC9F57270726002CE3D06888A080CC
:106AF000687AA071EEE7401D20F0030009B1414320
:106B0000091D01EB4000704713B5DB4A00201071EE
:106B1000009848B10024684608F057FE002C02D1C6
:106B2000D64A009911601CBD01240020F4E770B51D
:106B30000D46064686B014465C21284617F066FFCF
:106B400004B9FFDFA0786874A2782188284601F094
:106B500044FA0020A881E881228805F1140130461A
:106B600005F09DFC6A460121304606F02EFE19E034
:106B70009DF80300000715D5BDF806103046FFF755
:106B80002FFD9DF80300BDF8061040F010008DF8B1
:106B90000300BDF80300ADF81400FF233046059A4A
:106BA00006F074FF684606F01CFE0028E0D006B030
:106BB00070BD10B50C4601F1140005F0A7FC0146AC
:106BC000627C2046BDE8104001F03CBA70B5054635
:106BD000042108F0DDFF040000D1FFDF04F11401FF
:106BE0000C46284605F076FC21462846BDE8704054
:106BF00005F077BC70B58AB00C460646FAF714FC6F
:106C0000050014D02878222827D30CB1A08890B191
:106C100001208DF80C0003208DF8100000208DF865
:106C2000110054B1A088ADF81800206807E043F2C5
:106C300002000AB070BD0920FBE7ADF8180005900E
:106C40000421304608F0A4FF040000D1FFDF04F166
:106C5000140005F072FC000701D40820E9E701F0F8
:106C6000A9FE60B108A802210094CDE9011095F8B1
:106C7000232003A930466368FFF736FCD9E71120CB
:106C8000D7E72DE9F04FB2F802A0834689B0154648
:106C900089465046FAF7C8FB07460421504608F0DB
:106CA00077FF0026044605964FF002080696ADF8D9
:106CB0001C6007B9FFDF04B9FFDF4146504603F00F
:106CC00088FE60B907AA06A905A88DE80700424614
:106CD000214650466368FFF796FB00B1FFDF664828
:106CE00007AB0660DDE9051204F11400CDF8009051
:106CF000CDE90320CDE9013197F8232059465046CC
:106D00006B6805F063FC06000AD0022E04D0032E47
:106D100014D0042E00D0FFDF09B03046BDE8F08F5C
:106D2000BDF81C000028F7D00599CDE900104246B7
:106D3000214650466368FFF793FBEDE7687840F023
:106D400008006870E8E72DE9F04F9BB004464FF06B
:106D500000084948ADF85480ADF83080ADF8508057
:106D6000A0F80880ADF81480ADF81880ADF8208048
:106D7000ADF81C80007916460D464746012808D01C
:106D8000022806D0032804D0042802D008201BB013
:106D9000C4E720460CF0D0FBD0BB28460CF0CCFB5F
:106DA000B0BB60680CF015FC90BB606848B16089AE
:106DB0002189884202D8B1F5007F01D90C20E6E78D
:106DC00080460BAA06A92846FFF70FFA0028DED155
:106DD00068688078C0F34100022808D19DF8190046
:106DE00010F0380F03D028690CF0EAFB80B905A930
:106DF0002069FFF7B2F90028C9D1206950B1607845
:106E000080079DF8150000F0380002D5C0B301E0FE
:106E100011E0A8BB9DF8140080060ED59DF8150062
:106E200010F0380F03D060680CF0CAFB18B9606826
:106E30000CF0CFFB08B11020A9E707A96069FFF7A4
:106E40008CF90028A3D1606940B19DF81D0000F0C5
:106E5000070101293FD110F0380F3CD008A9A069E3
:106E6000FFF77BF9002892D19DF81C00800632D4F0
:106E70009DF82000800604E04C0200201400002051
:106E800029E028D4A06940B19DF8210000F0070155
:106E9000012920D110F0380F1DD0E06818B100781A
:106EA000C8B11C2817D20EAA611C2046FFF7C4F9EE
:106EB0000120B94660F30F27BA4607468DF84E0009
:106EC00042F60300ADF84C000DF13B0217A928680B
:106ED0000AF0FFFB08B1072059E79DF85C0016A9EE
:106EE000CDF80090C01CCDE9019100F0FF0B00230C
:106EF0000BF20122514613A806F0AAFBF0BBBDF825
:106F000058000990FE482A8929690092CDE90110AC
:106F10006B89BDF82C202868069906F099FB0100C2
:106F20007ED120784FF0020AC10601D480062BD50D
:106F3000ADF80C90606950B907A906A8FFF7ADF944
:106F40009DF81D0020F00700401C8DF81D009DF8E5
:106F50001C008DF84E7040F0C8008DF81C0042F601
:106F60000210ADF84C000CA903AACDF800A0CDE9A1
:106F70000121002340F2032213A800E01EE007993C
:106F800006F066FB01004BD1DD484D4608385B46F4
:106F90000089ADF839000EA8CDE90290CDF8049033
:106FA000CDF810904FF007090022CDF80090BDF801
:106FB00058104FF6FF7006F091FA10B1FFF79DF8E8
:106FC000E5E69DF83800000625D52946012060F346
:106FD0000F218DF84E704FF42450ADF84C00ADF8F1
:106FE000105062789DF81000002362F300008DF8C5
:106FF00010006278CDF800A0520862F341008DF8CD
:10700000100004AACDE9012540F2032213A806F0DE
:107010001FFB010004D1606888B32069A8B900E0B3
:1070200086E005A906A8FFF738F96078800706D43E
:107030009DF8150020F038008DF8150005E09DF84A
:10704000140040F040008DF814008DF84E7042F6A8
:107050000110ADF84C00208940F20121B0FBF1F2A3
:1070600001FB1202606814ABCDF80080CDE901038A
:10707000002313A8059906F0EBFA010058D12078F7
:10708000C00729D0ADF80C50A06950B908A906A8CE
:10709000FFF703F99DF8210020F00700401C8DF850
:1070A00021009DF820008DF84E7040F040008DF8D2
:1070B000200042F60310ADF84C0015A903AACDF844
:1070C00000A0CDE90121002340F2032213A8089972
:1070D00006F0BEFA01002BD1E06868B32946012012
:1070E00060F30F218DF84E7042F60410ADF84C009D
:1070F000E068002302788DF8602040788DF8610008
:10710000E06818AA4088ADF86200E06800798DF860
:107110006400E068C088ADF86500CDF80090CDE966
:1071200001254FF4027213A806F092FA010003D071
:10713000099800F0B3FF2AE671480321083801716D
:1071400056B100893080BDF850007080BDF8300025
:10715000B080BDF85400F080002018E670B501251D
:107160008AB016460B46012802D0022816D104E048
:107170008DF80E504FF4205003E08DF80E5042F67B
:107180000100ADF80C005BB10024601C60F30F241B
:1071900004AA08A918460AF09CFA18B1072048E585
:1071A000102046E504A99DF820205548CDE900218E
:1071B000801E02900023214603A802F2012206F05D
:1071C00047FA10B1FEF799FF33E54D4808380EB184
:1071D000C1883180057100202BE5F0B593B00746DA
:1071E00001268DF83E6041F60100ADF83C0012AA80
:1071F0000FA93046FFF7B2FF002848D1404C0025C8
:10720000083CE7B31C2102A817F000FC9DF8080019
:107210008DF83E6040F020008DF8080042F6052011
:10722000ADF83C000E959DF83A00119520F006004F
:10723000801C8DF83A009DF838006A4620F0FF0067
:107240008DF838009DF8390009A920F0FF008DF86D
:1072500039000420ADF82C00ADF830000EA80A90DB
:1072600011A80D900FA80990ADF82E5002A8FFF7B5
:107270006AFD00280BD1BDF80000608100E008E045
:10728000BDF80400A081401CE0812571002013B0EE
:10729000F0BD6581A581BDF84800F4E72DE9F74F01
:1072A0001749A0B00024083917940A79A146012A89
:1072B00004D0022A02D0082023B02FE5CA888242D7
:1072C00001D00620F8E721988A46824201D10720A2
:1072D000F2E701202146ADF848004FF6FF7860F351
:1072E0000F21ADF84A808DF86E0042F6020B069130
:1072F0008DF87240ADF86CB0ADF870401CA901E09B
:10730000540200201391ADF8508012A806F08DFAB7
:1073100000252E462F460DAB072212A9404606F047
:1073200087FA78B10A285DD195B38EB3ADF8645071
:10733000ADF866609DF85E008DF8144019AC012828
:1073400064D06BE09DF83A001FB3012859D1BDF815
:10735000381059451FD118A809A901940294CDE904
:10736000031007200090BDF836101023002240467D
:1073700006F0DEFAB0BBBDF86000042801D0062894
:107380004AD1BDF82410219881423AD10F2093E7C9
:107390003AE0012835D1BDF83800B0F5205F03D0C0
:1073A00042F6010188422CD1BAF80600BDF8361029
:1073B000884201D1012700E0002705B19EB1219844
:1073C00081421ED118A809AA01940294CDE9032094
:1073D000072000900D4610230022404606F0A8FA30
:1073E00000B902E02DE04E460BE0BDF86000022837
:1073F00001D0102810D1C0B217AA09A90AF04AF981
:1074000050B9BDF8369086E7052055E705A917A8BD
:10741000221D0AF05EF908B103204DE79DF8140023
:107420000023001DC2B28DF8142022980092CDE9ED
:1074300001401BA8069906F00BF910B902228AF840
:107440000420FEF75AFE37E710B50B46401E88B001
:1074500084B205AA00211846FEF7EEFE00200DF1C9
:10746000080C06AA05A901908CE8070007200090E7
:107470000123002221464FF6FF7006F02FF8044644
:10748000BDF81800012800D0FFDF2046FEF735FECA
:1074900008B010BDF0B5FF4F044687B038790E46EE
:1074A000032804D0042802D0082007B0F0BD04AAA5
:1074B00003A92046FEF799FE0500F6D160688078A2
:1074C000C0F3410002280AD19DF80D0010F0380FDA
:1074D00005D020690CF074F808B11020E5E7208988
:1074E00005AA21698DE807006389BDF8102020688E
:1074F000039906F0ADF810B1FEF7FFFDD5E716B120
:10750000BDF814003080042038712846CDE7F8B566
:107510000C0006460BD001464FF6FF7500236A4665
:10752000284606F087FA20B1FEF7E7FDF8BD1020E7
:10753000F8BD69462046FEF710FE0028F8D1A07875
:10754000314600F001032846009A06F09FFAEBE767
:1075500030B587B0144600220DF1080C05AD01923C
:107560008CE82C00072200920A46014623884FF639
:10757000FF7005F0B3FFBDF814102180FEF7BDFDCC
:1075800007B030BD70B50D46042108F001FB0400C2
:1075900000D1FFDF294604F11400BDE8704004F07B
:1075A000C5BF70B50D46042108F0F2FA040000D101
:1075B000FFDF294604F11400BDE8704004F0D9BF94
:1075C00070B50D46042108F0E3FA040000D1FFDF96
:1075D000294604F11400BDE8704004F0F1BF70B515
:1075E0000546042108F0D4FA040000D1FFDF21464B
:1075F00028462368BDE870400122FEF74BBF70B5F6
:107600000646042108F0C4FA040000D1FFDF04F1AB
:10761000140004F07BFF401D20F0030511E0011D64
:1076200000880022431821463046FEF733FF002829
:107630000BD0607CABB2684382B2A068011D08F039
:1076400064F9A06841880029E9D170BD70B505468C
:10765000042108F09DFA040000D1FFDF21462846EE
:107660006368BDE870400222FEF714BF70B50E4695
:10767000054601F09FF9040000D1FFDF01202072D0
:1076800066726580207820F00F00001D20F0F00069
:1076900040302070BDE8704001F08FB910B504464D
:1076A000012900D0FFDF2046BDE810400121FEF790
:1076B000F0BA2DE9F04F97B04FF0000A0C00834666
:1076C000ADF814A0D04619D0E06830B1A068A8B1D8
:1076D0000188ADF81410A0F800A05846F9F7A4FEF0
:1076E000070043F2020961D0387822285CD30421D4
:1076F000584608F04DFA050005D103E0102017B0F8
:10770000BDE8F08FFFDF05F1140004F0FFFE401D1F
:1077100020F00306A078012803D0022801D007201A
:10772000EDE7218807AA584606F04FF830BB07A8B6
:1077300006F057F810BB07A806F053F848B99DF8B3
:107740002600012805D1BDF82400A0F524510239F6
:1077500002D04FF45050D2E7E068B0B1CDE902A0BA
:107760000720009005AACDF804A00492A2882188E1
:10777000BDF81430584605F0B1FE10B1FEF7BDFC5F
:10778000BDE7A168BDF8140008809DF81F00C00681
:1077900002D543F20140B2E70B9838B1A1780078E6
:1077A000012905D080071AD40820A8E74846A6E793
:1077B000C007F9D002208DF83C00A8684FF00009FE
:1077C000A0B1697C4288714391420FD98AB2B3B2A9
:1077D000011D08F050F88046A0F800A006E0032044
:1077E0008DF83C00D5F800804FF001099DF820008D
:1077F00010F0380F00D1FFDF9DF820002649C0F3BC
:10780000C200084497F8231010F8010C884201D9EF
:107810000F2074E72088ADF8400014A90095CDE949
:107820000191434607220FA95846FEF75DFE002846
:1078300091D19DF8500050B9A078012807D1687CFB
:10784000B3B2704382B2A868011D08F028F8002086
:1078500055E770B5064615460C460846FEF70CFC83
:10786000002805D12A4621463046BDE8704075E41F
:1078700070BD13E570B51E4614460D000ED06CB1F8
:10788000616859B160B10349C988814208D00720B5
:1078900070BD00004C02002072ED01001020F7E7DF
:1078A0002068FEF7E9FB0028F2D13246214628463F
:1078B000BDE87040FFF747BA70B515460C0006D01A
:1078C00038B1FE490989814203D00720E0E7102042
:1078D000DEE72068FEF7D0FB0028D9D129462046F4
:1078E000BDE87040D6E570B5064686B00D46144634
:1078F00010460BF047FED0BB60680BF06AFEB0BBD1
:10790000A6F57F40FF3803D03046F9F78DFD80B1F2
:1079100028466946FEF7E3FC00280CD19DF81010BC
:107920000F2008293CD2DFE801F008060606060A07
:107930000A0843F2020006B0AAE70320FBE79DF81D
:107940000210012908D1BDF80010B1F5C05FF2D0D6
:107950006FF4C052D142EED09DF8061001290DD12E
:10796000BDF80410A1F52851062907D200E028E04F
:10797000DFE801F0030304030303DCE79DF80A10CA
:1079800001290ED1BDF80810B1F5245FD3D0A1F5BF
:1079900024510239CFD00129CDD0022901D1CAE723
:1079A000FFDF606878B9002305AA2946304606F053
:1079B00041F810B1FEF7A1FBBDE79DF81400800669
:1079C00001D41020B7E76188224628466368FFF794
:1079D000BFFDB0E72DE9F043814687B088461446E5
:1079E00010460BF0CFFD18B1102007B0BDE8F083B2
:1079F000002306AA4146484606F01CF818B100BF0D
:107A0000FEF77BFBF1E79DF81800C00602D543F2B4
:107A10000140EAE70025072705A801950097029590
:107A2000CDE9035062884FF6FF734146484605F0A2
:107A30007FFF060013D160680BF0A4FD60B9606899
:107A40000195CDE90250009704952388628841464C
:107A5000484605F06DFF0646BDF81400208030460C
:107A6000CEE739B1954B0A889B899A4202D843F2F6
:107A7000030070471DE610B586B0904C0423ADF8A6
:107A80001430638943B1A4898C4201D2914205D953
:107A900043F2030006B010BD0620FBE7ADF810105E
:107AA000002100910191ADF8003002218DF8021003
:107AB00005A9029104A90391ADF812206946FFF7C8
:107AC000F8FDE7E72DE9FC4781460E4608460BF036
:107AD00033FD88BB4846F9F7A7FC5FEA00080AD0E7
:107AE00098F80000222829D30421484608F050F8CD
:107AF000070005D103E043F20200BDE8FC87FFDF89
:107B000007F1140004F019FD05463078012803D070
:107B1000022804D00720F0E7A8070FD502E015F0EF
:107B20001C0F0BD0B079341DC00709D0E08838B1E4
:107B3000A0680BF001FD18B11020DEE70820DCE79B
:107B400032782088002628B3A0F201130721112BD8
:107B500018D20CD2DFE803F00B090D0B1D0B121D20
:107B6000100B0B1D1D1D1D0B1D00022A11D10846F7
:107B7000C3E7012AFBD00CE02A0700E0EA06002A4E
:107B8000F5DA06E0A0F5C0721F2A02D97D3A022A72
:107B9000EDD8C6B200F00EFF50B198F82300CDE941
:107BA0000006FA89234639464846FEF7E7FCA4E773
:107BB0001120A2E72DE9F04F8BB01F4615460C4669
:107BC00083460026F9F730FC28B10078222805D238
:107BD00008200BB094E543F20200FAE7B80801D0A0
:107BE0000720F6E7032F00D100274FF6FF79CCB12D
:107BF000022D73D320460BF0ECFC30B904EB0508E2
:107C0000A8F101000BF0E5FC08B11020E1E7AD1E82
:107C1000AAB22146484605F0C2FF38F8021C884245
:107C20005CD1ADB22549B80702D58889401C00E077
:107C300001201FFA80F8F80701D08F8900E04F4635
:107C400005AA4146584605F0C0FD4FF0070A4FF01F
:107C50000009ACB3204608E0408810283ED8361D05
:107C6000304486B2AE4239D2A01902884245F3D3DD
:107C700054E000BF9DF8170002074FD584B304EB12
:107C80000608361DB8F80230B6B2102B26D89A195D
:107C9000AA4223D8B8F8002091421FD1C00620D5AF
:107CA000CDE900A90DF1080C0AAAA11948468CE8F3
:107CB0000700B8F800100022584603E04C020020EC
:107CC0002CE00BE005F00AFC10B1FEF716FA80E795
:107CD000B8F80200BDF82810884202D00B2078E7DF
:107CE00004E0B8F80200304486B206E0C00604D5CD
:107CF0005846FEF775FC002888D19DF81700BDF89E
:107D00001A1020F010008DF81700BDF81700ADF81C
:107D10000000FF235846009A05F0B8FE05A805F0BC
:107D200060FD18B9BDF81A10B942A3D9042158460C
:107D300007F02EFF040000D1FFDFA2895AB1CDE980
:107D400000A94D46002321465846FEF717FC00289F
:107D5000BDD1A5813DE700203BE72DE9FF4F8BB06A
:107D60001E4617000D464FF0000412D0B00802D096
:107D700007200FB0C4E4032E00D100265DB10846F1
:107D80000BF01EFC28B93888691E08440BF018FC5B
:107D900008B11020EDE7C74AB00701D5D18900E04E
:107DA0000121F0074FF6FF7802D0D089401E00E095
:107DB000404686B206AA0B9805F007FD4FF0000971
:107DC0004FF0070B0DF1140A39E000BF9DF81B00BE
:107DD000000734D5CDF80490CDF800B0CDF8089068
:107DE000CDE9039A434600220B9805F0A1FD60BB44
:107DF00005B3BDF814103A8821442819091D8A4298
:107E000030D3BDF81E2020F8022BBDF8142020F836
:107E1000022BCDE900B9CDE90290CDF810A0BDF854
:107E20001E10BDF8143000220B9805F081FD08B13A
:107E300003209EE7BDF814002044001D84B206A86C
:107E400005F0CFFC20B10A2806D0FEF756F990E7DE
:107E5000BDF81E10B142B9D934B17DB13888A11C2A
:107E6000884203D20C2084E7052082E72246294677
:107E7000404605F094FE014628190180A41C3C8070
:107E8000002076E710B504460BF07CFB08B110200B
:107E900010BD8848C0892080002010BDF0B58BB08F
:107EA0000D460646142103A816F0B0FD01208DF8FA
:107EB0000C008DF8100000208DF81100ADF8145062
:107EC0003046F9F7B1FA48B10078222812D30421DC
:107ED000304607F05DFE040005D103E043F20200E6
:107EE0000BB0F0BDFFDF04F11400074604F025FBE2
:107EF000800601D40820F3E7207C022140F0010035
:107F0000207409A80094CDE90110072203A9304686
:107F10006368FEF7E9FA20B1217C21F001012174A8
:107F2000DEE729463046FDF7A5FE08A9384604F0ED
:107F3000F3FA00B1FFDFBDF82040172C01D2172063
:107F400000E02046A84201D92C4602E0172C00D2BE
:107F5000172421463046FFF724FB21463046FDF723
:107F6000ABFB0020BCE7F8B51C4615460E46069F45
:107F700007F040FF2346FF1DBCB231462A4600945D
:107F800007F02BFBF8BD70B50C4605460E212046C8
:107F900016F01AFD002020802DB1012D01D0FFDF49
:107FA00076E4062000E00520A07171E410B5488059
:107FB0000878134620F00F00001D20F0F0008030FC
:107FC0000C4608701422194604F1080016F0C2FC91
:107FD00000F0F3FC3748046010BD2DE9F047DFF8EE
:107FE000D890491D064621F0030117460C46D9F8E2
:107FF000000007F008FC050000D1FFDF4FF000088B
:108000003560A5F800802146D9F8000007F0FBFB99
:10801000050000D1FFDF7560A5F800807FB104FB8B
:1080200007F1091D0BD0D9F8000007F0ECFB0400A4
:1080300000D1FFDFB460C4F80080BDE8F087C6F867
:108040000880FAE72DE9F0411746491D21F00302A7
:10805000194D064601681446286807F0FFFB2246C2
:108060007168286807F0FAFB3FB104FB07F2121DA4
:1080700003D0B168286807F0F1FB042007F030FD59
:108080000446042007F034FD201A012804D1286892
:10809000BDE8F04107F0ACBBBDE8F08110B50C467F
:1080A00005F05FFB00B1FFDF2046BDE81040FEF7A2
:1080B00024B800004C020020140000204FF0E02201
:1080C0004FF400410020C2F880111D4908701D497D
:1080D00090020860704770B5194D04462878A04298
:1080E00002D00CB100B1FFDF2878A0420DD01649B4
:1080F000144A2C700020CCB1134E144B1436151FAB
:10810000012C03D0022C08D0FFDF70BD08600220D4
:10811000086033604FF0407005E00860032008609D
:1081200033604FF400001060286070BD0860086084
:108130004FF06070106070BD00B5FFDF00BD000043
:108140001800002008F5014000F500405C02002006
:1081500038B50C468288817B19B14189914200D99A
:108160000A462280C188121D90B26A4606F054FE6B
:10817000BDF80000032800D30320C1B2208800F01E
:1081800095FF38BD38B50C468288817B19B10189CD
:10819000914200D90A462280C188121D90B26A46D7
:1081A00006F03AFEBDF80000022800D30220C1B25A
:1081B000208800F07BFF401CC0B238BD2DE9FF5F76
:1081C0000C46FB4981462C22D1E90201CDE902018E
:1081D00009F1030020F00301C91C21F00301009103
:1081E0006846114607F0F1FAF24E002C02D1F2492E
:1081F000009A8A60009901440091357E05F10105DD
:1082000004D1E8B209F0ECF900B1FFDF00984FF0BB
:10821000000B00EB0510C01C20F0030100915CB9BD
:10822000307A727A81F800B01044C2B2B08B80B25A
:1082300005F01FF900B1FFDF0098F16908440090D4
:108240002146684600F0FCFE0098C01C20F00300A8
:108250000090737AB27A317A04B1002007F0ABFB58
:108260000099084400902146684600F02AFF002744
:108270003D46B24696F801800CE0284600F0C3FE69
:10828000064681788088FDF7AEFA71786D1C00FB98
:108290000177EDB24545F0D10098C01C20F00300F5
:1082A000009004B100203946FDF7A8FA0099002794
:1082B000084400903D469AF801800CE0284600F002
:1082C000A2FE0646C1788088FEF715FC71786D1C09
:1082D00000FB0177EDB24545F0D10098C01C20F0BD
:1082E0000300009004B100203946FEF70DFC009910
:1082F0004FF000080844009045469AF801700EE0DF
:10830000284600F080FE0646807B30B106F108006A
:1083100001F0A7FE727800FB02886D1CEDB2BD4231
:10832000EED10098C01C20F00300009004B10020A2
:10833000414601F09AFE00990844C01D20F0070252
:108340000092ECBB9D49002003F055FA05F0F2FBCA
:1083500099484178C06805F085FD97481030C0788D
:108360008DF8040010B1012804D005E001208DF83B
:10837000040001E08DF804B001A805F0B5FEF9F79E
:1083800072FF8C4802AA00210C30FAF755FE00B1AA
:10839000FFDF9AF81900FEF720FF00B1FFDF8548E4
:1083A0004FF4F671443016F031FB8248042144301A
:1083B00080F8E91180F8EA11062180F8EB1100E05D
:1083C00001E003210171009904B0A1EB0900BDE8AF
:1083D000F09F70B5774C06464434207804EB401586
:1083E000E078083590B9A01990F8E80100280ED07F
:1083F000A0780F2800D3FFDF2021284616F006FBC7
:10840000687866F3020068700120E070284670BD4D
:108410002DE9F04105460C460027007805219046DD
:108420003E46B1EB101F00D0FFDF287A50B1012883
:108430000ED0FFDFA8F800600CB127806680002016
:10844000BDE8F0810127092674B16888A08008E0A2
:108450000227142644B16888A0802869E060A88AB1
:108460002082287B2072E5E7A8F80060E7E710B5D6
:10847000514C6068C11D21F00701814200D0FFDF2F
:108480004C480121002201704270017203234372A3
:1084900081720273052282821F22C282417348A226
:1084A00002610A22027641764FF4B061C1616168CF
:1084B000416010BD30B5404C1568636810339D4273
:1084C00002D20420136030BD3A4B5D785A6802EB4B
:1084D0000512107051700320D08017209080012069
:1084E000D0709070002090735878401C587060686D
:1084F00010306060002030BD70B506462D48002465
:10850000457807E0204600F07EFD0178B14204D0B6
:10851000641CE4B2AC42F5D1002070BDF7B507464B
:1085200008780C4610B3FFF7E7FF0546A7F12006D1
:10853000202F06D0052E19D2DFE806F00F2B2B15C1
:108540001A0000F06BFD0DB1697800E00021401ABF
:10855000A17880B20844FF2808D8A07830B1A0885C
:10856000022831D202E0608817282DD20720FEBDF4
:10857000207AE0B161881729F8D3A1881729F5D3AB
:10858000A1790029F2D0E1790029EFD0402804D95F
:10859000ECE7242F18D1207A48B161884FF6FB70A0
:1085A000814202D8A18881420ED90420FEBD0BE091
:1085B00078ED0100680300201C000020000000206E
:1085C0006E5246357800000065B9207802AA012174
:1085D000FFF770FF0028E9D12078FFF78DFF050035
:1085E00000D1FFDF052E18D2DFE806F0030B0E08DE
:1085F0001100A0786870A088E8800FE06088A880EB
:108600000CE0A078A87009E0A078E87006E054F8C3
:10861000020FA8606068E86000E0FFDF0020C5E7A7
:108620001E2829D00EDC0C2822D008DC092825D2EF
:10863000DFE800F013241524241C1C181A0012284B
:108640001CD119E0302817D018DDA0F13A0003281A
:1086500014D2DFE800F00F1309000020704743F246
:1086600002007047042070470D2070470F207047AC
:10867000082070471120704707207047032070477B
:1086800010B5007800F0010006F0BDFBBDE8104019
:10869000C6E70EB5017801F001018DF800104178B0
:1086A00001F001018DF801100178C1F340018DF84E
:1086B00002104178C1F340018DF803100178890858
:1086C0008DF80410417889088DF8051081788DF8AF
:1086D0000610C1788DF8071000798DF808006846FB
:1086E00005F021FDFFF79CFF0EBD2DE9F84FDFF8E7
:1086F000F883FE4C00261FE0012000F025FD01203C
:10870000FFF767FE05462C214746D8F8080007F01A
:108710007AF8686000B9FFDF686805F0D6FBA8B199
:108720002846F9F7E3F8284600F014FD20B92C227A
:108730006968B86807F092F894F9E9010428DBDA6F
:10874000022007F0CDF907460025A6E02C22696833
:10875000D8F8080007F082F8F2E7B8F802104046AF
:10876000491C89B2A8F80210B94201D30021418006
:108770000221B8F8020007F00BFA002865D0B8F81B
:108780000200694606F0B2FAFFF74AFF00B1FFDFC8
:108790009DF8000078B1B8F8020007F03DFB5FEAF1
:1087A000000900D1FFDF484606F0ABFD18B1B8F86C
:1087B000020002F0FDF8B8F8020007F01BFB5FEAC8
:1087C000000900D1FFDF484606F093FDE8BB032116
:1087D000B8F8020007F0DCF95FEA000B48D1FFDFD0
:1087E00046E000BFDBF8100010B10078FF2849D048
:1087F000022000F0A9FC0220FFF7EBFD824648466C
:1088000006F083FECAF8040000B9FFDFDAF80400BE
:1088100006F04BFF002100900170B8F8021050469E
:10882000AAF8021001F0CAFD484606F040FF00B960
:10883000FFDF504600F08EFC18B99AF801000007DF
:1088400004D50099CBF8101012E024E0DBF81000FA
:1088500038B10178491C11F0FF01017008D1FFDF28
:1088600006E000221146484600F0CBFB00B9FFDFCE
:1088700094F9EA01022805DBB8F8020001F063FD73
:108880000028AFD194F9E901042804DB484606F03A
:1088900072FF00B101266D1CEDB2BD4204D294F905
:1088A000EA010228BFF659AF002E7FF423AFBDE8DE
:1088B000F84F032000F048BC10B58B4CE06008680E
:1088C0002061AFF2D91002F0FEFF607010BD874842
:1088D0000021443801708448017085494160704727
:1088E00070B505464FF080500C46D0F8A410491CD6
:1088F00005D1D0F8A810C9430904090C0BD050F8D1
:10890000A01F01F001012970416821608068A080EA
:10891000287830B970BD062120460AF0E8FA012017
:108920002870607940F0C000607170BD70B54FF084
:1089300080540D46D4F88010491C0BD1D4F8841013
:10894000491C07D1D4F88810491C03D1D4F88C10E5
:10895000491C0CD0D4F880100160D4F88410416018
:10896000D4F888108160D4F88C10C16002E0102126
:108970000AF0BDFAD4F89000401C0BD1D4F8940052
:10898000401C07D1D4F89800401C03D1D4F89C00B7
:10899000401C09D054F8900F286060686860A06897
:1089A000A860E068E86070BD2846BDE8704010210E
:1089B0000AF09DBA4D4800790BE570B54B4CE07854
:1089C00030B3207804EB4010407A00F007002044D8
:1089D00090F9E801002800DCFFDF2078002504EB97
:1089E0004010407A00F00700011991F8E801401E9C
:1089F00081F8E8012078401CC0B220700F2800D117
:108A00002570A078401CA0700AF0ACF9E57070BD2C
:108A1000FFDF70BD3EB50546032107F0B9F80446F7
:108A2000284607F0E7F9054604B9FFDF206918B1C9
:108A30000078FF2800D1FFDF01AA6946284600F030
:108A4000E0FA60B9FFDF0AE0002202A9284600F040
:108A5000D8FA00B9FFDF9DF8080000B1FFDF9DF8EC
:108A60000000411E8DF80010EED220690199884265
:108A700001D1002020613EBD70B50546A0F57F40C4
:108A80000C46FF3800D1FFDF012C01D0FFDF70BDA5
:108A9000FFF790FF040000D1FFDF207820F00F00E7
:108AA000401D20F0F00050302070658000202072C2
:108AB00001202073BDE870407FE72DE9F0411646A4
:108AC0000D460746FFF776FF040000D1FFDF207850
:108AD00020F00F00401D20F0F00050302070678023
:108AE00001202072286805E01C000020AC03002053
:108AF000281200202061A888A0822673BDE8F041DA
:108B00005BE77FB5FFF7F8FC040000D1FFDF02A9A7
:108B10002046FFF71DFB054603A92046FFF732FB61
:108B20008DF800508DF80100BDF80800001DADF86B
:108B30000200BDF80C00001DADF80400E088ADF89F
:108B40000600684606F049F9002800D0FFDF7FBD27
:108B50002DE9F047DFF8F8930546002799F8000063
:108B600010B10820BDE8F08728460AF00BFD08B1D7
:108B70001020F7E7F74C207808B9FFF778FC607A07
:108B8000217A0844C6B200F049FAB04207D2301A3E
:108B9000C1B22A460020FFF78DFC0700E2D1D9F8C8
:108BA00004004E46C01C20F00300C9F8040000F089
:108BB00044FB716800EB010801214046FFF7FEFA13
:108BC000064629684044884202D8B6F5803F15D34E
:108BD00028600020FFF790FC05000DD005F1130080
:108BE000D9F8041020F003004E46884200D0FFDF81
:108BF0006078401E607075600420B3E70021404635
:108C0000FFF7DCFA0446A64200D0FFDF04EB0801C0
:108C1000C9F8041029604FF6FF71A9F8021001216C
:108C200089F8001038469DE72DE9F0410446C84810
:108C300017460D46007810B10820BDE8F0810846BF
:108C40000AF07AFC08B11020F7E7C24E307808B974
:108C5000FFF70DFC601E1E2807D8012C3FD1287895
:108C6000FE283CD830760020E7E7A4F120001F283A
:108C700005D8E0B23A462946BDE8F0414EE4A4F1F9
:108C800040004FF000081F2821D8402C02D0412C72
:108C900025D117E0687829780C18A97881421ED868
:108CA000FF2C08D808F080FE07460AF014F8381A9E
:108CB000801EA04201DA1220BFE728883081A87800
:108CC000B07224E02846BDE8F04100F06BBAA4F190
:108CD000A0001F2803D8A02C03D0A12C06D0072069
:108CE000ABE7287800F00100707610E029680920D1
:108CF000F829A2D38A07A0D1727B02F00302012ACD
:108D000004D1F28AD73293B28B4296D8F1614046B1
:108D100093E72DE9F04781460E4608460AF032FCFB
:108D200048B948460AF04CFC28B909F1030020F084
:108D30000301494501D0102014E786484FF0000A8E
:108D40004430817869B14178804600EB41140834A1
:108D5000378832460021204600F00AFA050004D088
:108D600027E0A6F800A00520FCE6B9F1000F24D00A
:108D70003088B84201D90C251FE0607800F0070563
:108D8000284600F0E1F908EB0507324697F8E801BC
:108D90004946401C87F8E801204607F5F47700F0C3
:108DA000E7F905463878401E3870032000F0CCF90A
:108DB0002DB10C2D01D0A6F800A02846D2E660788F
:108DC000634E00F00701012923D002290CD00329AA
:108DD00033D0FFDF98F801104046491CC9B288F82B
:108DE00001100F2934D035E0616821B1000702D4A9
:108DF0006088FFF70FFE98F8EA014746012802D184
:108E0000707802F07FFD97F9EA010428E2DBFFDFCA
:108E1000E0E7616819B12C22B06806F01FFD98F8F0
:108E2000E9014746032802D1707802F06BFD97F9FB
:108E3000E9010428CEDBFFDFCCE7C00602D560885D
:108E4000FFF7E8FD98F9EB010628C3DBFFDFC1E778
:108E500080F801A08178491E8170617801F00701D6
:108E600001EB080090F8E811491C80F8E811A4E72C
:108E700070B50D4604460AF05FFB18B928460AF0A3
:108E800081FB08B1102070BD29462046BDE8704026
:108E900008F0DDBB70B5044615460E4608460AF0DC
:108EA0004BFB18B928460AF06DFB08B1102070BDC5
:108EB000022C03D0102C01D0092070BD2A46314667
:108EC000204608F0E7FB0028F7D0052070BD70B5FC
:108ED00014460D4606460AF02FFB38B928460AF01C
:108EE00051FB18B920460AF06BFB08B1102070BD89
:108EF00022462946304608F0ECFB0028F7D0072030
:108F000070BD3EB504460AF03DFB08B110203EBDE1
:108F1000684605F097F8FFF783FB0028F7D19DF826
:108F200006002070BDF808006080BDF80A00A0802F
:108F300000203EBD70B505460C4608460AF040FBD1
:108F400020B95CB120680AF01DFB28B1102070BD6B
:108F50001C00002068030020A08828B12146284674
:108F6000BDE87040FDF746BE0920F0E770B5044645
:108F70000D4608460AF0E0FA30B9601E1E2814D8E3
:108F800028460AF0D9FA08B11020E0E7022C01D9EE
:108F90000720DCE704B9FFDFDC4800EB840050F871
:108FA000041C2846BDE870400847A4F120001F2893
:108FB000EED829462046BDE87040F9F7C8B870B52C
:108FC00004460D4608460AF0DDFA30B9601E1E2838
:108FD0000DD828460AF0B0FA08B11020B7E7012CE6
:108FE00001D0022C01D10620B1E70720AFE7A4F1A0
:108FF00020001F28F9D829462046BDE87040F9F71F
:1090000005B906F045B930B5C14D04466878A042AF
:1090100000D8FFDF686800EB041030BD70B5BC48B5
:1090200000252C46467807E02046FFF7ECFF407805
:10903000641C2844C5B2E4B2B442F5D1284686E7A0
:109040002DE9F0410C46064600F02FF9074630683E
:10905000C01C20F0030232601CBBAD483B46092116
:1090600020300AF043F9002408E0092C11D2DFE88F
:1090700004F005070509090B05050700A54804E0EC
:10908000A54802E0A54800E0A5480AF04FF90546CA
:1090900000E0FFDFA54200D0FFDF641CE4B2092C32
:1090A000E3D3306800EB07103060C6E5021D514382
:1090B000452900D245210844C01CB0FBF2F0C0B2E3
:1090C00070472DE9FC5F064691484FF000088B463B
:1090D0004746444690F8019022E02046FFF793FF70
:1090E000050000D1FFDF687869463844C7B22846DA
:1090F000FFF72EF8824601A92846FFF743F80346FA
:10910000BDF804005246001D81B2BDF80000001DEC
:1091100080B206F0BBFD6A78641C00FB0288E4B2F2
:109120004C45DAD13068C01C20F003003060BBF140
:10913000000F00D000204246394606F0B5FD3168E8
:1091400008443060BDE8FC9F71494431087100203B
:10915000C87070476E494431CA782AB10A7801EB69
:1091600042110831814201D0012070470020704730
:109170002DE9F04106460078154600F00F04002066
:109180001080601E0F46052800D3FFDF5F482A4687
:10919000103000EB8400394650F8043C3046BDE8FE
:1091A000F041184738B50446407800F00300012824
:1091B00003D002280BD0072038BD606858B10AF0F0
:1091C00008FAD0B960680AF0FBF920B915E06068C8
:1091D0000AF0B2F988B969462046FBF771F9002810
:1091E000EAD1607800F00300022808D19DF8000061
:1091F00028B160680AF0E4F908B1102038BD61892F
:10920000F8290DD8208988420AD8607800F0030236
:109210003F48012A06D1D731C26989B28A4201D2B8
:10922000092038BD94E80E0000F10C0585E80E0019
:109230000AB900218182002038BD2DE9F05F4FF08E
:1092400000093348C8464F464E464D46CB464C462D
:1092500090F801A011E02046FFF7D5FE4178827812
:1092600009F10109884412FB0177C27812FB0166FB
:10927000807B10FB0155641CE4B25445EBD10BEB31
:10928000890000EBC80000EB870000EB860000EBD4
:10929000C5011F48027A01EBC201427A807A01EBD4
:1092A000C20101EBC000BDE8F09F2DE9F047DFF8F7
:1092B00060900026344699F8080099F8092099F83A
:1092C00001700244D5B299F80A20104400F0FF085A
:1092D00008E02046FFF797FE817B407811FB00668F
:1092E000641CE4B2BC42F4D199F8080099F8091062
:1092F000401C284428444044401C01B1012108443A
:109300008419FF2C00D9FFDFE0B22BE478ED0100D7
:1093100068030020E11F000037A10000B1B9000080
:10932000D31301002DE9F04107461446884608464C
:1093300001F020FD064608EB88001C22796802EB4C
:10934000C0000D18688C58B14146384601F01AFD2E
:10935000014678680078C200082305F120000CE07F
:10936000E88CA8B14146384601F013FD0146786803
:1093700008234078C20005F1240006F0C6FA38B18F
:10938000062121726681D0E90010C4E9031009E0CA
:10939000287809280BD00520207266816868E06073
:1093A000002028702046BDE8F04101F0D9BC07201C
:1093B00020726681F4E72DE9F04116460D46074616
:1093C000406801EB85011C2202EBC10144182046D4
:1093D00001F001FD40B10021708865F30F2160F3B9
:1093E0001F4108200AF05CF8092020703246294607
:1093F0003846BDE8F04195E72DE9F0410E460746B5
:1094000000241C21F07816E004EB8403726801EB61
:10941000C303D25C6AB1FFF7CDFA050000D1FFDFCC
:109420006F802A4621463046FFF7C5FF0120BDE880
:10943000F081641CE4B2A042E6D80020F7E770B5E2
:10944000064600241C21C0780AE000BF04EB840318
:10945000726801EBC303D5182A782AB1641CE4B200
:10946000A042F3D8402070BD2821284615F0ACFA60
:10947000706880892881204670BD70B50346002041
:109480001C25DC780DE000BF00EB80065A6805EB78
:10949000C6063244167816B1128A8A4204D0401C9D
:1094A000C0B28442F0D8402070BDF0B50446002020
:1094B0001C26E5780EE000BF00EB8007636806EB32
:1094C000C7073B441F788F4202D15B78934204D098
:1094D000401CC0B28542EFD84020F0BD0078032880
:1094E00001D000207047012070470078022801D089
:1094F00000207047012070470078072801D0002025
:109500007047012070472DE9F041064688461078E3
:10951000F1781546884200D3FFDF2C781C27641CA5
:10952000F078E4B2A04201D8201AC4B204EB84015E
:10953000706807EBC1010844017821B141468847B2
:1095400008B12C7073E72878A042E8D14020287039
:109550006DE770B514460B880122A240134207D173
:1095600013430B8001230A22011D06F098F90470B1
:1095700070BD2DE9FF4F81B00878DDE90E7B9A467A
:1095800091460E4640072CD4019806F045FC040095
:1095900000D1FFDF07F1040820461FFA88F105F02B
:1095A00084FD050000D1FFDF204629466A4605F00C
:1095B000CEFF0098A0F80370A0F805A0284606F09A
:1095C00074F8017869F306016BF3C7110170204646
:1095D0001FFA88F105F0ACFD00B9FFDF019804F037
:1095E000AEFB06EB0900017F491C017705B0BDE821
:1095F000F08F2DE9F84F0E469A4691460746032113
:1096000006F0C6FA0446008DDFF8B485002518B1CF
:1096100098F80000B0421ED1384606F0FDFB070066
:1096200000D1FFDF09F10401384689B205F03DFDA4
:10963000050010D0384629466A4605F088FF009894
:1096400000210A460180817004F030FC0098C01DA2
:10965000CAF8000021E098F80000B04216D104F1E9
:10966000260734F8341F012000FA06F911EA090F21
:1096700000D0FFDF2088012340EA090020800A2271
:10968000391D384606F026F9067006E0324604F128
:10969000340104F12600FFF75CFF0A2188F800106E
:1096A0002846BDE8F88FFEB514460D46064602ABC7
:1096B0000C220621FFF79DFF002826D0029968782A
:1096C00012220A70801C487008224A80A8702088E4
:1096D00088806088C880A0880881E088488100244C
:1096E0000C20CDE900040523062229463046FFF769
:1096F00040FF214666F31F41F0230022012009F0BC
:1097000025FE6878801C68700120FEBDFEB51446F9
:109710000D460622064602AB1146FFF76AFF0028F7
:1097200012D0029B132000211870A87858700220D4
:1097300058809C800620CDE9000102460523294679
:109740003046FFF716FF0120FEBD2DE9FE430C4613
:10975000804644E002AB0E2207214046FFF749FF56
:10976000002841D060681C2267788678BF1C06EB11
:10977000860102EBC101451802981421017047705F
:109780000A214180698A0181E98A4181A988818011
:10979000A9898181304601F0EDFA0299052307225B
:1097A000C8806F700420287000250E20CDE90005C8
:1097B00021464046FFF7DDFE294666F30F2168F398
:1097C0001F41F0230022082009F0C0FD6078FD4908
:1097D000801C607062682046921CFFF794FE6068EF
:1097E00080784028B6D10120BDE8FE83FEB50D4645
:1097F000064638E002AB0E2207213046FFF7F9FE9D
:10980000002835D068681C23C17801EB810203EB86
:10981000C2028418029815220270627842700A22ED
:109820004280A2894281A2888281084601F0A2FA80
:10983000014602988180618AC180E18A0181A08805
:10984000B8B10020207000210E20CDE900010523D1
:10985000072229463046FFF78CFE6A68DA49284617
:10986000D21CFFF750FE6868C0784028C2D10120A2
:10987000FEBD0620E6E72DE9FE430C46814644E0A6
:10988000204601F092FAD0B302AB082207214846E5
:10989000FFF7AFFE0028A7D060681C226578067924
:1098A000AD1C06EB860102EBC10147180298B7F820
:1098B000108006210170457004214180304601F07E
:1098C00059FA0146029805230722C180A0F80480B6
:1098D0007D70082038700025CDE9000521464846F6
:1098E000FFF747FE294666F30F2169F31F41F02376
:1098F0000022082009F02AFD6078801C60706268F0
:10990000B2492046121DFFF7FEFD6068017940292B
:10991000B6D1012068E72DE9F34F83B00E4680E011
:10992000304601F042FA002875D071681C2091F889
:10993000068008EB880200EBC2000C184146304656
:1099400001F027FA0146A078C30070684078C20091
:1099500004F1240005F0F5FF07468088E18B401AEA
:1099600080B2002581B3AA46218B814200D80846E7
:109970008146024602AB07210398FFF73AFE010039
:1099800028D0BAF1000F03D0029AB88802251080BF
:109990008B46E28B3968A9EB05001FFA80FA0A446E
:1099A0000398009206F038FAED1D009A5946534686
:1099B000009505F046FEE08B504480B2E083B98804
:1099C000884209D1012508E0FFE7801C4FF0010A19
:1099D00080B2C9E7002009E60025CDE90095238A79
:1099E000072231460398FFF7C4FDE089401EE0815D
:1099F0008DB1A078401CA0707068F178427811FB9E
:109A000002F1CAB2816901230E3005F048FF80F8E7
:109A100000800020E08372686D493046921DFFF798
:109A200072FD7068817940297FF47AAF0120DDE50D
:109A300070B5064648680D4614468179402910D114
:109A400004EB84011C2202EBC101084401F0E4F99B
:109A5000002806D06868294684713046BDE8704009
:109A600059E770BDFEB50C460746002645E0204686
:109A700001F09BF9D8B360681C22417901EB8101A8
:109A800002EBC1014518688900B9FFDF02AB08226B
:109A900007213846FFF7ADFD002833D002996078E2
:109AA00016220A70801C4870042048806068407943
:109AB00001F060F901460298052307228180698937
:109AC000C1800820CDE9000621463846FFF751FD48
:109AD0006078801C6070A88969890844B0F5803F6F
:109AE00000D3FFDFA88969890844A8816E81626874
:109AF00038492046521DFFF706FD6068417940292C
:109B0000B5D10120FEBD30B5438C458BC3F3C704EE
:109B1000002345B1838B641EED1AC38A6D1E1D445C
:109B200095FBF3F3E4B22CB1008918B1A04200D840
:109B3000204603444FF6FF70834200D30346138050
:109B40000C7030BD2DE9FC41074616460D464868AD
:109B500002EB86011C2202EBC10144186A4601A9EE
:109B60002046FFF7D0FFA089618901448AB2BDF881
:109B70000010914212D0081A00D500206081686858
:109B8000407940280AD1204601F03CF9002805D050
:109B90006868294646713846FFF764FFBDE8FC81D6
:109BA0002DE9FE4F8946804615465088032105F071
:109BB000EFFF8346B8F8020040280DD240200CE0A9
:109BC00030000020DD940000EB940000F9940000C8
:109BD00019AE000005AE0000403880B28246014652
:109BE000584601F0E2F800287ED00AEB8A001C22D9
:109BF000DBF8041002EBC0000C18204601F0EBF873
:109C0000002877D1B8F80000E18A88423CD8A189C1
:109C1000D1B348456ED100265146584601F0B2F8FE
:109C2000218C0F18608B48B9B9F1020F62D3B8F8D4
:109C300004006083618A884226D80226A9EB0600C8
:109C40001FFA80F9B888A28B801A002814DD4946D3
:109C5000814500DA084683B26888696802913968EC
:109C60000A44CDE9003206F0C5F8DDE90121F61D10
:109C7000009B009605F0B1FCA18B01EB090080B2BE
:109C8000A083618B884207D9688803B05246594641
:109C9000BDE8F04F01F0DDB81FD14FF00900287288
:109CA000B8F802006881D7E90001C5E90401608BBA
:109CB000A881284601F054F85146584601F062F850
:109CC0000146DBF8040008230078C20004F12000FC
:109CD00005F01BFE0020A0836083A0890AF0FF022C
:109CE000401EA081688800E004E003B05946BDE84A
:109CF000F04F27E7BDE8FE8F2DE9F04106461546F7
:109D00000F461C46184609F017FC18B9206809F0E0
:109D100039FC08B1102015E47168688C0978B0EB43
:109D2000C10F01D313200DE43946304601F02AF863
:109D30000146706808230078C20005F1200005F094
:109D4000AEFDD4E90012C0E900120020E3E710B52F
:109D50000446032105F01CFF0146007800F00300D3
:109D6000022805D02046BDE8104001F114029AE413
:109D70008A8A2046BDE81040C8E470B50446032135
:109D800005F006FF054601462046FFF774FD002852
:109D900016D029462046FFF765FE002810D0294638
:109DA0002046FFF723FD00280AD029462046FFF76A
:109DB000CCFC002804D029462046BDE87040AAE526
:109DC00070BD2DE9F0410C4680461EE0E1784278F6
:109DD00011FB02F1CAB2816901230E3005F095FD35
:109DE000077860681C22C179491EC17107EB8701A1
:109DF000606802EBC10146183946204600F0D5FFE5
:109E000018B1304600F0E0FF20B16068C179002948
:109E1000DCD180E7FEF7CEFD050000D1FFDF0A2090
:109E20002872384600F0A6FF68813946204600F0C7
:109E3000B0FF0146606808234078C20006F12400A4
:109E400005F063FDD0E90010C5E90310A5F8028014
:109E5000284600F085FFB07800B9FFDFB078401EDB
:109E6000B07058E770B50C460546032105F090FE2A
:109E700001464068C2792244C2712846BDE870405C
:109E80009FE72DE9FE4F8246507814460F464FF06B
:109E9000000800284FD0012807D0022822D0FFDF79
:109EA0002068B8606068F86024E702AB0E220821E1
:109EB0005046FFF79EFB0028F2D00298152105239B
:109EC0000170217841700A214180C0F80480C0F8F7
:109ED0000880A0F80C80628882810E20CDE90008FD
:109EE000082221E0A678304600F044FF054606EB44
:109EF00086012C22786802EBC1010822465A02AB87
:109F000011465046FFF775FB0028C9D0029807217B
:109F10000170217841700421418008218580C6802C
:109F2000CDE9001805230A4639465046FFF721FBC4
:109F300087F80880DEE6A678022516B1022E13D037
:109F4000FFDF2A1D914602AB08215046FFF751FB67
:109F50000028A5D002980121022E017021784170BD
:109F60004580868002D005E00625EAE7A188C18009
:109F7000E1880181CDE90098052308223946504641
:109F8000D4E710B50446032105F002FE014600F1B6
:109F900008022046BDE8104073E72DE9F05F0C464B
:109FA00001281DD0957992F80480567905EB85013A
:109FB0001F2202EBC10121F0030B08EB060111FB8C
:109FC00005F14FF6FF7202EAC10909F1030115FB21
:109FD0000611F94F21F0031A40B101283DD124E0C8
:109FE0006168E57891F800804E78DFE75946786837
:109FF00005F009FC606000B9FFDF5946606814F0A5
:10A0000005FDE5705146786805F0FDFB6168486123
:10A0100000B9FFDF6068426902EB09018161606895
:10A0200080F800806068467017E0606852464169B9
:10A03000786805F013FC5A466168786805F00EFCF4
:10A04000032005F04DFD0446032005F051FD201AC4
:10A05000012802D1786805F0CBFB0BEB0A00BDE8C4
:10A06000F09F02460021022097E773B5D24D0A20E7
:10A070002870009848B100244FEA0D0005F0A5FBB8
:10A08000002C01D1009969607CBD01240020F5E716
:10A0900070B50C4615463821204614F0B7FC012651
:10A0A00066700A2104F11C0014F0B0FC05B9FFDF52
:10A0B000297A207861F301002070A879002817D050
:10A0C0002A4621460020FFF768FF6168402088701B
:10A0D0006168C870616808716168487161688871F9
:10A0E000616828880881616868884881606886811D
:10A0F00070BDC878002802D0002201204DE77047CB
:10A1000070B50546002165F31F41012009F0C8F92B
:10A110000321284605F03CFD040000D1FFDF214665
:10A120002846FFF769F9002804D0207840F0100095
:10A130002070012070BD2DE9FF4180460E460F0CB6
:10A14000FEF738FC050007D06F800321384605F084
:10A150001FFD040008D106E004B03846BDE8F04118
:10A160001321F8F711BCFFDFB8F1010F05D0B8F1EA
:10A17000080F18D0FFDFBDE8FF8120782A4620F0C5
:10A18000080020700020ADF8020002208DF80000C9
:10A190004FF6FF70ADF80400ADF80600694638468A
:10A1A000F7F781FFE7E7C6F3072101EB81021C23E4
:10A1B000606803EBC202805C042803D008280AD040
:10A1C000FFDFD8E7012000904FF440432A462046A5
:10A1D00000F008FECFE704B02A462046BDE8F04173
:10A1E000FFF7E9B82DE9F05F0027B0F80A90904634
:10A1F0000C4605463E46B9F1400F01D2402001E031
:10A20000A9F140001FFA80FA287AC01E08286BD2F4
:10A21000DFE800F00D04192058363C47722710265D
:10A22000002C6CD0D5E90301C4E902015CE0702781
:10A230001226002C63D00A2205F10C0104F108005B
:10A2400014F088FB50E071270C26002C57D0E868EA
:10A25000A06049E0742710269CB3D5E90301C4E946
:10A2600002016888032105F093FC8346FEF7A2FBF8
:10A2700002466888508051465846FFF753F833E04D
:10A2800075270A26ECB1A88920812DE076271426AF
:10A29000BCB105F10C0004F1080307C883E807000E
:10A2A00022E07727102664B1D5E90301C4E9020151
:10A2B0006888032105F06CFC01466888FFF781FD82
:10A2C00012E01CE073270826CCB16888032105F052
:10A2D0005FFC01460078C00606D56888FFF78CF859
:10A2E00010B96888F7F7E6FAA8F800602CB1278063
:10A2F000A4F8069066806888A0800020AFE6A8F8E1
:10A300000060FAE72DE9FC410C461E4617468046E0
:10A31000032105F03DFC05460A2C0AD2DFE804F0D3
:10A3200005050505050509090907042303E00623BA
:10A3300001E0FFDF0023CDE90076224629464046B2
:10A34000FFF717F92AE438B50546A0F57F40FF3836
:10A3500030D0284605F04EFD040000D1FFDF204636
:10A3600005F0D3F8002815D001466A46204605F0CE
:10A37000EEF800980321B0F80540284605F008FCE7
:10A380000546052C03D0402C05D2402404E0007A79
:10A3900080B1002038BD403CA4B2214600F005FD4C
:10A3A00040B1686804EB84013E2202EBC101405ACF
:10A3B0000028EFD0012038BD300000202DE9F04FFB
:10A3C000044689B0408805F015FD050000D1FFDF87
:10A3D00006AA2846616800F0C1FC069D001F81B2F4
:10A3E00035F8032F6B888A4205D1042B0AD0052B40
:10A3F0001DD0062B15D022462846FFF7D1FB09B009
:10A40000BDE8F08F16462D1D224629463046FBF743
:10A410001BFC0828F3D1224629463046FCF731FCC4
:10A42000EDE76088291D6368F9F7B8FCE7E7174690
:10A430006088032105F0ACFB4FF000088DF8048024
:10A440000646ADF80680042FD9D36A79002AD6D003
:10A4500028794FF6FF794FF01C0A13282CD008DC1E
:10A46000012878D0062847D0072875D0122874D143
:10A4700006E0142872D0152871D016286DD1ACE1F1
:10A480000C2F6AD1307800F00301022965D140F029
:10A49000080030706879B07001208DF804002889B8
:10A4A000ADF808006889ADF80A00A889ADF80C007D
:10A4B000E889ADF80E0019E0B07890429FD130786D
:10A4C00001079CD5062F9AD120F0080030706088D3
:10A4D000414660F31F41012008F0E2FF02208DF8A1
:10A4E0000400ADF808902889ADF80A00608822467B
:10A4F00001A9F7F7D8FD82E7082F80D12F89B5F899
:10A500000A90402F01D2402001E0A7F1400080B224
:10A5100080460146304600F048FC08B3716808EBFD
:10A5200088002C2202EBC000095A4945E3D1FE48BD
:10A5300007AAD0E90210CDE9071068798DF81C0050
:10A5400008F0FF058DF81E5060883146FFF799FC32
:10A550002246294639E0B6E014E03CE039E0E6E086
:10A56000F148D0E90010CDE907106879ADF8207006
:10A570008DF81C00ADF82290608807AA3146FFF7DD
:10A5800080FC3CE7082FB6D16889B5F808804028E0
:10A5900001D2402000E0403887B23946304600F012
:10A5A00004FC0028A7D007EB870271680AEBC20001
:10A5B0000844028A42459ED1017808299BD14078FF
:10A5C0006979884297D1F9B222463046FEF7F3FE08
:10A5D00015E70E2F07D0CDF81C80CDF820806879C4
:10A5E0008DF81C00C8E76989EF898B46B5F80C9097
:10A5F0003046FEF742FFABF14001402901D309206C
:10A600004AE0B9F1170F01D3172F01D20B2043E015
:10A6100040280ED000EB800271680AEBC2000844AB
:10A620000178012903D1407869798842A9D00A20AC
:10A6300032E03046FEF703FF014640282BD001EB05
:10A64000810372680AEBC30002EB0008012288F85C
:10A6500000206A7988F8012070682A894089B84208
:10A6600000D938462D8A03232372A282E7812082F3
:10A67000A4F80C906582084600F07CFB6081A8F885
:10A680001490A8F81870A8F80E50A8F810B020463A
:10A6900000F066FBB3E6042005212172A4F80A80CD
:10A6A000E08101212173A049D1E90421CDE90721ED
:10A6B00069798DF81C10ADF81E00608807AA314634
:10A6C000FFF7DFFBE3E7062FE4D3B078904215D124
:10A6D0003078010712D520F00800307060884146BC
:10A6E00060F31F41012008F0DBFE02208DF804001A
:10A6F0002889ADF80800ADF80A90F7E60421304645
:10A70000FEF7D3FE05464028C4D002208303009004
:10A7100022462946304600F065FB4146608865F3D5
:10A720000F2160F31F41082008F0BAFE67E60E2FE4
:10A73000B0D104213046FEF7B8FE81464028A9D0AA
:10A740004146608869F30F2160F31F41082008F03B
:10A75000A7FE288A0790E88900907068AF89408931
:10A76000B84200D938468346B5F80A802889059052
:10A77000484600F0FFFA6081079840B10220079B2D
:10A78000009022464946304600F02CFB37E6B8F1EF
:10A79000170F1ED3172F1CD304202072009860823D
:10A7A000E781A4F810B0A4F80C8009EB8902716865
:10A7B0000AEBC2000D1800990598A5F81480A5F8B9
:10A7C00018B0E9812882204600F0CAFA06202870D5
:10A7D00015E601200B230090D3E7082FA6D1298985
:10A7E0003046FEF74AFE074640289FD007EB870217
:10A7F00071680AEBC2000844804600F0ECFA0028B9
:10A8000094D16D89B8F80E002844B0F5803F05D387
:10A8100060883A46314600F01CFBF0E5002D85D0FB
:10A82000A8F80E0060883A463146FFF701F9082083
:10A830002072384600F09EFA6081A58127E770B546
:10A840000D460646032105F0A3F9040004D0207844
:10A85000000704D5112070BD43F2020070BD2A46E6
:10A8600021463046FEF71FFF18B928686061686806
:10A87000A061207840F008002070002070BD70B505
:10A880000D460646032105F083F9040004D0207824
:10A89000000704D4082070BD43F2020070BD2A46B0
:10A8A00021463046FEF732FF00B9A582207820F01D
:10A8B00008002070002070BD2DE9F04F0E4691B0C9
:10A8C0008046032105F064F90446404605F0A4FAE9
:10A8D00007460020079008900990ADF830000A90D4
:10A8E00002900390049004B9FFDF0DF1080917BB33
:10A8F000FFDF20E038460BA9002204F0C9FC9DF8D8
:10A900002C0000F07F050A2D00D3FFDF6019017FC6
:10A91000491E01779DF82C0000060CD52A460CA98B
:10A9200007A8FEF716FE01E0A0ED010019F80510DA
:10A93000491C09F80510761EF6B2DBD204F134008A
:10A94000FC4D04F1260BDFF8F0A304F12A07069072
:10A9500010E05846069900F06EFA064628700A285C
:10A9600000D3FFDF5AF8261040468847E08CC05DD0
:10A97000B04202D0208D0028EBD10A202870EE4D85
:10A980004E4628350EE00CA907A800F054FA0446FC
:10A99000375D55F8240000B9FFDF55F8242039460B
:10A9A00040469047BDF81E000028ECD111B027E5C5
:10A9B00010B5032105F0ECF8040000D1FFDF0A21F7
:10A9C00004F11C0014F022F8207840F004002070FC
:10A9D00010BD10B50C46032105F0DAF801190A7F05
:10A9E00001211AB9808EA140084000D0012010BD7D
:10A9F0002DE9F84F894615468246032105F0C8F82F
:10AA0000070004D0284608F097FD40B903E043F260
:10AA10000200BDE8F88F484608F0B4FD08B11020E8
:10AA2000F7E7786828B169880089814201D909204F
:10AA3000EFE7B9F800001C2418B1402809D24020E3
:10AA400008E03846FEF7FBFC8046402819D1132069
:10AA5000DFE7403880B280460146384600F0A5F96D
:10AA600048B108EB8800796804EBC000085C012855
:10AA700003D00820CDE70520CBE7FDF79BFF0600BC
:10AA80000BD008EB8800796804EBC0000C18B9F80B
:10AA9000000020B1E88910B113E01120B9E728883F
:10AAA000172802D36888172801D20720B1E7686801
:10AAB00038B12B1D224641463846FFF71DF90028C4
:10AAC000A7D104F10C0269462046FFF71CF828883C
:10AAD00060826888E082B9F8000030B102202070FE
:10AAE000E889A080E889A0B12BE003202070A88924
:10AAF000A08078688178402905D180F802803946A5
:10AB00005046FEF722FE404600F034F9A9F8000056
:10AB100021E07868218B4089884200D9084620834B
:10AB2000A6F802A004203072B9F800007081E08914
:10AB30007082F181208B3082A08AB081304600F093
:10AB40000FF97868C178402905D180F8038039462B
:10AB50005046FEF74BFE00205BE770B50D460646FB
:10AB6000032105F015F8040003D0402D04D2402540
:10AB700003E043F2020070BD403DADB2294600F053
:10AB800014F958B105EB85011C22606802EBC10184
:10AB9000084400F020F918B1082070BD052070BDF0
:10ABA0002A462146304600F054F9002070BD2DE9B8
:10ABB000F0410D4616468046032104F0E9FF0446A5
:10ABC000402D01D2402500E0403DADB28CB1294678
:10ABD00000F0EBF880B105EB85011C22606802EB08
:10ABE000C1014718384600F0F6F838B10820BDE832
:10ABF000F08143F20200FAE70520F8E733463A46CF
:10AC000029462046FFF778F80028F0D1EAB221461D
:10AC10004046FEF797FF0020E9E72DE9F0410D4699
:10AC200016468046032104F0B3FF0446402D01D2AE
:10AC3000402500E0403DAFB224B1304608F07CFC36
:10AC400038B902E043F20200D1E7306808F074FC42
:10AC500008B11020CBE73946204600F0A6F860B1D5
:10AC600007EB87011C22606802EBC10145182846EA
:10AC700000F0B1F818B10820B9E70520B7E7B088AF
:10AC8000A98A884201D90C20B1E76168E88C49782B
:10AC9000B0EBC10F01D31320A9E73946204600F0DD
:10ACA00078F80146606808234078C20005F1240066
:10ACB00004F0F5FDD6E90012C0E90012FAB221460F
:10ACC0004046FEF7B5FE002091E72DE9F0470D461E
:10ACD0001F4690468146032104F05AFF0446402D4A
:10ACE00001D2402001E0A5F1400086B23CB14DB157
:10ACF000384608F065FC50B11020BDE8F08743F2FB
:10AD00000200FAE76068C8B1A0F80C8024E0314680
:10AD1000204600F04AF888B106EB86011C226068E4
:10AD200002EBC1014518284600F055F840B1082053
:10AD3000E3E7000030000020B8ED01000520DCE76B
:10AD4000A5F80880F2B221464846FEF7FBFE1FB187
:10AD5000A8896989084438800020CEE704F0F7BB51
:10AD6000017821F00F01491C21F0F0011031017030
:10AD7000FDF723BE10B50446402800D9FFDF40345C
:10AD8000A0B210BD406842690078484302EBC000A1
:10AD90007047C2784068037812FB03F24378406939
:10ADA00001FB032100EBC1007047C2788A4209D938
:10ADB000406801EB81011C2202EBC101405C08B13B
:10ADC00001207047002070470078062801D9012033
:10ADD0007047002070470078062801D00120704796
:10ADE00000207047F0B401EB81061C27446807EB94
:10ADF000C6063444049D05262670E3802571F0BC08
:10AE0000FEF790BA10B5418911B1FFF7DDFF08B127
:10AE1000002010BD012010BD10B5C18C8278B1EBAF
:10AE2000C20F04D9C18911B1FFF7CEFF08B10020CC
:10AE300010BD012010BD10B50C4601230A22011DD2
:10AE400004F063FD00782188012282409143218033
:10AE500010BDF0B402EB82051C264C6806EBC5055C
:10AE6000072363554B681C79402C03D11A71F0BC41
:10AE7000FEF701BDF0BC704770B50B2000F0B5F9CE
:10AE8000082000F0B2F900210B2000F0C4F90021E5
:10AE9000082000F0C0F9EC4C01256560A560002099
:10AEA000C4F84001C4F84401C4F848010B2000F084
:10AEB000A7F9082000F0A4F90B2000F08BF9256019
:10AEC00070BD10B50B2000F090F9082000F08DF94E
:10AED000DD48012141608160DC490A68002AFCD11B
:10AEE0000021C0F84011C0F84411C0F848110B20EF
:10AEF00000F086F9BDE81040082000F081B910B5D7
:10AF00000B2000F07DF9BDE81040082000F078B972
:10AF100000B530B1012806D0022806D0FFDF00209E
:10AF200000BDCB4800BDCB4800BDCA48001D00BDD8
:10AF300070B5C9494FF000400860C84DC00BC5F856
:10AF40000803C74800240460C5F840410820C43500
:10AF500000F04BF9C5F83C41C248047070BD08B51B
:10AF6000B94A002128B1012811D002281CD0FFDFE6
:10AF700008BD4FF48030C2F80803C2F84803B34854
:10AF80003C300160C2F84011BDE80840D0E74FF402
:10AF90000030C2F80803C2F84803AC4840300160F2
:10AFA000C2F84411AB480CE04FF48020C2F808030B
:10AFB000C2F84803A54844300160C2F84811A548CA
:10AFC000001D0068009008BD70B516460D46044689
:10AFD000022800D9FFDF00229B48012304F1100161
:10AFE0008B4000EB8401C1F8405526B1C1F84021E7
:10AFF000C0F8043303E0C0F80833C1F84021C0F8BA
:10B00000443370BD2DE9F0411C46154630B101288E
:10B0100034D0022839D0FFDFBDE8F081891E00223C
:10B0200021F07F411046FFF7CFFF012C24D00020F4
:10B030008C4E8A4F012470703C61894900203C3954
:10B0400008600220091D0860854904203039086025
:10B0500083483D350560C7F80042082000F0D0F86D
:10B060002004C7F80403082000F0B4F87A49E00788
:10B07000091F08603470CFE70120D9E7012B02D007
:10B080000022012005E00122FBE7012B04D0002271
:10B090000220BDE8F04197E70122F9E76B4800681C
:10B0A000704770B500F0C7F8674C0546D4F840010A
:10B0B0000026012809D1D4F80803C00305D54FF4B0
:10B0C0008030C4F80803C4F84061D4F84401012872
:10B0D0000CD1D4F80803800308D54FF40030C4F82D
:10B0E0000803C4F84461012007F0B7FAD4F8480116
:10B0F00001280CD1D4F80803400308D54FF4802070
:10B10000C4F80803C4F84861022007F0A6FA5648BC
:10B11000056070BD70B500F08EF8524D0446287879
:10B1200058B1FFF705FF687820B1002085F80100CD
:10B1300007F093FA4C48046070BD0320F8E74FF025
:10B14000E0214FF40010C1F800027047152000F014
:10B1500057B8424901200861082000F051B83F4922
:10B160004FF47C10C1F808030020024601EB800375
:10B17000C3F84025C3F84021401CC0B20628F5D3CF
:10B180007047410A43F609525143C0F3080010FBCF
:10B1900002F000F5807001EB5020704710B5430BB2
:10B1A00048F2376463431B0C5C020C602F4C03FBBA
:10B1B00004002F4B4CF2F72443435B0D13FB04F4C4
:10B1C00004EB402000F580704012107008681844AD
:10B1D000086010BD00F01F0201219140400980006D
:10B1E00000F1E020C0F80011704700F01F020121BB
:10B1F00091404009800000F1E020C0F880117047C4
:10B2000000F01F02012191404009800000F1E02080
:10B21000C0F8801270474907090E002806DA00F0CE
:10B220000F0000F1E02080F8141D704700F1E020CD
:10B2300080F8001470470C48001F00680A4A0D4946
:10B24000121D11607047000000B0004004B50040BE
:10B250004081004044B1004008F5014000800040BA
:10B26000408500403800002014050240F7C2FFFF6F
:10B270006F0C01000100000110B5EFF3108000F029
:10B28000010472B6E9484178491C417040780128B0
:10B2900001D107F087FD002C00D162B610BD70B55A
:10B2A000E24CE07848B90125E570FFF7E5FF07F0CB
:10B2B00081FD20B1002007F05CFD002070BD4FF043
:10B2C00080406571C0F80453F7E770B5EFF3108064
:10B2D00000F0010572B6D54C607800B9FFDF6078E8
:10B2E000401E6070607808B907F060FD002D00D145
:10B2F00062B670BDCD4810B5C17821B10021417151
:10B30000C170FFF7E2FF002010BD10B5044607F042
:10B3100051FDC649C978084000D0012020600020B6
:10B3200010BD2DE9F05FDFF804934278817889F849
:10B330000620002689F80710074689F8086000787B
:10B34000354620B101280FD002280FD0FFDF07F0CB
:10B350003EFD98B107F042FDB0420FD1304607F0F4
:10B3600041FD0028FAD047E00126F0E7FFF784FF0F
:10B3700007F020FD0028FBD00226E8E70120840723
:10B38000E060C4F80451AA490E600107D1F84412E4
:10B39000A74AC1F3423124321160A5493431086013
:10B3A0004FF0020BC4F804B3A060DFF888A2DAF80B
:10B3B0000010C94341F3001101F10108DAF800104F
:10B3C00041F01001CAF8001000E020BFD4F80401D9
:10B3D0000028FAD0304607F005FD0028FAD0B8F171
:10B3E000000F05D1DAF8001021F01001CAF80010A2
:10B3F000C4F808B3C4F8045199F807004C4670B17A
:10B40000387860B907F0D6FC074607F037FE6FF0D2
:10B41000004117B1C4E9031001E0C4E9030116B10A
:10B420002571BDE8F09F0127BE0727714FF019086D
:10B43000C6F80883B761C6F80051C6F80C51C6F8C3
:10B44000105107F0B7FC10B1A770376100E027700A
:10B45000FFF712FF7649A07920310860C6F804830F
:10B46000DFE770B5050000D1FFDF4FF080424FF0FD
:10B47000FF30C2F808030021C2F80011C2F804111D
:10B48000C2F80C11C2F81011684C617007F098FCFA
:10B4900010B10120E07060702846BDE8704040E7C0
:10B4A0002DE9F05F6448D0F800B0634A6349083280
:10B4B00011608406D4F8080110B14FF0010801E0D2
:10B4C0004FF00008D4F8000100B101208146D4F803
:10B4D000040108B1012600E00026D4F80C0100B1F7
:10B4E00001208246D4F8100108B1012700E00027AE
:10B4F00048EA090126EA010020EA0A00B84300D020
:10B50000FFDF0025B8F1000F04D0C4F80851012076
:10B5100007F02FFC5FEA0900DFF810814FF0010906
:10B5200013D0C4F8005198F8050020B188F80550F0
:10B53000002007F01EFC98F8000030B107F03AFC3C
:10B5400018B188F80290C4F810900EB1C4F80451F4
:10B55000BAF1000F0CD0C4F80C5198F8020046461E
:10B5600000B9FFDFB5703570C4F81490FFF7ADFE79
:10B5700037B1C4F8105198F8040008B100F020F871
:10B580002D49091DC1F800B04BE770B5274DE8788B
:10B5900008B907F00BFC01208407A061A87850B11E
:10B5A000D4F80C0120B9002007F01CFC0028F7D1CA
:10B5B0000020C4F80C014FF0FF30C4F8080370BD40
:10B5C0002DE9F041194C4FF080470125E079F0B1A9
:10B5D000012803D0217A401E814218DA07F0EAFBE5
:10B5E000064607F04BFDE179012902D9217A491C71
:10B5F00021720EB1216900E0E168411A022902DAE4
:10B6000011F1020F0BDC0EB1206100E0E060FFF7EA
:10B6100033FE07F0CFFB28B13D61A57003E07D61EB
:10B62000BDE8F081257000202072F9E73C00002081
:10B630001805004010ED00E0100502400100000177
:10B6400010B50D2000F06FF8C4B26FF0040000F0E8
:10B650006AF8C0B2844200D0FFDF3A490120086096
:10B6600010BD70B50D2000F048F8374C0020C4F82C
:10B6700000010125C4F804530D2000F049F82560AD
:10B680004FF0E0216014C1F8000170BD10B50D202D
:10B6900000F033F82C48012141600021C0F800116E
:10B6A000BDE810400D2000F033B8284810B50468FC
:10B6B00026492748083108602349D1F800010128AC
:10B6C00004D0FFDF2148001D046010BD1D48001D8F
:10B6D00000680022C0B2C1F8002107F027FCF1E7A2
:10B6E00010B51948D0F800110029FBD0FFF7DDFF95
:10B6F000BDE810400D2000F00BB800F01F02012142
:10B7000091404009800000F1E020C0F880117047AE
:10B7100000F01F02012191404009800000F1E0206B
:10B72000C0F880127047002806DA00F00F0000F120
:10B73000E02090F8140D03E000F1E02090F8000400
:10B740004009704704D5004000D000401005024079
:10B750000100000110B5202000F082F8202000F048
:10B760008AF84A49202081F8000449490006086007
:10B77000091D48480860F5F7CFFD4549C831086004
:10B780004548D0F8041341F00101C0F80413D0F883
:10B79000041341F08071C0F804133C4901201C39A6
:10B7A000C1F8000110BD10B5202000F059F838484C
:10B7B00000210160001D0160354A481EE83A106012
:10B7C000354AC2F80803324BC8331960C2F8000189
:10B7D000C2F8600131490860BDE81040202000F047
:10B7E0004AB82B492E48EC390860704728492C4844
:10B7F000E8390860704726480160001D521E02604B
:10B80000704723490120E8390860BFF34F8F704724
:10B8100070B51F4A8069E83A214911601E49D1F884
:10B82000006100231F4D1D4A5C1E1EB1A84206D3B5
:10B8300000210FE0D1F8606186B1A84209D2C1F8B9
:10B840000031C1F860311460BDE87040202000F084
:10B8500012B81168BDE8704013F004B9FFDF70BD85
:10B8600000F01F02012191404009800000F1E0201A
:10B87000C0F88011704700F01F020121914040097B
:10B88000800000F1E020C0F88012704720E000E066
:10B890000006024024120020000002400004024082
:10B8A00001000001003002004FF0E0214FF0007075
:10B8B000C1F88001C1F88002384B802283F800244F
:10B8C000C1F80001704700B502460420344903E086
:10B8D00001EBC0031B792BB1401EC0B2F8D2FFDFD1
:10B8E000FF2000BD41F8302001EBC00100224A7169
:10B8F0008A7101220A7100BD294A002102EBC000B1
:10B900000171704710B50446042800D3FFDF2448B6
:10B9100000EBC4042079012800D0FFDF6079A17911
:10B92000401CC0B2814200D060714FF0E0214FF066
:10B930000070C1F8000210BD2DE9F04119480568FA
:10B9400018491948083108601448042690F8000482
:10B95000134F4009154C042818D0FFDF16E021785A
:10B9600007EBC1000279012A08D1427983799A4212
:10B9700004D04279827157F8310080472078401C0A
:10B98000C0B22070042801D300202070761EF6B2C9
:10B99000E5D20448001D0560BDE8F08119E000E033
:10B9A0009805002010050240010000015000002011
:10B9B00070B50C46054600F043FB21462846BDE81D
:10B9C000704001F026BC0000F8B51D46DDE90647D1
:10B9D0000E000AD004F020FA2346FF1DBCB2314607
:10B9E0002A46009403F02DFEF8BDD01922461946D0
:10B9F00012F06BFF2046F8BD70B50D4604461021CD
:10BA000012F0E2FF258117206081A07B40F00A0040
:10BA1000A07370BD4FF6FF720A800146032007F045
:10BA20003FBD704700897047827BD30701D19207E1
:10BA300003D4808908800020704705207047827BEE
:10BA4000920700D58181704701460020098841F6A0
:10BA5000FE52114200D00120704700B50346807BA2
:10BA6000C00701D0052000BD59811846FFF7ECFF43
:10BA7000C00703D0987B40F004009873987B40F097
:10BA800001009873002000BD827B520700D509B1E8
:10BA90004089704717207047827B61F3C30282732D
:10BAA00070472DE9FC5F0E4604460178964601205A
:10BAB00000FA01F14DF6FF5201EA020962684FF601
:10BAC000FF7B1188594506D0B9F1000F06D041F629
:10BAD000FE55294202D00120BDE8FC9F41EA090140
:10BAE00011801D0014D04FF0000C85F800C02378A1
:10BAF0000521032267464FF0020A0E2B74D2DFE8BD
:10BB000003F0F809252F47626974479092B3D0D7A4
:10BB10000420E1E7616820898B7B9B077DD517288E
:10BB200048D30B89834245D38989172901D38142A0
:10BB300040D185F800A0A5F80100328061688881B5
:10BB40006068817B21F002018173C5E004202870C8
:10BB50002089A5F801006089A5F803003180BBE0C9
:10BB6000208A3188C01D1FFA80F8414522D3062063
:10BB700028702089A5F801006089A5F80300A08934
:10BB8000A5F805000721208ACDE9000163693EE0A0
:10BB9000082B10D0082028702089A5F801006089A2
:10BBA000A5F8030031806A1D694604F10C0005F018
:10BBB00090FD10B15FE01020EDE730889DF8001097
:10BBC0000844308088E00A2028702089A5F8010008
:10BBD000328045E00C2028702089A5F8010060899A
:10BBE000A5F8030031803BE083E02189338800EB36
:10BBF00041021FFA82F843453DD3B8F1050F3AD30D
:10BC00000E222A700BEA4101CDE90010E36860883A
:10BC10002A467146FFF7D8FE00E04DE0A6F8008006
:10BC20005AE04020287060893188C01C1FFA80F8D3
:10BC3000414520D32878714620F03F00123028700B
:10BC40002089A5F801006089CDE9000260882A46B4
:10BC5000E368FFF7B9FEA6F80080287840063BD4D9
:10BC600061682089888037E0A0893288401D1FFAEA
:10BC700080F8424501D204273EE016202870208932
:10BC8000A5F801006089A5F80300A089CDE90001AD
:10BC900060882A4671462369FFF796FEA6F8008061
:10BCA000DEE718202870207A6870A6F800A013E05C
:10BCB00061680A88920401D405271DE0C988228999
:10BCC000914201D0062717E01E212970308060685C
:10BCD000018821F400510180B9F1000F0CD0618876
:10BCE00078230022032007F031FB616820788870F8
:10BCF00007E0A6F800C003276068018821EA09016F
:10BD000001803846E8E62DE9FF4F85B01746129CC2
:10BD10000D001E461CD03078C10703D000F03F0054
:10BD2000192801D9012100E000212046FFF7ACFECF
:10BD3000A8420DD32088A0F57F41FF3908D0307884
:10BD4000410601D4000605D5082009B0BDE8F08FF2
:10BD50000720FAE700208DF800008DF80100307808
:10BD60006B1E00F03F0C0121A81E4FF0050A4FF09A
:10BD700002094FF0030B9AB2BCF1200F75D2DFE835
:10BD80000CF08B10745E7468748C749C74B674BB05
:10BD900074C974D574E2747474F274F074EF74EE50
:10BDA000748B052D78D18DF80090A0788DF8040063
:10BDB0007088ADF8060030798DF80100707800F0D9
:10BDC0003F000C2829D00ADCA0F10200092863D228
:10BDD000DFE800F0126215621A621D62200012286C
:10BDE00024D004DC0E281BD01028DBD11BE0162841
:10BDF0001FD01828D6D11FE02078800701E02078D6
:10BE00004007002848DAEFE020780007F9E72078BB
:10BE1000C006F6E720788006F3E720784006F0E7D2
:10BE200020780006EDE72088C005EAE72088400575
:10BE3000E7E720880005E4E72088C004E1E72078F0
:10BE4000800729D5032D27D18DF800B0B6F8010061
:10BE500082E0217849071FD5062D1DD381B2707865
:10BE6000012803D0022817D102E0CAE0022000E036
:10BE7000102004228DF8002072788DF80420801C98
:10BE8000B1FBF0F2ADF8062092B242438A4203D1F0
:10BE90000397ADF80890A7E07AE02078000777D5FF
:10BEA00098B282088DF800A0ADF80420B0EB820FA4
:10BEB0006ED10297ADF8061096E02178C90667D5D5
:10BEC000022D65D381B206208DF80000707802281B
:10BED0005ED300BFB1FBF0F28DF80400ADF8062090
:10BEE00092B242438A4253D1ADF808907BE0207869
:10BEF00080064DD5072003E0207840067FD5082036
:10BF00008DF80000A088ADF80400ADF80620ADF86B
:10BF1000081068E02078000671D50920ADF80420EB
:10BF20008DF80000ADF8061002975DE02188C90584
:10BF300065D5022D63D381B20A208DF80000707898
:10BF400004285CD3C6E72088400558D5012D56D17A
:10BF50000B208DF80000A088ADF8040044E021E03B
:10BF600026E016E0FFE72088000548D5052D46D3DA
:10BF70000C208DF80000A088ADF80400B6F803008E
:10BF80006D1FADF80850ADF80600ADF80AA02AE024
:10BF900035E02088C00432D5012D30D10D208DF838
:10BFA000000021E02088800429D4B6F80100E08058
:10BFB000A07B000723D5032D21D3307800F03F006C
:10BFC0001B2818D00F208DF80000208840F4005066
:10BFD000A4F80000B6F80100ADF80400ED1EADF8BD
:10BFE0000650ADF808B0039769460598F9F773FB5A
:10BFF000050008D016E00E208DF80000EAE70725BE
:10C0000010E008250EE0307800F03F001B2809D032
:10C010001D2807D00320059907F042FA208800F474
:10C0200000502080A07B400708D52046FFF70CFD7C
:10C03000C00703D1A07B20F00400A073284684E64B
:10C040001FB5032806D101208DF8000088B269468B
:10C05000F9F741FB1FBD0000F8B51D46DDE90647B5
:10C060000E000AD003F0D8FE2346FF1DBCB23146B5
:10C070002A46009403F0E5FAF8BDD0192246194685
:10C0800012F023FC2046F8BD2DE9FF4F8DB09B46F2
:10C09000DDE91B57DDF87CA00C46082B05D0E069D4
:10C0A00001F000F950B11020D2E02888092140F0B9
:10C0B000100028808AF80010022617E0E1690120AC
:10C0C0008871E2694FF420519180E1698872E069DA
:10C0D00042F601010181E069002181732888112164
:10C0E00040F0200028808AF80010042638780A9052
:10C0F0000A2038704FF0020904F118004D460C90E8
:10C1000001F093FBB04681E0BBF1100F0ED1022D80
:10C110000CD0A9EB0800801C80B20221CDE90010F0
:10C1200005AB52461E990D98FFF796FFBDF8161005
:10C130001A98814203D9F74800790F9004E003D19F
:10C140000A9808B138702FE04FF00201CDE90019CC
:10C150000DF1160352461E990D98FFF77DFF1D98AD
:10C160000088401B801B83B2C6F1FF00984200D2BA
:10C1700003461E990BA8D9B15FF00002DDF878C024
:10C18000CDE9032009EB060189B2CDE901C10F9881
:10C190000090BDF8161000220D9801F0C9FB387010
:10C1A00070B1C0B2832807D0BDF8160020833AE0F2
:10C1B0000AEB09018A19E1E7022011B0BDE8F08F0E
:10C1C000BDF82C00811901F0FF08022D0DD09AF85E
:10C1D0000120424506D1BDF82010814207D0B8F1B8
:10C1E000FF0F04D09AF801801FE08AF80180C94847
:10C1F00000680178052902D1BDF81610818009EB8D
:10C2000008001FFA80F905EB080085B2DDE90C1083
:10C2100005AB0F9A01F00CFB28B91D980088411B53
:10C220004145BFF671AF022D13D0BBF1100F0CD1F9
:10C23000A9EB0800801C81B20220CDE9000105AB0A
:10C2400052461E990D98FFF707FF1D9805800020A4
:10C2500038700020B1E72DE9F8439C46089E13464C
:10C260000027B26B9AB3491F8CB2F18FA1F57F45BD
:10C27000FF3D05D05518AD882944891D8DB200E0D9
:10C2800000252919B6F83C800831414520D82A44B8
:10C29000BCF8011022F8021BBCF8031022F8021BA4
:10C2A000984622F8024B914603F0A4FD4FF00C0C87
:10C2B00041464A462346CDF800C003F08EF9F58783
:10C2C000B16B00202944A41D2144088003E001E053
:10C2D000092700E083273846BDE8F88310B50B88AE
:10C2E000848F9C420CD9846BE018048844B1848804
:10C2F00024F40044A41D23440B801060002010BDD2
:10C300000A2010BD2DE9F0478AB0002590468946E5
:10C310008246ADF8185007274BE0059806888088BC
:10C32000000446D4A8F8006007A80195009702957C
:10C33000CDE903504FF4007300223146504601F01E
:10C34000F7FA04003CD1BDF81800ADF820000598BC
:10C3500004888188B44216D10A0414D40195029548
:10C36000039521F400410097049541F480434288ED
:10C370002146504601F0B2F804000BD1059881889F
:10C3800041F40041818005AA08A94846FFF7A6FFAD
:10C390000400DCD00097059802950195039504955B
:10C3A0000188BDF81C300022504601F097F80A2C95
:10C3B00006D105AA06A94846FFF790FF0400ACD0B5
:10C3C000ADF8185004E00598818821F4004181807F
:10C3D00005AA06A94846FFF781FF0028F3D00A2CDA
:10C3E00003D020460AB0BDE8F0870020FAE710B578
:10C3F0000C46896B86B051B10C218DF80010A18FCD
:10C40000ADF80810A16B01916946FAF715F9002003
:10C410004FF6FF71A063E187A08706B010BD2DE93C
:10C42000F0410D460746896B0020069E1446002900
:10C4300011D0012B0FD1324629463846FFF762FF53
:10C44000002808D1002C06D0324629463846BDE8DF
:10C45000F04100F036BFBDE8F0812DE9FC41144603
:10C46000DDE9087C0E46DDE90A15521DBCF800E046
:10C4700092B2964502D20720BDE8FC81ACF80020BC
:10C4800017222A70A5F80160A5F803300522CDE92E
:10C4900000423B462A46FFF7DFFD0020ECE770B57F
:10C4A0000C4615464821204612F0B0FA04F1080067
:10C4B00044F81C0F00204FF6FF71E0616184208476
:10C4C000A5841720E08494F82A0040F00A0084F83C
:10C4D0002A0070BD4FF6FF720A800146042006F064
:10C4E000DFBF30B585B00C460546FFF780FFA18E53
:10C4F000284629B101218DF800106946FAF79CF809
:10C500000020E0622063606305B030BDB0F84000F9
:10C51000704700005400002090F84620920703D492
:10C52000408808800020F3E70620F1E790F84620D5
:10C530009207EDD5A0F84410EAE7014600200988EB
:10C540000A0700D5012011F0F00F01D040F00200E1
:10C55000CA0501D540F004008A0501D540F0080065
:10C560004A0501D540F010000905D1D540F0200062
:10C57000CEE700B5034690F84600C00701D006207C
:10C5800000BDA3F842101846FFF7D7FF10F03E0F8A
:10C5900005D093F8460040F0040083F8460013F8F5
:10C5A000460F40F001001870002000BD90F84620B2
:10C5B000520700D511B1B0F84200A9E71720A7E74C
:10C5C00010F8462F61F3C3020270A1E72DE9FF4F77
:10C5D0009BB00E00DDE92B34DDE92978289D24D0BD
:10C5E0002878C10703D000F03F00192801D90121A4
:10C5F00000E000212046FFF7D9FFB04215D328788C
:10C60000410600F03F010CD41E290CD0218811F402
:10C610007F6F0AD13A8842B1A1F57F42FF3A04D038
:10C6200001E0122901D1000602D504201FB0C5E5A2
:10C63000F9491D984FF0000A08718DF818A08DF87F
:10C640003CA00FAA0A60ADF81CA0ADF850A0297854
:10C65000994601F03F02701F5B1C04F1180C4FF06B
:10C66000060E4FF0040BCDF858C01F2A7ED2DFE82B
:10C6700002F07D7D107D267DAC7DF47DF37DF27D25
:10C68000F17DF47DF07D7D7DEF7DEE7D7D7D7D7D99
:10C69000ED0094F84610B5F80100890701D5032E86
:10C6A00002D08DF818B022E34FF40061ADF85010BD
:10C6B000608003218DF83C10ADF84000D8E2052ED3
:10C6C000EFD1B5F801002083ADF81C00B5F80310D8
:10C6D000618308B1884201D901207FE10020A07266
:10C6E00020814FF6FF702084169801F09EF80520F7
:10C6F00089F800000220029083460AAB1D9A169921
:10C700001B9801F095F890BB9DF82E00012804D0ED
:10C71000022089F80100102003E0012089F80100BF
:10C7200002200590002203A90BA804F0D2FFE8BB69
:10C730009DF80C00059981423DD13A88801CA2EBFE
:10C740000B01814237DB02990220CDE900010DF196
:10C750002A034A4641461B98FFF77EFC02980BF1DC
:10C76000020B801C80B217AA03A901E0A0E228E016
:10C7700002900BA804F0ADFF02999DF80C00CDE9E2
:10C78000000117AB4A4641461B98FFF765FC9DF830
:10C790000C100AAB0BEB01001FFA80FB02981D9AEC
:10C7A000084480B2029016991B9800E003E001F063
:10C7B0003FF80028B6D0BBF1020F02D0A7F800B0B6
:10C7C00053E20A208DF818004FE200210391072E52
:10C7D000FFF467AFB5F801002083ADF81C00B5F891
:10C7E0000320628300283FF477AF90423FF674AF96
:10C7F0000120A072B5F8050020810020A073E06937
:10C8000000F050FD78B9E16901208871E2694FF4C8
:10C8100020519180E1698872E06942F6010101814D
:10C82000E06900218173F01F20841E986062072058
:10C830006084169800F0F9FF072089F800000120B5
:10C84000049002900020ADF82A0028E01DE2A3E148
:10C850003AE1EAE016E2AEE086E049E0029801281B
:10C8600014D0E0698079012803D1BDF82800ADF823
:10C870000E00049803ABCDE900B04A4641461B9830
:10C88000FFF7EAFB0498001D80B20490BDF82A006F
:10C89000ADF80C00ADF80E00059880B202900AAB1E
:10C8A0001D9A16991B9800F0C3FF28B90298398881
:10C8B000001D05908142D1D20298012881D0E06903
:10C8C0008079012805D0BDF82810A1F57F40FF38F8
:10C8D00003D1BDF82800ADF80E00049803ABCDE9F4
:10C8E00000B04A4641461B98FFF7B6FB0298BBE1F1
:10C8F000072E02D0152E7FF4D4AEB5F80110218397
:10C90000ADF81C10B5F80320628300293FF4E4AEB3
:10C9100091423FF6E1AE0121A1724FF0000BA4F865
:10C9200008B084F80EB0052E07D0C0B2691DE269C8
:10C9300004F0B0FE00287FF444AF4FF6FF7020846F
:10C9400001A906AA14A8CDF800B081E885032878CB
:10C95000214600F03F031D9A1B98FFF795FB824686
:10C96000208BADF81C0080E10120032EC3D14021B3
:10C97000ADF85010B5F801102183ADF81C100AAACB
:10C98000B8F1000F00D00023CDE9020304921D98F6
:10C99000CDF80480009038880022401E83B21B9896
:10C9A00000F0C6FF8DF8180090BB0B2089F800003E
:10C9B000BDF8280037E04FF0010C052E9BD18020F8
:10C9C000ADF85000B5F801102183B5F803002084BC
:10C9D000ADF81C10B0F5007F03D907208DF81800C2
:10C9E00085E140F47C4222840CA8B8F1000F00D00D
:10C9F0000023CDE90330CDE9018C1D9800903888E3
:10CA0000401E83B21B9800F093FF8DF8180028B1E8
:10CA10008328A8D10220BDE0540000200D2189F810
:10CA20000010BDF83000401C1EE1032E04D2480661
:10CA30007FF537AE002017E1B5F80110ADF81C10F6
:10CA40002878400602D58DF83CE002E007208DF8FA
:10CA50003C004FF000080320CDE902081E9BCDF8F2
:10CA600010801D980193A6F1030B00901FFA8BF321
:10CA700042461B9800F032FD8DF818008DF83C807E
:10CA8000297849060DD52088C00506D5208BBDF82C
:10CA90001C10884201D1C4F8248040468DF81880CB
:10CAA000E2E0832801D14FF0020A4FF48070ADF824
:10CAB0005000BDF81C002083A4F820B01E986062CE
:10CAC000032060841321CCE0052EFFF4EAADB5F815
:10CAD0000110ADF81C10A28F62B3A2F57F43FE3B9C
:10CAE00028D008228DF83C204FF0000B0523CDE91B
:10CAF000023BDDF878C0CDF810B01D9A80B2CDF8B9
:10CB000004C040F400430092B5F803201B9800F0E5
:10CB1000E5FC8DF83CB04FF400718DF81800ADF8CD
:10CB20005010832810D0F8B1A18FA1F57F40FE38B6
:10CB300007D0DCE00B228DF83C204FF6FE72A28776
:10CB4000D2E7A4F83CB0D2E000942B4631461E9ABE
:10CB50001B98FFF780FB8DF8180008B183284BD194
:10CB6000BDF81C00208355E700942B4631461E9AE1
:10CB70001B98FFF770FB8DF81800E8BBE18FA06BE6
:10CB80000844811D8DE882034388828801881B98B0
:10CB9000FFF763FC824668E095F80180022E70D1B1
:10CBA0005FEA080002D0B8F1010F6AD109208DF8C0
:10CBB0003C0007A800908DF84080434600222146A3
:10CBC0001B98FFF72CFC8DF842004FF0000B8DF8FE
:10CBD00043B050B9B8F1010F12D0B8F1000F04D131
:10CBE000A18FA1F57F40FF380AD0A08F40B18DF80A
:10CBF0003CB04FF4806000E037E0ADF850000DE04D
:10CC00000FA91B98F9F718FD82468DF83CB04FF438
:10CC10008060ADF85000BAF1020F06D0FB48006802
:10CC2000C07928B18DF8180027E0A4F8188044E0F6
:10CC3000BAF1000F03D081208DF818003DE007A85D
:10CC400000904346012221461B98FFF7E8FB8DF830
:10CC5000180021461B98FFF7CAFB9DF8180020B961
:10CC6000192189F80010012038809DF83C0020B17E
:10CC70000FA91B98F9F7E0FC8246BAF1000F33D0F8
:10CC80001BE018E08DF818E031E02078000712D59D
:10CC9000012E10D10A208DF83C00E088ADF840004C
:10CCA00004201B9906F0FCFB0820ADF85000C1E6FB
:10CCB00048067FF5F6AC4FF0040A2088BDF8501006
:10CCC00008432080BDF8500080050BD5A18FA1F549
:10CCD0007F40FE3806D11E98E06228982063A68621
:10CCE0004FF0030A5046A1E49DF8180078B10120E6
:10CCF00089F80000297889F80110BDF81C10A9F8FE
:10CD000002109DF8181089F804100520388020883A
:10CD1000BDF8501088432080E4E72DE9FF4F884696
:10CD2000087895B0012181404FF20900249C014010
:10CD3000ADF820102088DDF88890A0F57F424FF0F4
:10CD4000000AFF3A02D029B1000703D5012019B02B
:10CD5000BDE8F08F239E4FF0000B0EA886F800B0C0
:10CD600018995D460988ADF83410A8498DF81CB0B3
:10CD7000179A0A718DF838B0086098F800000128F9
:10CD80003BD0022809D003286FD1307820F03F0033
:10CD90001D303070B8F80400E08098F800100320CF
:10CDA000022904D1317821F03F011B31317094F810
:10CDB0004610090759D505ABB9F1000F13D0002172
:10CDC00002AA82E80B000720CDE90009BDF8340073
:10CDD000B8F80410C01E83B20022159800F0A8FD18
:10CDE0000028D1D101E0F11CEAE7B8F80400A6F868
:10CDF0000100BDF81400C01C04E198F805108DF87E
:10CE00001C1098F80400012806D04FF4007A02287C
:10CE10002CD00328B8D16CE12188B8F8080011F4AF
:10CE20000061ADF8201020D017281CD3B4F84010B2
:10CE3000814218D3B4F84410172901D3814212D18A
:10CE4000317821F03F01C91C3170A6F8010003219F
:10CE5000ADF83410A4F8440094F8460020F0020025
:10CE600084F8460065E105257EE177E1208808F138
:10CE7000080700F4FE60ADF8200010F0F00F1BD0A2
:10CE800010F0C00F03D03888228B9042EBD199B9B3
:10CE9000B878C00710D0B9680720CDE902B1CDF845
:10CEA00004B00090CDF810B0FB88BA883988159886
:10CEB00000F014FB0028D6D12398BDF82010401CA8
:10CEC00080294ED006DC10290DD020290BD0402916
:10CED00087D124E0B1F5807F6ED051457ED0B1F589
:10CEE000806F97D1DEE0C80601D5082000E0102051
:10CEF00082460DA907AA0520CDE902218DF8380048
:10CF0000ADF83CB0CDE9049608A93888CDE9000118
:10CF10005346072221461598FFF7B6F8A8E09DF87A
:10CF20001C2001214FF00A0A002A9BD105ABB9F160
:10CF3000000F00D00020CDE902100720CDE9000944
:10CF4000BDF834000493401E83B2218B0022159853
:10CF500000F0EEFC8DF81C000B203070BDF81400C2
:10CF600020E09DF81C2001214FF00C0A002A22D15C
:10CF700013ABB9F1000F00D00020CDE9021007205B
:10CF8000CDE900090493BDF83400228C401E83B221
:10CF9000218B159800F0CCFC8DF81C000D20307012
:10CFA000BDF84C00401CADF8340005208DF8380069
:10CFB000208BADF83C00BCE03888218B88427FF4A0
:10CFC00052AF9DF81C004FF0120A00281CD1606A75
:10CFD000A8B1B878C0073FF446AF00E018E0BA68DF
:10CFE0000720CDE902B2CDF804B00090CDF810B022
:10CFF000FB88BA88159800F071FA8DF81C00132090
:10D0000030700120ADF8340093E00000540000209F
:10D010003988208B8142D2D19DF81C004FF0160A2E
:10D020000028A06B08D0E0B34FF6FF7000215F46E8
:10D03000ADF808B0019027E068B1B978C907BED152
:10D04000E18F0DAB0844821D03968DE80C024388E6
:10D050008288018809E0B878C007BCD0BA680DABF7
:10D0600003968DE80C02BB88FA881598FFF7F5F94E
:10D0700005005ED0072D72D076E0019005AA02A9C6
:10D080002046FFF72BF90146E28FBDF808008242E7
:10D0900001D00029F1D0E08FA16B084407800198EE
:10D0A000E08746E09DF81C004FF0180A40B1208B45
:10D0B000C8B13888208321461598FFF798F938E0E1
:10D0C00004F118000090237E012221461598FFF7F5
:10D0D000A6F98DF81C000028EDD119203070012030
:10D0E000ADF83400E7E7052521461598FFF77FF9ED
:10D0F0003AE0208800F40070ADF8200050452DD1B2
:10D10000A08FA0F57F41FE3901D006252CE0D8F88C
:10D1100008004FF0160A48B1A063B8F80C10A187B8
:10D120004FF6FF71E187A0F800B002E04FF6FF7004
:10D13000A087BDF8200030F47F611AD07823002248
:10D140000420159906F002F998F800002071208853
:10D15000BDF82010084320800EE000E0072520885D
:10D16000BDF8201088432080208810F47F6F1CD0E9
:10D170003AE02188814321809DF8380020B10EA932
:10D180001598F9F759FA05469DF81C000028EBD0D0
:10D1900086F801A001203070208B70809DF81C0063
:10D1A00030710520ADF83400DEE7A18EE1B11898AA
:10D1B0000DAB0088ADF834002398CDE90304CDE928
:10D1C0000139206B0090E36A179A1598FFF7FEF972
:10D1D000054601208DF838000EA91598F9F72CFAAC
:10D1E00000B10546A4F834B094F8460040070AD5CB
:10D1F0002046FFF7A2F910F03E0F04D114F8460FB5
:10D2000020F0040020701898BDF8341001802846E2
:10D210009DE500B585B0042806D102208DF80000F8
:10D2200088B26946F9F708FA05B000BD10B5384C68
:10D230000B782268012B02D0022B2AD111E013783F
:10D240000BB1052B01D10423137023688A889A80BF
:10D250002268CB88D38022680B8913814989518148
:10D260000DE08B8893802268CB88D38022680B895D
:10D2700013814B8953818B899381096911612168DD
:10D28000F9F7DAF9226800210228117003D000288A
:10D2900000D0812010BD832010BD806B002800D0FD
:10D2A000012070478178012909D10088B0F5205FFD
:10D2B00003D042F60101884201D1002070470720C7
:10D2C0007047F0B587B0002415460E460746ADF806
:10D2D000144010E0069801882980811DCDE90241A3
:10D2E000072101940494009183884288018838467C
:10D2F00000F0F4F830B906AA05A93046FEF7EEFFB3
:10D300000028E7D00A2800D1002007B0F0BD0000B7
:10D310005400002010B58B7883B102789A4205D171
:10D320000B885BB102E08B79091D4BB18B789A4277
:10D33000F9D1B0F801300C88A342F4D1002010BD1F
:10D34000812010BD072826D012B1012A27D103E081
:10D35000497801F0070102E04978C1F3C2010529CB
:10D360001DD2DFE801F00318080C12000AB10320F7
:10D3700070470220704704280DD250B10DE00528F7
:10D3800009D2801E022808D303E0062803D0032810
:10D3900003D005207047002070470F207047812080
:10D3A0007047C0B282060BD4000607D5FE48807ACB
:10D3B0004143C01D01EBD00080B270470846704762
:10D3C0000020704770B513880B800B781C0625D59C
:10D3D000F54CA47A844204D843F010000870002071
:10D3E00070BD956800F0070605EBD0052D78F54077
:10D3F00065F304130B701378D17803F0030341EA4B
:10D40000032140F20123B1FBF3F503FB15119268F0
:10D41000E41D00FB012000EBD40070BD906870BDDE
:10D4200037B51446BDF8041011809DF804100A06A3
:10D430001ED5C1F30013DC49A568897A814208D85A
:10D44000FE2811D1C91DC9085A42284611F0B4FA64
:10D450000AE005EBD00100F00702012508789540AD
:10D46000A843934018430870207820F010002070E3
:10D470003EBD2DE9F0410746C81C0E4620F00300D2
:10D48000B04202D08620BDE8F081C74D002034466E
:10D490002E60AF802881AA72E8801AE0E988491CD2
:10D4A000E980810614D4E17800F0030041EA00200D
:10D4B00040F20121B0FBF1F201FB12012068FFF7FD
:10D4C00070FF2989084480B22881381A3044A0604E
:10D4D0000C3420784107E1D40020D4E72DE9FF4F38
:10D4E00089B01646DDE9168A0F46994623F4404571
:10D4F000084600F00DFB04000FD0099802F00EFB67
:10D500000290207800060AD5A748817A02988142C5
:10D5100005D887200DB0BDE8F08F0120FAE722463C
:10D5200001A90298FFF74EFF834600208DF80C00FA
:10D530004046B8F1070F1AD001222146FFF702FF3B
:10D540000028E7D12078400611D502208DF80C0084
:10D55000ADF81070BDF80400ADF81200ADF814601D
:10D560001898ADF81650CDF81CA0ADF818005FEA79
:10D57000094004D500252E46A84601270CE0217855
:10D58000E07801F0030140EA012040F20121B0FB04
:10D59000F1F2804601FB12875FEA494009D5B845A0
:10D5A00007D1A178207901F0030140EA0120B042BF
:10D5B00001D3BE4201D90720ACE7A8191FFA80F9B0
:10D5C000B94501D90D20A5E79DF80C0028B103A9A4
:10D5D0000998F9F72FF800289CD1B84507D1A07811
:10D5E0004FEA192161F30100A07084F804901A98A1
:10D5F00000B10580199850EA0A0027D0199830B177
:10D600000BEB06002A46199911F05FF90EE00BEBBF
:10D6100006085746189E099802F0ECFB2B46F61DAB
:10D62000B5B239464246009501F0D7FF224601A91E
:10D630000298FFF7C7FE9DF80400224620F0100074
:10D640008DF80400DDE90110FFF7EAFE002061E734
:10D650002DE9FF4FDFF8509182461746B9F80610C2
:10D66000D9F8000001EB410100EB810440F20120F8
:10D67000B2FBF0F185B000FB11764D46DDF84C8031
:10D6800031460698FFF78DFE29682A898B46611A74
:10D690000C3101441144AB8889B28B4202D88420FA
:10D6A00009B038E70699CDB2290603D5A90601D5F8
:10D6B0000620F5E7B9F806C00CF1010C1FFA8CFC46
:10D6C000A9F806C0149909B1A1F800C0A90602D5AD
:10D6D000C4F8088007E0104480B2A9F80800191ABD
:10D6E00001EB0B00A0602246FE200699FFF798FE92
:10D6F000E77026712078390A61F30100320AA178B7
:10D7000040F0040062F30101A17020709AF8020059
:10D710006071BAF80000E08000262673280602D562
:10D7200099F80A7000E00127A80601D54FF000081B
:10D730004D4600244FF007090FE0CDE9026801963D
:10D74000CDF800900496E9882046129B089AFFF7CE
:10D75000C5FE0028A4D1641CE4B2BC42EDD3002075
:10D760009EE72DE9F047804600F0D2F9070005D08A
:10D77000002644460C4D40F2012919E00120BDE885
:10D78000F087204600F0C4F90278C17802F0030265
:10D7900041EA0222B2FBF9F309FB13210068FFF70B
:10D7A00000FE304486B201E0B8050020641CA4B23B
:10D7B000E988601E8142E4DCA8F10100E880288944
:10D7C000801B288100203870D9E710B5144631B18C
:10D7D000491E218002F0A2F9A070002010BD012096
:10D7E00010BD10B5D24904460088CA88904201D3C2
:10D7F0000A2010BD096800EB400001EB800250795F
:10D80000A072D08820819178107901F0030140EA5C
:10D810000120A081A078E11CFFF7D4FD20612088C1
:10D82000401C2080E080002010BD01210182704753
:10D830002DE9FF4F85B04FF6FF788246A3F80080B0
:10D8400048681F460D4680788DF8060048680088B5
:10D85000ADF8040000208DF80A00088A0C88A04268
:10D8600000D304462C8241E0288A401C2882701D87
:10D870006968FFF74FFDB8BB3988414501D1601E8B
:10D8800038806888A04236D3B178307901F003013E
:10D8900040EA012901A9701DFFF73CFD20BB298941
:10D8A00041452CD0002231460798FFF74BFDD8B9EF
:10D8B0002989494518D1E9680391B5F80AC0D6F815
:10D8C00008B05046CDF800C002F094FADDF800C070
:10D8D0005A460CF1070C1FFA8CFC4B460399CDF805
:10D8E00000C001F044FE50B1641CA4B2204600F018
:10D8F0000FF90600B8D1641E2C820A20D0E67C8085
:10D900007079B871F088B8803178F07801F003014F
:10D9100040EA01207881A7F80C90504602F0FEF80A
:10D92000324607F10801FFF74DFD38610020B7E6E8
:10D930002DE9FF4F87B081461C469246DDF860B066
:10D94000DDF85480089800F0E3F805000CD0484654
:10D9500002F0E4F82978090608D57549897A8142E8
:10D9600004D887200BB0D6E50120FBE7CAF30906EF
:10D970002A4601A9FFF726FD0746149807281CD060
:10D9800000222946FFF7DEFC0028EBD1287840066C
:10D9900013D501208DF808000898ADF80C00BDF8EB
:10D9A0000400ADF80E00ADF81060ADF8124002A909
:10D9B0004846F8F73FFE0028D4D12978E87801F0EE
:10D9C000030140EA0121AA78287902F0030240EA23
:10D9D0000220564507D0B1F5007F04D9611E81426F
:10D9E00001DD0B20BEE7864201D90720BAE7801B84
:10D9F00085B2A54200D92546BBF1000F01D0ABF896
:10DA00000050179818B1B9192A4610F05EFFB8F106
:10DA1000000F0DD03E4448464446169F02F0FCF9E4
:10DA20002146FF1DBCB232462B46009401F009FE90
:10DA3000002097E72DE9F04107461D4616460846A7
:10DA400000F066F804000BD0384602F067F8217841
:10DA5000090607D53649897A814203D8872012E51D
:10DA6000012010E522463146FFF7ACFC65B1217874
:10DA7000E07801F0030140EA0120B0F5007F01D811
:10DA8000012000E0002028700020FCE42DE9F04196
:10DA900007461D461646084600F03AF804000BD02B
:10DAA000384602F03BF82178090607D52049897AE3
:10DAB000814203D88720E6E40120E4E4224631468F
:10DAC000FFF7AEFCFF2D14D02178E07801F00302BF
:10DAD00040EA022040F20122B0FBF2F302FB130005
:10DAE00015B900F2012080B2E070000A60F3010174
:10DAF00021700020C7E410B50C4600F009F828B1E9
:10DB0000C18821804079A070002010BD012010BD87
:10DB10000749CA88824209D340B1096800EB400036
:10DB20006FF00B0202EB8000084470470020704742
:10DB3000B805002010B505F0BCFEFAF7BFFA05F0F5
:10DB400079FDBDE8104005F007BE70B50346002022
:10DB500002466FF02F050EE09C5CA4F130060A2E01
:10DB600002D34FF0FF3070BD00EB800005EB4000AA
:10DB7000521C2044D2B28A42EED370BD30B50A2482
:10DB80000AE0B0FBF4F304FB13008D18303005F805
:10DB9000010C521E1846D2B2002AF2D130BD30B567
:10DBA00000234FF6FF7510E0040A44EA002084B217
:10DBB000C85C6040C0F30314604005EA0034444090
:10DBC000E0B25B1C84EA40109BB29342ECD330BDC0
:10DBD0000178406829B190F8041190F8720038B9C2
:10DBE00001E001F0EFB919B1042901D0012070471B
:10DBF0000020704770B50C460546062101F0C8FFAD
:10DC0000606008B1002006E00721284601F0C0FF4F
:10DC1000606018B101202070002070BD022070BD2E
:10DC20002DE9FC470C4606466946FFF7E3FF00284E
:10DC30007DD19DF8000050B106F016FEB0427CD0B8
:10DC40002146304609F0B8FB002873D12DE00CF0D6
:10DC500067F9B04271D0214630460FF024FA00280F
:10DC600068D1019D95F8C80022E0012000E0002065
:10DC7000804695F835004FF0010A4FF00009F0B1E9
:10DC800095F8360080071AD584F8019084F800A032
:10DC900084F80290A68095F83710A171298F218110
:10DCA000698F618185F8359044E0019D95F8040104
:10DCB00058350028DBD1A87E0028D8D0D5E73046DB
:10DCC00002F0AAF8070000D1FFDF384601F0BAFAE7
:10DCD00040B184F801900E212170A680E08084F884
:10DCE00002A027E0304602F085F8070000D1FFDFF0
:10DCF000B8F1000F21D0384601F0FBFAB8B19DF819
:10DD0000000038B90198D0F8F0004188B14201D143
:10DD100080F80090304606F046FC84F801900B2114
:10DD2000217084F80290A680E97EA17100E004E0F1
:10DD300085F81A900120BDE8FC870020FBE71CB5A0
:10DD40006946FFF757FF00B1FFDF684601F046F96B
:10DD5000FE4900208968A1F8CA001CBD2DE9FC41DC
:10DD600004460E46062001F0BBFE0546072001F0E2
:10DD7000B7FE2844C7B20025A8463E4417E02088D5
:10DD8000401C80B22080B04202D34046A4F80080FC
:10DD900080B2B84204D3B04202D20020BDE8FC8178
:10DDA0006946FFF727FF0028F8D06D1CEDB2AE42A0
:10DDB000E5D84FF6FF7020801220EFE738B54FF618
:10DDC000FF70ADF800000DE00621BDF8000001F085
:10DDD000F1FE04460721BDF8000001F0EBFE0CB196
:10DDE00000B1FFDF00216846FFF7B8FF0028EBD045
:10DDF00038BD2DE9F04106F047FC0AF0C7FED44CCF
:10DE0000042710206780A0804FF6FF76E6832684E3
:10DE10000025D0A0257001680079A4F13E02A5710B
:10DE200042F8451FE11D1071A01D0FF06CFA25731B
:10DE30001B21E1814FF4A47020826182A082032221
:10DE4000A2752046E775018341833E38A2830570A1
:10DE50004680BE480C300570A4F110000570468065
:10DE6000BDE8F08170B5B94C0D466060217006F0D8
:10DE700098FBFFF7A3FFFFF7BCFF20780DF0B0FA87
:10DE80000CF04EFA217860680FF0E1F920780AF082
:10DE9000F9F8284607F08BFE06F026FD2178606829
:10DEA00009F079FBBDE870400AF070BE10B501249E
:10DEB0000AB1002010BD21B1012903D00024204661
:10DEC00010BD02210BF066FEF9E72DE9F0470400D2
:10DED00000D1FFDF9E48022120308146FFF73EFF40
:10DEE00000B1FFDF9A4D0620B5F8208001F0F8FD63
:10DEF0000646072001F0F4FD3044C6B2701CC7B2DC
:10DF0000288CB04211D120460BF094FF48BB2878F2
:10DF100078B300266670132020702021A01C10F01A
:10DF200053FD0220A0702E7020E0B8421AD1204686
:10DF300006F052FCE8B12078132817D1A0783C28CD
:10DF400014D1A088072101F023FE050000D1FFDFD6
:10DF5000288806F028FBA088072101F02BFE00B1DD
:10DF6000FFDF03E02146FFF75BFE10B10120BDE8B3
:10DF7000F087FFE702214846FFF7F0FE10B9298C31
:10DF80004145BDD10020F2E710B500F0C3FF08B154
:10DF90000C2010BD0AF031FE002010BD10B5044663
:10DFA000007818B1012801D0122010BD00F0C3FF85
:10DFB00020B10AF07FFE08B10C2010BD207800F0DF
:10DFC00078FFE21D04F11703611CBDE810400AF060
:10DFD00029BE10B50446007818B1012801D01220DE
:10DFE00010BD00F097FF08B10C2010BD207800F0A4
:10DFF00060FF611C0AF0DDFD08B1002010BD0720A4
:10E0000010BD10B50AF05AFE08B1002010BD302036
:10E0100010BD10B5044600F08EFF08B10C2010BDF5
:10E0200020460AF043FE002010BD10B500F083FF2B
:10E0300020B10AF03FFE08B10C2010BD0AF028FE06
:10E04000002010BDFF2181704FF6FF7181803F4994
:10E0500049680A7882718A88028149884181012150
:10E0600041700020704710B510F1080F17D00CDC7C
:10E0700010F1280F13D010F1140F10D010F1100F61
:10E080000DD010F10C0F08D109E010F1040F06D0EB
:10E0900028B1032803D0042801D0122010BD05F0B8
:10E0A00014FD002010BD10B5134601220BF08AF9B3
:10E0B000002010BD10B504460DF005FC052804D065
:10E0C00020460DF07CF9002010BD0C2010BD10B5CD
:10E0D000044600F030FF08B10C2010BD214600209E
:10E0E00006F0D3FA002010BD10B504460DF0F0F98B
:10E0F00050B107F0AAFF38B1207807F08AFD2078E8
:10E100000CF0ACFA002010BD0C2010BD10B5044678
:10E1100000F011FF08B10C2010BD2146012006F0CF
:10E12000B4FA002010BD38B504464FF6FF70ADF8C4
:10E130000000A079E17988421CD021791F2919D8E3
:10E1400061791F2916D80022114607E05C000020E3
:10E1500002060020FFFFFFFF1F0000000FF026FE59
:10E1600040B90022E07911460FF020FE10B9207A64
:10E17000072801D9122038BD07F073FF60B90DF0F0
:10E18000A2FB48B900216846FFF7E8FD20B1204610
:10E1900005F0BEFB002038BD0C2038BD2DE9FC4148
:10E1A000817805461A2925D00EDC16292DD2DFE804
:10E1B00001F02C2C2C2C2C212C2C2C2C2C2C2C2C11
:10E1C0002C2C2C2C2C2121212A291ED00BDCA1F156
:10E1D0001E010C2919D2DFE801F0181818181818B8
:10E1E00018181818180D3A3904290ED2DFE801F072
:10E1F0000D020D022888B0F5706F06D2012769461E
:10E20000FFF7F8FC18B10220C8E51220C6E59DF81A
:10E21000000000F055FE019C08B1EC3401E004F56B
:10E22000B3749DF8000000F04BFE019E08B1ED367E
:10E2300001E006F267166846FFF7CAFC08B12078CD
:10E2400008B10C20AAE52770A8783070684600F065
:10E25000C5FE0020A2E57CB50D466946FFF7CAFC65
:10E26000002618B12E602E7102207CBD9DF80000A2
:10E2700000F026FE019C9DF80000583400F020FEBE
:10E28000DDF8040084F83E6081682960017B297113
:10E2900094F83E100029F5D100207CBD10B540B1A6
:10E2A0000478406813B1B0F84A0003E0B0F84C00BD
:10E2B00000E0FB201B2908D3814206D8B2F5A47FD9
:10E2C00003D340F64800824201D9122010BD00203D
:10E2D00010BD2DE9FC41044600886946FFF78AFC21
:10E2E000002843D12289E18801236846FFF7D6FF41
:10E2F00000283BD1A288618800236846FFF7CEFF43
:10E30000070033D19DF80000019DB846012640B1B9
:10E3100085F88961019890F8C80105F5C47538B988
:10E3200013E085F8FD60019890F82001FC3508B1F4
:10E330003A2718E0E08868802089A8806088E88013
:10E34000A08828810122019909E0E088688020895D
:10E35000A8806088E880A08828810199002228464A
:10E360000BF03CF92E7085F80180384616E530B583
:10E3700085B00D460446008803A9FFF73BFC002842
:10E3800048D19DF80C0040B100220499E388B1F80F
:10E390004A00984203D2181A02E00122F5E7002051
:10E3A0006880B1F84C006388984201D2181A00E0E6
:10E3B0000020A8800020009001900290E088ADF835
:10E3C00002002089ADF804006088ADF80600A0883E
:10E3D000ADF8080068460BF001F92089BDF804107B
:10E3E000401AE880A088BDF80810401A2881E0880B
:10E3F000BDF80210411A6888814200DD0846688035
:10E400006088BDF80610411AA888814200DD0846E0
:10E41000A880002005B030BD10B5044600F08BFD8B
:10E4200020B10AF047FC08B10C2010BD207800F0A4
:10E4300040FDE279611C0AF082FD08B1002010BDA8
:10E44000022010BD7CB5044600886946FFF7D2FB68
:10E4500000282FD1A17801B90321E27802B9032263
:10E460009DF8005000240123002D019D06D085F861
:10E470009331019D95F8DC512DBB1CE085F80731E7
:10E48000019D95F82C513DB9019D95F806511DB996
:10E49000019D95F87B500DB13A2008E0019D85F86B
:10E4A0000631019B83F80811019981F8092101992E
:10E4B00081F807417CBD019D95F892511DB9019DE0
:10E4C00095F87B500DB13A2008E0019D85F8923116
:10E4D000019B83F89411019981F89521019981F8A4
:10E4E00093417CBD8178CA0802D1C278D30801D09B
:10E4F00012207047490701D4510701D511207047F8
:10E50000A0E710B5044600F0F8FC08B10C2010BDDF
:10E51000A1791220012904D019B1022901D00329BF
:10E52000F5D1217809B10129F1D1E17929B1012988
:10E5300003D0022901D00329E9D1618843F6FD7295
:10E540000B1F30209342E2D2A3881B1F9342DED2DE
:10E55000F9484180A1888180A0790BF0D3FFE07950
:10E560000CF00CF82078012805D00120BDE81040FF
:10E5700000210CF036B80220F8E710B5122201286D
:10E5800002D008B1104610BD09B10129FAD1012805
:10E5900007D00DF098F9052811D0BDE810400CF017
:10E5A000C7BE0BF0A5FF40B10BF0B4FFE248818875
:10E5B0004088BDE810400CF097BF122010BD0C2021
:10E5C00010BD2DE9F047DC4E92460C46B0F84C20C9
:10E5D0000546F1891046814200D20846074695F863
:10E5E0005210104600F080FC318A814200D2084669
:10E5F000B5F84A208046718A1046B146814200D261
:10E600000846064695F85110104600F06DFCB9F822
:10E610001410814200D208464FF4A4721B2E01D080
:10E62000904203D11B2F0DD090450BD0E780A4F86A
:10E6300008806680A0805246294620460AF0CEFF18
:10E640000120207093E430B5428840F67B43911F4F
:10E65000994219D281888C1F9C4215D28A4213D8C4
:10E66000C288B2F5FA7F0FD2038940F67745A3F14D
:10E670000A04AC4208D2521C4A43B2EB830F03DABD
:10E6800041898089814201D9302030BD002030BDD0
:10E690001FB5018843F6FD720B1F934205D24388D4
:10E6A0001C1F944201D28B4202D9302004B010BD0D
:10E6B000017911B1012910D107E0417929B101296E
:10E6C00003D0022901D0032907D1017B39B10129E7
:10E6D00005D0022903D0032901D01220E6E7C18921
:10E6E000ADF80210018AADF80410418AADF80610A9
:10E6F000818AADF80810C18AADF80A10008BADF818
:10E700000C006846FFF79FFFD0E72DE9F04385B086
:10E710000546AFF2C051D1E90086FFF7B9FF0028E6
:10E7200011D10DF0D0F805280CD00DF0CCF804284C
:10E7300008D0814F387828B90BF0F2FBA0F57F4163
:10E74000FF3903D00C2005B0BDE8F0837A4801AA58
:10E750003E3801907948029077480621103803909E
:10E7600004A801F0E3F904007ED003210AF07BFD48
:10E770007148B946018BA4F84A10418BA4F84C109B
:10E78000428B018BFB7D0093BB7D208801F0BBFA9F
:10E7900000B1FFDF208805F005FF218804F10E009D
:10E7A00000F0D3FB66A004F112070068009003217B
:10E7B000684604F073FB002069460A5C3A54401C2A
:10E7C000C0B20328F9D3288A6080688AA080A88A0A
:10E7D000E08094F8522094F85110B9F81C000CF025
:10E7E00009FF0146A06220460CF012FF002784F8C2
:10E7F0005E7084F85F70687900F05BFB6076D5F836
:10E800000600C4F81A006889E083C4F808802673FB
:10E81000012084F8F800024604F1FC012046FFF7CD
:10E82000D0FE8DF800700121684604F037FB9DF89A
:10E83000000000F00701C0F3C1021144C0F3401012
:10E8400008448DF80000401D2076092801D20830C8
:10E850002076002120460AF006FD287B0BF052FEB0
:10E8600069792879AA1D00E00CE00BF023FE58B16D
:10E870000BF050FE69792879AA1D0BF08AFE06007C
:10E8800004D010E009205EE712260CE021460320A8
:10E890000BF0A7FE060006D16A88298820460CF0F6
:10E8A000DBFD060008D0208805F07DFE20880621CB
:10E8B00001F080F900B1FFDF304644E738B51E4C67
:10E8C000207870B90CF0FFFF052805D00BF028FB6D
:10E8D000A0F57F41FF3904D068460CF033FE10B13B
:10E8E00013E00C2038BD0098008805F05CFE00980D
:10E8F0000621008801F05EF900B1FFDF01202070E1
:10E900000E480C380078FCF7FDFF002038BD70B5CC
:10E910000546FFF798FE002815D12888062101F04A
:10E9200037F904000ED000F04DFB58B1D4F8F000D8
:10E93000017869B908E000000206002068000020A4
:10E9400011223300022070BDD4F83C11097809B1BE
:10E950003A2070BD05218171D4F8F01000200881A3
:10E96000D4F8F010A8884881D4F8F010E88888819D
:10E97000D4F8F0102889C881D4F8F00002894189C0
:10E980008A4204D88279082A01D88A4201D3122007
:10E9900070BD29884180D4F8F01002200870002052
:10E9A00070BD3EB504460AF0DBFCB0B1FC48012561
:10E9B000A0F13E028571236842F8453F237900218A
:10E9C000137181716946062001F06BF800B1FFDF19
:10E9D000684601F044F810B10EE012203EBDBDF8CB
:10E9E0000440029880F8F850684601F038F818B9E9
:10E9F000BDF80400A042F4D100203EBD70B505462C
:10EA00000088062101F0C4F8040007D000F0DAFA0B
:10EA100020B1D4F8F010087830B901E0022070BDC0
:10EA2000D4F83C01007808B13A2070BD9420005D14
:10EA300010F0010F18D0D5F802004860D5F8060094
:10EA4000886054F8F00F698910228181206805F1EF
:10EA50000C010E300FF039FF216803200870216887
:10EA600028884880002070BD0C2070BD10B5044679
:10EA700007F0F7FA08B10C2010BD6079032824D8FC
:10EA8000A179012921D8A17B03291ED8617BE1B19D
:10EA900007291AD82179052917D2DFE801F0030CDC
:10EAA000030303002288202A0FD361888A420CD8EE
:10EAB000B1F5804F09D805F071FFB9492079487048
:10EAC0002046BDE8104006F031B8122010BD10B548
:10EAD0001F2801D9122010BD06F0A2F8002010BD99
:10EAE00010B51F2801D9122010BD06F088F80020AB
:10EAF00010BD7CB5012802D000285DD070E005F083
:10EB0000FDFE00286CD005F02FFF002868D007F02C
:10EB1000A8FA002856D105F0A7FEA0F57F41FF39DD
:10EB200050D105F0B9FF9E4E707848B1012807D04A
:10EB3000042805D0002007F06FF8D0B3FFDF4DE0C8
:10EB40000022072101A800F0F1FF040032D095480F
:10EB50000321846020460AF013FB204606F065F985
:10EB60008F4D0121288BA4F84A00688BA4F84C0033
:10EB7000B08B07F019F90146A0620022204606F08A
:10EB800052FC6A8B298BF07D0090B37D208801F0C8
:10EB9000BAF800B1FFDF208805F004FD204607F039
:10EBA0003BF800B1FFDF002204F5C4712046FFF7F7
:10EBB00008FD13E009207CBD06F016FC044606F0B3
:10EBC000CFFF08B10C207CBD44B1208805F0EBFCE0
:10EBD0002088072100F0EEFF00B1FFDF00207CBDA0
:10EBE00012207CBD70B50D46072100F0D1FF040056
:10EBF00003D094F8690110B10AE0022070BD94F8C6
:10EC00006400142801D0152802D194F8AA0108B193
:10EC10000C2070BD1022294604F5B5700FF055FE8A
:10EC2000012084F86901002070BD10B5072100F0B3
:10EC3000AFFF18B190F8691111B107E0022010BDC3
:10EC400090F86410142903D0152901D00C2010BDB0
:10EC5000022180F86911002010BD2DE9FC410C460D
:10EC60004BF68032122194421DD8E4B16946FEF77A
:10EC7000C1FF002815D19DF8000000F021F9019E88
:10EC80009DF80000583600F01BF9019DAD1C2F883F
:10EC90002246394630460AF036FA2888B842F6D17C
:10ECA0000020BDE8FC810846FBE77CB504460088EF
:10ECB0006946FEF79FFF002817D19DF8000000F07D
:10ECC000FFF8019D9DF80000583500F0F9F87F210C
:10ECD0000198297269720021A972A17800F82C1F8D
:10ECE000E17841702179817000207CBD1CB50C4613
:10ECF0006946FEF77FFF00280AD19DF8000000F06A
:10ED0000DFF8019890F8720000B101202070002017
:10ED10001CBD1CB50C466946FEF76CFF002809D1E6
:10ED20009DF8000000F0CCF8019890F82C00012824
:10ED300001D00C201CBD9DF8000000F0C1F8019826
:10ED400090F86000207000201CBD70B50D4616467E
:10ED5000072100F01DFF38B381880124C388428851
:10ED600004EB4104AC4217D842F210746343A41080
:10ED70006243B3FBF2F2521E94B24FF4FA72944221
:10ED800000D91446A54200D22C46491C641CB4FB91
:10ED9000F1F24A43521E91B290F8962142B906E030
:10EDA000020600205C000020FFE7022070BD018405
:10EDB0003180002070BD10B50C46072100F0E8FE40
:10EDC00048B180F8D74024B190F8D51009B107F0C8
:10EDD00008F8002010BD022010BD017889B14178EB
:10EDE00079B141881B290CD381881B2909D3C1889B
:10EDF000022906D3814902684A6540688865002077
:10EE000070471220704710B504460CF0EFFB204607
:10EE100006F099FF002010BD2DE9F04115460F4680
:10EE200006460122114638460CF0E4FB0446012157
:10EE3000384606F0B9FF844200D20446012130462C
:10EE400000F043F806460121002000F03EF831189A
:10EE5000012096318C4206D901F19600611AB1FB6E
:10EE6000F0F0401C80B228800020BDE8F08110B591
:10EE7000044600F060F808B10C2010BD601C0AF0D8
:10EE800035F8207800F0010005F08BFD207800F0C7
:10EE900001000BF03BFB002010BD10B5044607F04D
:10EEA000E0F808B10C2010BD204605F0C9FE002096
:10EEB00010BD18B1022801D0012070470020704712
:10EEC00008B1002070470120704710B5012904D017
:10EED000022905D0FFDF204610BDC000503001E000
:10EEE00080002C3084B2F6E7022903D0C0007030D5
:10EEF00080B2704780003C30FAE710B50CF0E3FCBC
:10EF0000042805D00CF0DFFC052801D0002010BD3E
:10EF1000012010BD10B5FFF7F0FF10B10BF06AFB38
:10EF200028B907F09EF820B105F017FD08B10120BF
:10EF300010BD002010BD10B5FFF7DFFF18B907F0B6
:10EF400090F8002800D0012010BD2DE9FE430025D7
:10EF50000F4680460A260421404603F0C8FF40467B
:10EF60000AF0DCF9062000F0BBFD044615E0694616
:10EF7000062000F096FD0AE0BDF80400B84206D075
:10EF80000298042241460E300FF073FC50B16846DF
:10EF900000F065FD0500EFD0641E002C06DD002D9D
:10EFA000E5D005E040460AF0C3F9F5E705B9FFDF13
:10EFB000D8F800000AF0B1F8761E01D00028CAD0B7
:10EFC000BDE8FE8390F8C81090F8720020B919B11E
:10EFD000042901D0012070470020704701780029E2
:10EFE0000AD0416891F8D520002A05D0002281F886
:10EFF000D520406806F0F5BE70470000C40500202B
:10F0000030B5058825F4004421448CB24FF400410A
:10F0100094420AD2121B92B21B339A4201D2A943E4
:10F0200007E005F40041214303E0A21A92B2A9438C
:10F030001143018030BD0844083050434A31084430
:10F0400080B2704770B51D4616460B4604462946E9
:10F050003046049AFFF7EFFF0646B34200D2FFDFC7
:10F06000282120460FF0D2FC4FF6FF70A082283EE8
:10F07000B0B265776080B0F5004F00D9FFDF6188DE
:10F0800005F13C00814200D2FFDF60880835401B5B
:10F09000343880B220801B2800D21B202080002022
:10F0A000A07770BD8161886170472DE9F05F0D46E2
:10F0B000C188044600F12809008921F4004620F4A3
:10F0C000004800F062FB10B10020BDE8F09F4FF057
:10F0D000000A4FF0010BB0450CD9617FA8EB060088
:10F0E000401A0838854219DC09EB0600002105802A
:10F0F00041801AE06088617F801B471A083F0DD469
:10F100001B2F00DAFFDFBD4201DC294600E0B9B267
:10F11000681A0204120C04D0424502DD84F817A0DC
:10F12000D2E709EB06000180428084F817B0CCE7F3
:10F1300070B5044600F12802C088E37D20F4004049
:10F140002BB110440288438813448B4201D2002023
:10F1500070BD00258A4202D30180458008E0891AEB
:10F160000904090C418003D0A01D00F01EFB08E03B
:10F17000637F00880833184481B26288A01DFFF7BE
:10F180003FFFE575012070BD70B5034600F128040E
:10F19000C588808820F400462644A84202D1002079
:10F1A000188270BD98893588A84206D3401B75889F
:10F1B0002D1A2044ADB2C01E05E02C1AA5B25C7F0A
:10F1C00020443044401D0C88AC4200D90D809C89FD
:10F1D00024B1002414700988198270BD0124F9E754
:10F1E00070B5044600F12801808820F400404518DD
:10F1F000208A002825D0A189084480B2A0812988CE
:10F200006A881144814200D2FFDF2888698800267D
:10F210000844A189884212D1A069807F2871698839
:10F2200019B1201D00F0C1FA08E0637F2888083377
:10F23000184481B26288201DFFF7E2FEA681268273
:10F24000012070BD2DE9F0414189878800260446E0
:10F2500000F12805B94218D004F10A0821F4004051
:10F260002844418819B1404600F09FFA08E0637FC6
:10F2700000880833184481B262884046FFF7C0FE18
:10F28000761C6189B6B2B942E8D13046BDE8F0815A
:10F290002DE9F04104460B4627892830A68827F43B
:10F2A0000041B4F80A8001440D46B74201D1002064
:10F2B000ECE70AB1481D106023B1627F691D184652
:10F2C0000FF003FB2E88698804F1080021B18A1928
:10F2D00096B200F06AFA06E0637F628808339919F3
:10F2E00089B2FFF78DFE474501D120896081304604
:10F2F000CCE78188C088814201D10120704700207D
:10F30000704701898088814201D101207047002027
:10F31000704770B58588C38800F1280425F4004241
:10F3200023F4004114449D421AD08389058A5E1952
:10F3300025886388EC18A64214D313B18B4211D3ED
:10F340000EE0437F08325C192244408892B2801A52
:10F3500080B22333984201D211B103E08A4201D135
:10F36000002070BD012070BD2DE9F0478846C1889E
:10F370000446008921F4004604F1280720F40045E2
:10F3800007EB060900F001FA002178BBB54204D969
:10F39000627FA81B801A002503E06088627F801BC3
:10F3A000801A083823D4E28962B1B9F80020B9F88C
:10F3B00002303BB1E81A2177404518DBE089384438
:10F3C000801A09E0801A217740450ADB607FE189D5
:10F3D0000830304439440844C01EA4F81280BDE807
:10F3E000F087454503DB01202077E7E7FFE76182EF
:10F3F0000020F4E72DE9F74F044600F12805C08806
:10F40000884620F4004A608A05EB0A0608B14045A8
:10F4100002D20020BDE8FE8FE08978B13788B6F8C7
:10F42000029007EB0901884200D0FFDF207F4FF0F8
:10F43000000B50EA090106D088B33BE00027A07F0B
:10F44000B9463071F2E7E18959B1607F294408304B
:10F4500050440844B4F81F1020F8031D94F82110FC
:10F460008170E28907EB080002EB0801E18130803E
:10F47000A6F802B002985F4650B1637F3088083327
:10F48000184481B26288A01DFFF7BAFDE78121E030
:10F49000607FE18908305044294408442DE0FFE7AB
:10F4A000E089B4F81F102844C01B20F8031D94F80D
:10F4B0002110817009EB0800E28981B202EB08009B
:10F4C000E081378071800298A0B1A01D00F06DF935
:10F4D000A4F80EB0A07F401CA077A07D08B1E08802
:10F4E000A08284F816B000BFA4F812B084F817B058
:10F4F00001208FE7E0892844C01B30F8031DA4F8E1
:10F500001F10807884F82100EEE710B5818800F1A3
:10F51000280321F400442344848AC288A14212D0E3
:10F52000914210D0818971B9826972B11046FFF79A
:10F53000E8FE50B91089283220F4004010441979AF
:10F540000079884201D1002010BD184610BD00F19D
:10F550002803407F08300844C01E1060088808B99E
:10F56000DB1E136008884988084480B270472DE983
:10F57000F04100F12806407F1C46083090464318B1
:10F5800008884D88069ADB1EA0B1C01C80B290424C
:10F5900014D9801AA04200DB204687B298183A4658
:10F5A00041460FF066F9002816D1E01B84B2B8443A
:10F5B000002005E0ED1CADB2F61EE8E7101A80B29F
:10F5C0000119A94206D8304422464146BDE8F0411F
:10F5D0000FF04FB94FF0FF3058E62DE9F04100F140
:10F5E0002804407F1E4608309046431800250888AE
:10F5F0004F88069ADB1E90B1C01C80B2904212D98F
:10F60000801AB04200DB304685B299182A4640463F
:10F610000FF05BF9701B86B2A844002005E0FF1CC8
:10F62000BFB2E41EEAE7101A80B28119B94206D8C7
:10F630002118324640460FF048F9A81985B22846ED
:10F6400024E62DE9F04100F12804407F1E460830F1
:10F6500090464318002508884F88069ADB1E90B113
:10F66000C01C80B2904212D9801AB04200DB3046F2
:10F6700085B298182A4641460FF027F9701B86B2CA
:10F68000A844002005E0FF1CBFB2E41EEAE7101A00
:10F6900080B28119B94206D82044324641460FF063
:10F6A00014F9A81985B22846F0E5401D704710B539
:10F6B000044600F12801C288808820F400431944E0
:10F6C000904206D0A28922B9228A12B9A28A904217
:10F6D00001D1002010BD0888498831B1201D00F0FB
:10F6E00064F800202082012010BD637F6288083307
:10F6F000184481B2201DFFF783FCF2E70021C1818D
:10F7000001774182C1758175704703881380C28972
:10F7100042B1C28822F4004300F128021A440A6070
:10F72000C08970470020704710B50446808AA0F554
:10F730007F41FF3900D0FFDFE088A082E08900B17F
:10F740000120A07510BD4FF6FF71818200218175E7
:10F75000704710B50446808AA0F57F41FF3900D17B
:10F76000FFDFA07D28B9A088A18A884201D10020AE
:10F7700010BD012010BD8188828A914201D1807D17
:10F7800008B1002070470120704720F4004221F4A6
:10F7900000439A4207D100F4004001F4004188423E
:10F7A00001D0012070470020704730B50446008822
:10F7B0000D4620F40040A84200D2FFDF21884FF41C
:10F7C000004088432843208030BD70B50C000546BA
:10F7D00009D0082C00D2FFDF1DB1A1B2286800F0CB
:10F7E00044F8201D70BD0DB100202860002070BDC0
:10F7F0000021026803E093881268194489B2002A44
:10F80000F9D100F032B870B500260D46044608293B
:10F8100000D2FFDF206808B91EE004462068818816
:10F82000A94202D001680029F7D181880646A94281
:10F8300001D100680DE005F1080293B2002299425F
:10F8400009D32844491B026081802168096821602E
:10F850000160206000E00026304670BD00230B6090
:10F860008A8002680A600160704700234360021DBD
:10F87000018102607047F0B50F4601884088154647
:10F880000C181E46AC4200D3641B3044A84200D979
:10F89000FFDFA019A84200D9FFDF3819F0BD2DE91C
:10F8A000F041884606460188408815460C181F46D8
:10F8B000AC4200D3641B3844A84200D9FFDFE019F2
:10F8C000A84200D9FFDF70883844708008EB04003C
:10F8D000BDE8F0812DE9F041054600881E46174637
:10F8E000841B8846BC4200D33C442C80688830444A
:10F8F000B84200D9FFDFA019B84200D9FFDF6888FD
:10F900003044688008EB0400E2E72DE9F041068806
:10F910001D460446701980B2174688462080B842BA
:10F9200001D3C01B20806088A84200D2FFDF70197D
:10F93000B84200D9FFDF6088401B608008EB0600FA
:10F94000C6E730B50D460188CC18944200D3A41AFE
:10F950004088984200D8FFDF281930BD2DE9F041DA
:10F96000C84D04469046A8780E46A04200D8FFDF56
:10F9700005EB8607B86A50F8240000B1FFDFB868CD
:10F98000002816D0304600F044F90146B868FFF769
:10F990003AFF05000CD0B86A082E40F8245000D376
:10F9A000FFDFB9484246294650F82630204698479E
:10F9B0002846BDE8F0812DE9F8431E468C19914692
:10F9C0000F460546FF2C00D9FFDFB14500D9FFDF08
:10F9D000E4B200954DB300208046E81C20F00300FF
:10F9E000A84200D0FFDF4946DFF89892684689F8C0
:10F9F000001089F8017089F8024089F8034089F8FD
:10FA0000044089F8054089F8066089F80770414686
:10FA100000F008F9002142460F464B460098C01CF2
:10FA200020F00300009012B10EE00120D4E703EBB8
:10FA30008106B062002005E0D6F828C04CF820709E
:10FA4000401CC0B2A042F7D30098491C00EB8400D0
:10FA5000C9B200900829E1D3401BBDE8F88310B576
:10FA6000044603F08FFD08B1102010BD2078854AB0
:10FA7000618802EB800092780EE0836A53F82130AF
:10FA800043B14A1C6280A180806A50F82100A060C6
:10FA9000002010BD491C89B28A42EED86180052041
:10FAA00010BD70B505460C46084603F06BFD08B165
:10FAB000102070BD082D01D3072070BD25700020D7
:10FAC000608070BD0EB56946FFF7EBFF00B1FFDF48
:10FAD0006846FFF7C4FF08B100200EBD01200EBD2F
:10FAE00010B50446082800D3FFDF6648005D10BD4E
:10FAF0003EB5054600246946FFF7D3FF18B1FFDF86
:10FB000001E0641CE4B26846FFF7A9FF0028F8D0C2
:10FB10002846FFF7E5FF001BC0B23EBD5949897872
:10FB2000814201D9C0B27047FF2070472DE9F041F2
:10FB3000544B062903D007291CD19D7900E00025EC
:10FB400000244FF6FF7603EB810713F801C00AE0AB
:10FB50006319D7F828E09BB25EF823E0BEF1000FEE
:10FB600004D0641CA4B2A445F2D8334603801846DE
:10FB7000B34201D100201CE7BDE8F041EEE6A0F55C
:10FB80007F43FF3B01D0082901D300207047E5E601
:10FB9000A0F57F42FF3A0BD0082909D2394A937861
:10FBA000834205D902EB8101896A51F82000704730
:10FBB000002070472DE9F04104460D46A4F57F4131
:10FBC00043F20200FF3902D0082D01D30720F0E6EE
:10FBD0002C494FF000088A78A242F8D901EB85063B
:10FBE000B26A52F82470002FF1D0274839462030ED
:10FBF00050F8252020469047B16A284641F82480D5
:10FC000000F007F802463946B068FFF727FE0020EB
:10FC1000CFE61D49403131F810004FF6FC71C01C91
:10FC2000084070472DE9F843164E884605460024E3
:10FC30002868C01C20F0030028602046FFF7E9FF79
:10FC4000315D4843B8F1000F01D0002200E02A687E
:10FC50000146009232B100274FEA0D00FFF7B5FDD3
:10FC60001FB106E001270020F8E706EB8401009AA7
:10FC70008A602968641C0844E4B22860082CD7D341
:10FC8000EBE600002406002008EE010070B50E46E9
:10FC90001D46114600F0D4F804462946304600F0CF
:10FCA000D8F82044001D70BD2DE9F04190460D4666
:10FCB00004004FF0000610D00027E01C20F00300E5
:10FCC000A04200D0FFDFDDB141460020FFF77DFDFF
:10FCD0000C3000EB850617B112E00127EDE7614F0C
:10FCE00004F10C00A9003C602572606000EB850007
:10FCF000206060680EF08AFE41463868FFF765FDB7
:10FD00003046BDE8F0812DE9FF4F564C804681B06A
:10FD100020689A46934600B9FFDF2068027A424580
:10FD200003D9416851F8280020B143F2020005B020
:10FD3000BDE8F08F5146029800F082F886B258462E
:10FD40000E9900F086F885B27019001D87B2206800
:10FD5000A14639460068FFF756FD04001FD06780B2
:10FD600025802946201D0E9D07465A4601230095F1
:10FD7000FFF768F92088314638440123029ACDF80C
:10FD800000A0FFF75FF92088C1193846FFF78AF90C
:10FD9000D9F800004168002041F82840C7E7042056
:10FDA000C5E770B52F4C0546206800B9FFDF206815
:10FDB000017AA9420ED9426852F8251051B10023A8
:10FDC00042F825304A880068FFF748FD2168002086
:10FDD0000A7A08E043F2020070BD4B6853F8203005
:10FDE00033B9401CC0B28242F7D80868FFF700FD63
:10FDF000002070BD70B51B4E05460024306800B968
:10FE0000FFDF3068017AA94204D9406850F8250024
:10FE100000B1041D204670BD70B5124E0546002489
:10FE2000306800B9FFDF3068017AA94206D940681E
:10FE300050F8251011B131F8040B4418204670BD5C
:10FE400010B50A460121FFF7F6F8C01C20F00300A8
:10FE500010BD10B50A460121FFF7EDF8C01C20F0D7
:10FE6000030010BD7000002070B50446C2F11005FB
:10FE700028190EF02AFD15F0FF0108D0491EC9B25D
:10FE8000802060542046BDE870400EF09DBD70BDDE
:10FE900030B505E05B1EDBB2CC5CD55C6C40C45475
:10FEA000002BF7D130BD10B5002409E00B78521EAD
:10FEB00044EA430300F8013B11F8013BD2B2DC09EC
:10FEC000002AF3D110BD2DE9F04389B01E46DDE9CB
:10FED000107990460D00044622D002460846F949A2
:10FEE000FEF7E1F8102221463846FFF7DCFFE07B01
:10FEF000000606D5F34A3946102310320846FFF7AC
:10FF0000C7FF102239464846FFF7CDFFF87B0006B1
:10FF100006D5EC4A4946102310320846FFF7B8FFD1
:10FF2000102120460EF050FD0DE0103EB6B208EB59
:10FF30000601102322466846FFF7AAFF22462846FC
:10FF40006946FEF7B0F8102EEFD818D0F2B241464D
:10FF50006846FFF789FF10234A46694604A8FFF761
:10FF600097FF1023224604A96846FFF791FF224617
:10FF700028466946FEF797F809B0BDE8F0831023DC
:10FF80003A464146EAE770B59CB01E460546134620
:10FF900020980C468DF80800202219460DF1090022
:10FFA0000EF093FC202221460DF129000EF08DFC6D
:10FFB00017A913A8CDE90001412302AA314628461A
:10FFC000FFF781FF1CB070BD2DE9FF4F9FB014AE4D
:10FFD000DDE92D5410AFBB49CDE900762023203157
:10FFE0001AA8FFF770FF4FF000088DF808804FF057
:10FFF00001098DF8099054F8010FCDF80A00A08886
:020000040001F9
:10000000ADF80E0014F8010C1022C0F340008DF87A
:10001000100055F8010FCDF81100A888ADF81500B3
:1000200015F8010C2C99C0F340008DF8170006A8B4
:1000300082460EF04AFC0AA88346102222990EF04E
:1000400044FCA0483523083802AA40688DF83C805B
:10005000CDE900760E901AA91F98FFF734FF8DF8AE
:1000600008808DF809902068CDF80A00A088ADF8C6
:100070000E0014F8010C1022C0F340008DF810009F
:100080002868CDF81100A888ADF8150015F8010C06
:100090002C99C0F340008DF8170050460EF015FC67
:1000A0005846102222990EF010FC86483523083855
:1000B00002AA40688DF83C90CDE900760E901AA90E
:1000C0002098FFF700FF23B0BDE8F08FF0B59BB09C
:1000D0000C460546DDE922101E461746DDE92032B2
:1000E000D0F801C0CDF808C0B0F805C0ADF80CC01C
:1000F0000078C0F340008DF80E00D1F80100CDF873
:100100000F00B1F80500ADF8130008781946C0F3E8
:1001100040008DF815001088ADF8160090788DF825
:1001200018000DF1190010220EF0CFFB0DF129007F
:10013000102231460EF0C9FB0DF13900102239466C
:100140000EF0C3FB17A913A8CDE90001412302AAB1
:1001500021462846FFF7B7FE1BB0F0BDF0B5A3B0AF
:1001600017460D4604461E46102202A828990EF096
:10017000ACFB06A8202239460EF0A7FB0EA82022D1
:1001800029460EF0A2FB1EA91AA8CDE900015023B2
:1001900002AA314616A8FFF796FE1698206023B0F3
:1001A000F0BDF0B589B00446DDE90E070D4639789B
:1001B000109EC1F340018DF8001031789446C1F3D0
:1001C00040018DF801101968CDF802109988ADF83A
:1001D000061099798DF808100168CDF8091081880A
:1001E000ADF80D1080798DF80F0010236A46614636
:1001F00004A8FFF74DFE2246284604A9FDF753FF49
:10020000D6F801000090B6F80500ADF80400D7F864
:100210000100CDF80600B7F80500ADF80A0000208F
:10022000039010236A46214604A8FFF731FE2246B8
:10023000284604A9FDF737FF09B0F0BD1FB51C68BB
:1002400000945B680193136802935268039202461C
:1002500008466946FDF727FF1FBD10B588B0044664
:10026000106804905068059000200690079008469A
:100270006A4604A9FDF717FFBDF80000208008B00A
:1002800010BD1FB51288ADF800201A88ADF8022005
:100290000022019202920392024608466946FDF747
:1002A00002FF1FBD7FB5074B14460546083B9A1C4D
:1002B0006846FFF7E6FF224669462846FFF7CDFF6E
:1002C0007FBD000060EE010070B5044600780E4668
:1002D000012813D0052802D0092813D10EE0A06808
:1002E00061690578052003F0DBF8052D0AD0782335
:1002F00000220520616903F029F803E00520616907
:1003000003F0CEF831462046BDE8704001F086B8D3
:1003100010B500F12D02C3799478411D64F00304F7
:100320002340C371DB070DD04B79547923404B71C7
:100330000B79127913400B718278C9788A4200D9FF
:10034000817010BD00224A710A71F5E741780129D8
:1003500000D00C21017070472DE9F04F93B04FF0A1
:10036000000B0C690D468DF820B0097801260C2091
:1003700017464FF00D084FF0110A4FF008091B29DE
:1003800075D2DFE811F01B00C30206031E035D03F4
:100390007003A203B703F803190461049304A004D3
:1003A000EC042A05340552055D05EE0531063406D8
:1003B00063067F06F9061D07E606EB0614B12078F2
:1003C0001D282AD0D5F808805FEA08004FD0012008
:1003D0008DF82000686A02220D908DF824200A20F2
:1003E0008DF82500A8690A90A8880028EED098F812
:1003F000001091B10F2910D27ED2DFE801F07D13F9
:1004000049DEFEFDFCFBFAF938089CF8F7000228EB
:100410002DD124B120780C2801D00026EFE38DF8EF
:100420002020CBE10520696A03F03AF8A888072864
:10043000EED1204600F0EDFF022809D0204600F062
:10044000E8FF032807D9204600F0E3FF072802D27F
:100450000120207004E0002CB8D020780128D7D1EA
:1004600098F80400C11F0A2902D30A2061E0C4E100
:10047000A070D8F80010E162B8F80410218698F84E
:10048000060084F83200012028700320207044E028
:100490000728BDD1002C99D020780D28B8D198F824
:1004A000031094F82F20C1F3C000C2F3C002104221
:1004B00001D0062000E00720890707D198F8051031
:1004C0000142D2D198F806100142CED194F83120E1
:1004D00098F8051020EA02021142C6D194F83220A1
:1004E00098F8061090430142BFD198F80400C11F4C
:1004F0000A29BAD2617D00E006E281427ED8D8F8AE
:1005000000106160B8F80410218198F80600A0720C
:10051000012028700E20207003208DF82000686ACA
:100520000D9004F12D000990601D0A900F300B9082
:1005300022E12875FDE3412891D1204600F069FFB2
:10054000042802D1E078C00704D1204600F061FF02
:100550000F2884D1A88CD5F80C8080B24FF0400BC6
:10056000E669FFF747FC324641465B464E46CDF80A
:100570000090FFF732F80B208DF82000686A0D908C
:10058000E0690990002108A8FFF79EFE2078042862
:1005900006D0A07D58B1012809D003280AD049E32C
:1005A00005202070032028708DF82060CDE184F8AC
:1005B00000A032E712202070E9E11128BCD12046CA
:1005C00000F027FF042802D1E078C00719D02046A8
:1005D00000F01FFF062805D1E078C00711D1A07DEB
:1005E00002280ED0204600F014FF08E0CAE081E0A7
:1005F0006FE14EE121E101E1E7E017E0ADE1112813
:100600009AD1102208F1010104F13C000EF05DF9CD
:10061000607801287ED012202070E078C00760D07A
:10062000A07D0028C8D00128C6D05AE0112890D15A
:10063000204600F0EEFE082804D0204600F0E9FE37
:10064000132886D104F16C00102208F1010106463E
:100650000EF03BF9207808280DD014202070E178A6
:10066000C8070DD0A07D02280AD06278022A04D0E3
:100670000328A1D035E00920F0E708B1012837D1DF
:10068000C80713D0A07D02281DD000200090D4E917
:10069000062133460EA8FFF776FC10220EA904F1BE
:1006A0003C000EF0E6F8C8B1042042E7D4E9091294
:1006B000201D8DE8070004F12C0332460EA8616B63
:1006C000FFF76FFDE9E7606BC1F34401491E006865
:1006D000C84000F0010040F08000D7E720780928EA
:1006E00006D185F800908DF8209033E32870ECE374
:1006F0000920FBE711289AD1204600F08AFE0A283B
:1007000002D1E078C00704D1204600F082FE15280F
:100710008DD100E08DE104F13C00102208F10101CF
:1007200006460EF0D2F820780A2816D0162020703F
:10073000D4E90932606B611D8DE80F0004F15C03A0
:1007400004F16C0247310EA8FFF7C0FC10220EA97D
:1007500030460EF08EF818B1F5E20B20207071E2F1
:100760002046FFF7D5FDA078216A0A18C0F11001D4
:1007700010460EF029F923E3394608A8FFF7A4FD37
:1007800006463BE20228B6D1204600F042FE04288D
:1007900004D3204600F03DFE082809D3204600F08F
:1007A00038FE0E2829D3204600F033FE122824D22A
:1007B000A07D02289FD10E208DF82000686A0D9040
:1007C00098F801008DF82400F0E3022893D1204628
:1007D00000F01FFE002810D0204600F01AFE01286D
:1007E000F9D0204600F015FE0C28F4D004208DF836
:1007F000240098F801008DF825005EE21128FCD154
:10080000002CFAD020781728F7D16178606A022985
:1008100011D0002101EB4101182606EBC101102285
:10082000405808F101010EF050F80520696A00F007
:10083000E3FD2670F1E50121ECE70B28DDD1002C6A
:10084000DBD020781828D8D16078616A02281CD0C3
:100850005FF0000000EB4002102000EBC2000958DE
:10086000B8F8010008806078616A02280FD0002083
:1008700000EB4002142000EBC2000958404650F83B
:10088000032F0A604068486039E00120E2E7012058
:10089000EEE71128B1D1002CAFD020781928ACD1C7
:1008A0006178606A022912D05FF0000101EB41011A
:1008B0001C2202EBC1011022405808F101010EF088
:1008C00004F80520696A00F097FD1A20B6E00121BE
:1008D000ECE7082891D1002C8FD020781A288CD1F1
:1008E000606A98F80120017862F347010170616A3B
:1008F000D8F8022041F8012FB8F8060088800520BA
:10090000696A00F079FD8EE2072012E63878012846
:1009100094D1182204F1140079680EF01BF8E079E4
:10092000C10894F82F0001EAD001E07861F30000DB
:10093000E070217D002974D12178032909D0C007F6
:1009400025D0032028708DF82090686A0D904120F2
:1009500004E3607DA178884201D90620E9E50226FA
:100960002671E179204621F0E001E171617A21F000
:10097000F0016172A17A21F0F001A172FFF7C8FCC9
:100980002E708DF82090686A0D900720E6E2042012
:10099000ACE6387805289DD18DF82000686A0D9066
:1009A000B8680A900720ADF824000A988DF830B096
:1009B0006168016021898180A17A817104202070A1
:1009C000F4E23978052985D18DF82010696A0D91F6
:1009D000391D09AE0EC986E80E004121ADF824107C
:1009E0008DF830B01070A88CD7F80C8080B24026FB
:1009F000A769FFF711FA41463A463346C846CDF893
:100A00000090FEF71EFE002108A8FFF75DFCE078CD
:100A100020F03E00801CE0702078052802D00F20D6
:100A20000CE049E1A07D20B1012802D0032802D0CA
:100A300002E10720BFE584F80080EEE42070ECE4DA
:100A4000102104F15C0002F052FA606BB0BBA07D93
:100A500018B1012801D00520FDE006202870F748D4
:100A60006063A063BEE23878022894D1387908B177
:100A70002875B3E3A07D022802D0032805D022E028
:100A8000B8680028F5D060631CE06078012806D0C3
:100A9000A07994F82E10012805D0E84806E0A17945
:100AA00094F82E00F7E7B8680028E2D06063E07899
:100AB000C00701D0012902D0E04803E003E0F86854
:100AC0000028D6D0A063062010E68DF82090696A31
:100AD0000D91E1784846C90709D06178022903D110
:100AE000A17D29B1012903D0A17D032900D00720D0
:100AF000287031E138780528BBD1207807281ED02E
:100B000084F800A005208DF82000686A0D90B86870
:100B10000A90ADF824A08DF830B003210170E1787F
:100B2000CA070FD0A27D022A1AD000210091D4E971
:100B3000061204F15C03401CFFF725FA67E384F812
:100B40000090DFE7D4E90923211D8DE80E0004F1B0
:100B50002C0304F15C02401C616BFFF722FB56E39F
:100B6000626BC1F34401491E1268CA4002F00101E0
:100B700041F08001DAE738780528BDD18DF82000F2
:100B8000686A0D90B8680A90ADF824A08DF830B06E
:100B9000042100F8011B102204F15C010DF095FE08
:100BA000002108A8FFF790FB2078092801D0132026
:100BB00044E70A2020709BE5E078C10742D0A17D80
:100BC000012902D0022927D038E0617808A801293C
:100BD00016D004F16C010091D4E9061204F15C0313
:100BE000001DFFF7BBFA0A20287003268DF820802D
:100BF000686A0D90002108A8FFF766FBDDE2C3E2FA
:100C000004F15C010091D4E9062104F16C03001D9C
:100C1000FFF7A4FA0026E9E7C0F3440114290DD236
:100C20004FF0006101EBB0104FEAB060E070607807
:100C3000012801D01020BEE40620FFE660780128DC
:100C40003FF4B7AC0A2051E5E178C90708D0A17D8F
:100C5000012903D10B20287004202FE028702DE0FB
:100C60000E2028706078616B012817D004F15C03B6
:100C700004F16C020EA8FFF7E1FA2046FFF748FBEB
:100C8000A0780EAEC0F1100130440DF09DFE06209C
:100C90008DF82000686A09960D909AE004F16C03C3
:100CA00004F15C020EA8FFF7C9FAE9E739780229D6
:100CB00003D139790029D1D029758FE28DF8200030
:100CC000686A0D9058E538780728F6D1D4E90921EB
:100CD0006078012808D004F16C00CDE9000202918F
:100CE00005D104F16C0304E004F15C00F5E704F1C4
:100CF0005C0304F14C007A680646216AFFF764F948
:100D00006078012821D1A078216A0A18C0F1100169
:100D100010460DF059FED4E90923606B04F12D0152
:100D20008DE80F0004F15C0304F16C0231460EA85B
:100D300000E055E2FFF7CAF910220EA904F13C00C9
:100D40000DF097FD08B10B20AFE485F8008000BFDF
:100D50008DF82090686A0D908DF824A00CE5387805
:100D60000528AAD18DF82000686A0D90B8680A900D
:100D7000ADF824A08DF830B080F8008061780129AA
:100D80001AD0D4E9093204F12D01A66B0392009622
:100D9000CDE9011304F16C0304F15C0204F14C0190
:100DA000401CFFF793F9002108A8FFF78DFA60783F
:100DB000012805D0152041E6D4E90923611DE4E7A7
:100DC0000E20287006208DF82000686ACDF824B027
:100DD0000D90A0788DF82800CEE438780328C0D193
:100DE000E079C00770D00F202870072066E73878B8
:100DF00004286BD11422391D04F114000DF0AAFD52
:100E0000616A208CA1F80900616AA078C871E17953
:100E1000626A01F003011172616A627A0A73616A9F
:100E2000A07A81F82400162060E485F800A08DF8EF
:100E30002090696A50460D9190E0000060EE01003C
:100E40003878052842D1B868A8616178606A0229BB
:100E500001D0012100E0002101EB4101142606EB45
:100E6000C1014058082102F042F86178606A022905
:100E700001D0012100E0002101EB410106EBC1019D
:100E8000425802A8E169FFF70DFA6078626A022809
:100E900001D0012000E0002000EB4001102000EB19
:100EA000C1000223105802A90932FEF7F1FF626A5D
:100EB000FD4B0EA80932A169FFF7E3F96178606A7A
:100EC000022904D0012103E042E18BE0BDE00021D2
:100ED00001EB4101182606EBC101A27840580EA98A
:100EE0000DF0F3FC6178606A022901D0012100E075
:100EF000002101EB410106EBC1014058A1780844F3
:100F0000C1F110010DF060FD05208DF82000686A28
:100F10000D90A8690A90ADF824A08DF830B0062194
:100F200001706278616A022A01D0012200E0002289
:100F300002EB420206EBC202401C895810220DF05F
:100F4000C4FC002108A8FFF7BFF91220C5F818B0AB
:100F500028708DF82090686A0D900B208DF8240081
:100F60000AE43878052870D18DF82000686A0D9061
:100F7000B8680A900B20ADF824000A980721017088
:100F80006178626A022901D0012100E0002101EBB1
:100F90004103102101EBC30151580988A0F8011049
:100FA0006178626A022902D0012101E02FE100216B
:100FB00001EB4103142101EBC30151580A6840F8C9
:100FC000032F4968416059E01920287001208DF8ED
:100FD000300077E6162028708DF830B0002108A880
:100FE000FFF772F9032617E114202870B0E638786D
:100FF00005282AD18DF82000686A0D90B8680A90FB
:10100000ADF824A08DF830B080F800906278616A65
:101010004E46022A01D0012200E0002202EB4202E9
:101020001C2303EBC202401C895810220DF04DFC1A
:10103000002108A8FFF748F9152028708DF82060D6
:10104000686A0D908DF824603CE680E038780528C9
:101050007DD18DF82000686A0D90B8680A90ADF8CF
:10106000249009210170616909784908417061691A
:1010700051F8012FC0F802208988C18020781C28EF
:10108000A8D1A1E7E078C00702D04FF0060C01E03C
:101090004FF0070C607802280AD04FF0000000BF24
:1010A00000EB040101F1090105D04FF0010004E05B
:1010B0004FF00100F4E74FF000000B78204413EAF2
:1010C0000C030B7010F8092F02EA0C02027004D115
:1010D0004FF01B0C84F800C0D2B394F801C0BCF1EF
:1010E000010F00D09BB990F800C0E0465FEACC7CCD
:1010F00004D028F001060670102606E05FEA887C1E
:1011000005D528F00206067013262E70032694F8E3
:1011100001C0BCF1020F00D092B991F800C05FEAA3
:10112000CC7804D02CF001060E70172106E05FEA9F
:101130008C7805D52CF002060E701921217000263E
:101140000078D0BBCAB3C3BB1C20207035E012E0CE
:1011500002E03878062841D11A2019E420780128C5
:101160003CD00C283AD02046FFF7F0F809208DF843
:101170002000686A0D9031E03878052805D00620F7
:10118000387003261820287046E005218DF82010BD
:10119000686A0D90B8680A900220ADF8240001201A
:1011A0008DF830000A980170297D4170394608A8F1
:1011B000FFF78AF8064618202870012E0ED02BE083
:1011C00001208DF82000686A0D9003208DF824001E
:1011D000287D8DF8250085F814B012E0287D80B1B7
:1011E0001D202070172028708DF82090686A0D90BF
:1011F00002208DF82400394608A8FFF765F8064656
:101200000AE00CB1FE2020709DF8200020B10021E2
:1012100008A8FFF759F810E413B03046BDE8F08F86
:101220002DE9F04387B00C464E6900218DF804107B
:1012300001202578034602274FF007094FF0050CDF
:1012400085B1012D53D0022D39D1FE2030708DF89B
:101250000030606A059003208DF80400207E8DF830
:10126000050063E02179012925D002292DD0032929
:1012700028D0042923D1B17D022920D131780D1F36
:10128000042D04D30A3D032D01D31D2917D1218933
:10129000022914D38DF80470237020899DF804105E
:1012A00088421BD2082001E058EE01008DF80000B2
:1012B000606A059057E070780128EBD0052007B0F0
:1012C000BDE8F0831D203070E4E771780229F5D184
:1012D00031780C29F3D18DF80490DDE7083402F859
:1012E00004CB94E80B0082E80B000320E7E71578B5
:1012F000052DE4D18DF800C0656A059595680295C5
:101300008DF8101094F80480B8F1010F13D0B8F1E3
:10131000020F2DD0B8F1030F1CD0B8F1040FCED1BD
:10132000ADF804700E202870207E68700021684699
:10133000FEF7CAFF0CE0ADF804700B202870207E89
:10134000002100F01F0068706846FEF7BDFF37708F
:101350000020B4E7ADF804708DF8103085F800C0B7
:10136000207E6870277011466846FEF7ADFFA6E73D
:10137000ADF804902B70207F6870607F00F0010052
:10138000A870A07F00F01F00E870E27F2A71C007FC
:101390001CD094F8200000F00700687194F8210038
:1013A00000F00700A87100216846FEF78DFF28684D
:1013B000F062A8883086A87986F83200A069407863
:1013C00070752879B0700D203070C1E7A97169710E
:1013D000E9E700B587B005280CD101208DF80000A1
:1013E0008DF80400002005918DF80500014668463F
:1013F000FEF76AFF07B000BD70B50C46054602F067
:101400004FF821462846BDE870407823002201F0BD
:101410009DBF08B1007870470C20704770B50C0074
:1014200005784FF000010CD021702146F2F793F9B6
:1014300069482178405D884201D1032070BD0220B7
:1014400070BDF2F788F9002070BD0279012A05D03D
:1014500000220A704B78012B02D003E00420704771
:101460000A758A6102799300521C0271C1500320EF
:101470007047F0B587B00F4605460124287905EB83
:10148000800050F8046C7078411E02290AD252493B
:101490003A46083901EB8000314650F8043C2846B2
:1014A000984704460CB1012C11D12879401E10F048
:1014B000FF00287101D00324E0E70A208DF8000026
:1014C000706A0590002101966846FFF7A7FF032C7C
:1014D000D4D007B02046F0BD70B515460A46044684
:1014E00029461046FFF7C5FF064674B12078FE284E
:1014F0000BD1207C30B100202870294604F10C006B
:10150000FFF7B7FF2046FEF721FF304670BD70475A
:1015100070B50E4604467C210DF078FA0225012EA6
:1015200003D0022E04D0052070BD0120607000E0C1
:1015300065702046FEF70AFFA575002070BD28B132
:10154000027C1AB10A4600F10C01C5E70120704780
:1015500010B5044686B0052001F0A2FF2078FE28D1
:1015600006D000208DF8000069462046FFF7E7FF0F
:1015700006B010BD7CB50E4600218DF804104178F0
:10158000012903D0022903D0002405E0046900E00A
:1015900044690CB1217C89B16D4601462846FFF7AC
:1015A00054FF032809D1324629462046FFF794FF0D
:1015B0009DF80410002900D004207CBD04F10C0526
:1015C000EBE730B40C460146034A204630BC034BDF
:1015D0000C3AFEF756BE00009CEE010058EE0100EA
:1015E00070B50D46040011D085B1210128460DF0DB
:1015F000EBF910224E4928460DF067F94C480121BD
:101600000838018044804560002070BD012070BD15
:1016100070B5474E00240546083E10E07068AA7B6E
:1016200000EB0410817B914208D1C17BEA7B91429F
:1016300004D10C2229460DF01CF930B1641C30880D
:101640008442EBDB4FF0FF3070BD204670BD70B5BB
:101650000D46060006D02DB1FFF7DAFF002803DBA8
:10166000401C14E0102070BD314C083C208862887A
:10167000411C914201D9042070BD6168102201EB28
:10168000001031460DF021F92088401C2080287080
:10169000002070BD70B514460D0018D0BCB10021FB
:1016A000A170022802D0102811D105E0288870B15D
:1016B0000121A170108008E02846FFF7A9FF00284B
:1016C00005DB401CA070A8892080002070BD01208F
:1016D00070BD70B5054614460E000BD0002030706A
:1016E000A878012808D005D91149A1F108010A8874
:1016F00090420AD9012070BD24B128782070288832
:10170000000A5070022008700FE064B1496810228E
:1017100001EB0011204610390DF0D7F8287820731E
:101720002888000A607310203070002070BD00000F
:101730007C0000202DE9F04190460C46074600252C
:10174000FE48072F00EB881607D2DFE807F00707EF
:10175000070704040400012500E0FFDF06F8147009
:10176000002D13D0F548803000EB880191F8270058
:10177000202803D006EB4000447001E081F82640A9
:1017800006EB44022020507081F82740BDE8F0812C
:10179000F0B51F4614460E460546202A00D1FFDF4D
:1017A000E649E648803100EB871C0CEB440001EB76
:1017B0008702202E07D00CEB460140784B7848700A
:1017C000184620210AE092F82530407882F825005A
:1017D000F6E701460CEB410005704078A142F8D1D4
:1017E00092F82740202C03D00CEB4404637001E0F6
:1017F00082F826300CEB41042023637082F8271016
:10180000F0BD30B50D46CE4B44190022181A72EBCC
:10181000020100D2FFDFCB48854200DDFFDFC9486F
:101820004042854200DAFFDFC548401C844207DAA7
:10183000002C01DB204630BDC148401C201830BDC3
:10184000BF48C043FAE710B504460168407ABE4A73
:1018500052F82020114450B10220084420F07F406B
:10186000F9F78FFC94F90810BDE81040C9E704208F
:10187000F3E72DE9F047B14E803696F82D50DFF8AA
:10188000BC9206EB850090F8264034E009EB851702
:101890004FF0070817F81400012806D004282ED0AE
:1018A00005282ED0062800D0FFDF01F0E3F801461E
:1018B00007EB4400427806EB850080F8262090F87C
:1018C0002720A24202D1202280F82720084601F0DA
:1018D000DCF82A4621460120FFF72CFF9B484146B1
:1018E00000EB041002682046904796F82D5006EB56
:1018F000850090F82640202CC8D1BDE8F087022052
:1019000000E003208046D0E710B58C4C20218034C5
:1019100084F8251084F8261084F82710002084F815
:10192000280084F82D0084F82E10411EA16044F890
:10193000100B2074607420736073A0738449E07787
:1019400020750870487000217C4A103C02F8110094
:10195000491CC9B22029F9D30120F9F700FB002066
:10196000F9F7FDFA012084F82200F9F79DFF794884
:10197000F9F7A9FF764CA41E20707748F9F7A3FF6A
:101980006070BDE81040F9F777BA10B5F9F799FA29
:101990006F4CA41E2078F9F7AFFF6078F9F7ACFF21
:1019A000BDE8104001F09EB8202070472DE9F34FAC
:1019B000624E0025803606EB810A89B09AF8250030
:1019C000202822D0691E02916049009501EB001089
:1019D0008146D0E90112C0680391CDE90420B08BA3
:1019E000ADF81C00B07F8DF81E009DF81500C8B141
:1019F0000227554951F820400399E219114421F07A
:101A00007F41019184B102210FE00120F9F7A7FA8B
:101A10000020F9F7A4FAF9F772FA01F063F886F8F2
:101A20002F50A0E00427E4E700218DF818100228C9
:101A300001D0012820D10398391901440998081AC6
:101A40009DF81C1020F07F4001B10221333181420A
:101A50000BD203208DF815000398C4F13201401A0F
:101A600020F07F40322403900CE096F8240018B94F
:101A700001F0A0F900284CD0322C03D214B101F0AF
:101A800025F801E001F02EF8314A107818B393469A
:101A90005278039B121B00219DF81840984601289C
:101AA0001AD0032818D000208DF81E00002A04DD6B
:101AB000981A039001208DF818009DF81C0000B1C1
:101AC00002210398254A20F07F40039003AB099838
:101AD00001F014F810B110E00120E5E79DF81D00B9
:101AE00018B99BF80000032812D08DF81C50CDF8CF
:101AF0000C808DF818408DF81E509DF8180058B1D4
:101B000003980123C11900221846F9F77BFA06E071
:101B100000200BB0BDE8F08F0120F9F720FA99F909
:101B20000C20012300200199F9F76CFA012086F8B6
:101B30002F008AF828502022694611E06C08002006
:101B4000FF7F841E0020A107ACEE01006C06002080
:101B50008E000020FB31010073180100FFFF3F00E1
:101B6000F9480CF0F7FE0120D3E72DE9F05FDFF82C
:101B7000D883064608EB860090F82550202D1FD00C
:101B8000A8F180002C4600EB8617A0F50079DFF85D
:101B9000BCB305E0A24607EB4A004478202C0AD0EB
:101BA000F9F77CFA09EB04135A4601211B1D00F0DA
:101BB000A5FF0028EED0AC4202D0334652461EE0CC
:101BC000E34808B1AFF30080F9F768FA98F82F20DE
:101BD0006AB1D8F80C20411C891A0902CA1701EB16
:101BE00012610912002902DD0020BDE8F09F314694
:101BF000FFF7DCFE08B10120F7E733462A46202133
:101C00000420FFF7C5FDEFE72DE9F041CE4C256933
:101C1000F9F744FA401B0002C11700EB11600012F3
:101C200000D4FFDF94F8220000B1FFDF012784F821
:101C3000227094F82E00202800D1FFDF94F82E6047
:101C4000202084F82E00002584F82F5084F820509E
:101C500084F82150BF4825600078022833D003283B
:101C600031D000202077A068401C05D04FF0FF3015
:101C7000A0600120F9F773F90020F9F770F9F9F77E
:101C80006EFAF9F766FAF9F73AF90CF02BF9B2485F
:101C9000056005604FF0E0214FF40040B846C1F800
:101CA0008002F1F776F994F82D703846FFF75DFF62
:101CB0000028FAD0A448803800EB871010F81600EE
:101CC000022802D006E00120CCE73A463146062041
:101CD000FFF730FD84F8238004EB870090F826009E
:101CE000202804D09B48801E4078F9F70BFE207F07
:101CF000002803D0F9F723FA2577657746E50146F2
:101D0000914810B590F82D200024803800EB821007
:101D100010F814302BB1641CE4B2202CF8D320202E
:101D200010BD8E4800EB0410016021460120FFF732
:101D300001FD204610BD10B5012801D0032800D1B7
:101D400071B3814A92F82D307F4C0022803C04EB25
:101D5000831300BF13F812400CB1082010BD521CB1
:101D6000D2B2202AF6D37B4A48B1022807D00729ED
:101D700016D2DFE801F01506080A0C0E100000214B
:101D80000AE01B2108E03A2106E0582104E077210F
:101D900002E0962100E0B52151701070002010BDC6
:101DA000072010BD6B4810B54078F9F7EAF980B20A
:101DB00010BD10B5202811D2634991F82D30A1F142
:101DC000800202EB831414F810303BB191F82D30EF
:101DD00002EB831212F81020012A01D0002010BD5E
:101DE00091F82D2001460020FFF7A4FC012010BD32
:101DF00010B5F9F753F9BDE81040F9F7C2B92DE96C
:101E0000F0410E46504F01782025803F0C4607EBED
:101E1000831303E0254603EB45046478944202D023
:101E2000202CF7D108E0202C06D0A14206D103EBEC
:101E300041014978017007E00020A7E403EB44006A
:101E400003EB450140784870454F7EB127B1002132
:101E500040F2DA30AFF300803078A04206D127B1EB
:101E6000002140F2DD30AFF30080357027B1002152
:101E700040F2E230AFF30080012087E410B5426801
:101E80000B689A1A1202D41702EB1462121216D4BB
:101E9000497A91B1427A82B9324A006852F82110E7
:101EA000126819441044001D891C081A0002C11749
:101EB00000EB11600012322801DB012010BD002070
:101EC00010BD2DE9F04781461F48244E00EB8100EC
:101ED000984690F825402020107006F500701546B1
:101EE00000EB81170BE000BF06EB04104946001D14
:101EF000FFF7C4FF28B107EB44002C704478202C76
:101F0000F2D1297888F8001013E000BF06EB041521
:101F1000291D4846FFF7B2FF68B988F80040A97B41
:101F200099F80A00814201D80020E6E407EB44005A
:101F30004478202CEAD10120DFE42DE9FC410E4653
:101F400007460024054D18E0EC080020FFFF3F0085
:101F5000000000008E00002000F500406C0600200C
:101F600000000000ACEE01009DF8000005EB001041
:101F70008168384600F0D6FD01246B4601AA31463F
:101F80003846FFF79EFF0028EED02046BDE8FC81D2
:101F900070B50446FF480125A54300EB841100EB12
:101FA000851040220CF091FCFB4E26B1002140F23E
:101FB0005C40AFF30080F748803000EB850100EB18
:101FC0008400D0F82500C1F8250026B100214FF487
:101FD0008C60AFF30080284670BD2DE9FC4184463B
:101FE000EC481546089C00EB85170E4617F81400C0
:101FF000012803D0022801D00020C7E70B46E74A9A
:102000000121604600F07AFDA8B101AB6A4629467D
:102010003046FFF756FF70B1DE489DF804209DF86A
:102020000010803000EB85068A4208D02B46052040
:10203000FFF7AEFB0BE02A462146042014E02029DE
:1020400003D007EB4100407801E096F8250007EB4C
:10205000440148709DF80000202809D007EB40009B
:1020600044702A4621460320FFF764FB01208DE7D8
:1020700006F8254F0120F070F3E7C94901EB001085
:10208000001DFFF7E0BB7CB51D46134604460E4617
:1020900000F1080221461846F9F780F894F9080083
:1020A0000F2804DD1F3820722068401C206096B184
:1020B0000220BC4951F82610461820686946801B4A
:1020C00020F07F40206094F908002844C01C1F289D
:1020D00003DA012009E00420EBE701AAF9F75EF832
:1020E0009DF8040010B10098401C009000992068F1
:1020F00031440844C01C20F07F4060607CBD2DE965
:10210000FE430C460646097860799072207998461D
:102110001546507241B19F48803090F82E1020290A
:102120000AD00069401D0BE0D4E90223217903B0F5
:102130002846BDE8F043A6E79B484178701D084457
:1021400020F07F47217900222846A368FFF79BFFF4
:102150003946284600F0E6FCD4E902322179684687
:10216000FFF791FF41462846019CFFF7E6FE2B460C
:1021700022460021304600F0C1FC002803D1314640
:10218000284600F0CFFCBDE8FE832DE9FE4F8146D6
:1021900000F084FC30B1002799F8000020B1002045
:1021A000BDE8FE8F0127F7E77A4D7B4C4FF0000A20
:1021B000803524B1002140F2D340AFF3008095F880
:1021C0002D8085F823A0002624B100214FF49B60C8
:1021D000AFF300801FB94046FFF7DAFE804624B116
:1021E00000214FF49C60AFF30080F8F757FF43469F
:1021F0006A464946FFF783FF24B1002140F2E640DA
:10220000AFF3008095F82E0020280CD029690098A3
:10221000401A0002C21700EB1260001203D5684694
:1022200000F080FC012624B100214FF49E60AFF342
:10223000008095F823000028BBD124B1002140F292
:10224000F640AFF30080F8F729FF6B46534A0021B0
:1022500000F054FC0028A3D027B941466846FFF798
:102260006CFE064326B16846FFF7EDFAC9F8080090
:1022700024B1002140F20950AFF3008001208FE724
:102280002DE9FF5F8A46814600F008FC414C80340E
:1022900010B39AF80000002710B1012800D0FFDF2A
